:100000000C943B2F0C9440320C946B320C9496322F
:100010000C94C1320C94EC320C9417330C94423390
:100020000C946D330C946C2F0C946C2F0C946C2FDF
:100030000C946C2F0C946C2F0C946C2F0C946C2FD4
:100040000C946C2F0C94F6C80C946C2F0C946C2FA1
:100050000C946C2F0C946C2F0C94FFBB0C946E2F93
:100060000C946C2F0C94AFA70C945BA80C946C2F81
:100070000C946C2F0C946C2F0C946C2F0C946C2F94
:100080000C946C2F0C946C2F0C946C2F0C946C2F84
:100090000C946C2F0C946C2F0C946C2F0C946C2F74
:1000A0000C946C2F0C946C2F0C946C2F0C946C2F64
:1000B0000C946C2F0C946C2F0C946C2F0C946C2F54
:1000C0000C946C2F0C946C2F0C946C2F0C946C2F44
:1000D0000C946C2F0C946C2F0C946C2F0C946C2F34
:1000E0000C946C2FB630BB30C030CA30D4304D3198
:1000F000DE30E630EE30F83002310C311B31253184
:100100004D312F31393143317131743163316731C0
:100110006D31AB3178317C31823186318A31903129
:1001200094319831AB319E31A231A631B5679567D4
:100130009B6798679E67A167A467B067A767C26758
:10014000AA67AD67F5A4F3A417A514A512A549A540
:1001500046A544A5A2A570A56DA56BA5E2A7E8A735
:10016000F9A704A80CA821A810A821A814A818A8C9
:1001700021A81EA8084AD73B3BCE016E84BCBFFD18
:10018000C12F3D6C74319ABD56833DDA3D00C77F67
:1001900011BED9E4BB4C3E916BAAAABE0000008000
:1001A0003F05A84CCDB2D44EB93836A9020C50B98F
:1001B000918688083CA6AAAA2ABE000000803F00BB
:1001C0000D94BD540D94B34F0D94BF050D949840FC
:1001D0004E414E494E495459494E46CDCCCC3D0A2C
:1001E000D7233C17B7D13877CC2B329595E6241F0F
:1001F000B14F0A000020410000C84200401C4620C8
:10020000BCBE4CCA1B0E5AAEC59D7400407A10F39A
:100210005A00A0724E18090010A5D4E80000E87634
:1002200048170000E40B54020000CA9A3B0000008B
:10023000E1F505000080969800000040420F0000A4
:1002400000A08601000000102700000000E8030065
:100250000000006400000000000A0000000000012F
:1002600000000000002C76D888DC674F0823DFC12F
:10027000DFAE59E1B1B796E5E3E453C63AE65199EA
:100280007696E8E6C28426EB898C9B62ED407C6F13
:10029000FCEFBC9C9F40F2BAA56FA5F490055A2ACA
:1002A000F75C936B6CF9676DC11BFCE0E40D47FED6
:1002B000F520E6B500D0ED902E03009435770500CB
:1002C00080841E080000204E0A000000C80C333352
:1002D00033330F986E12831141EF8D2114893BE661
:1002E0005516CFFEE6DB18D1844B381BF77C1D90EA
:1002F0001DA4BBE424203284725E228100C9F12453
:10030000ECA1E53D2700000A0B02090C0D0E0807C1
:1003100003040100000000000000000000000000D5
:1003200000000000000000000000000000000000CD
:10033000001211100000000000000000000000008A
:10034000000000000000000000000001021020205A
:100350000808102040102040800201020108040219
:10036000010102040810204080804020100804028F
:1003700001800402018040201008040201080402E8
:1003800001010204081020408001020408102040EE
:100390008005050505070508080808020202020A8B
:1003A0000A08080404040401010101010101010318
:1003B00003030303030303040707070C0C0C0C0CD3
:1003C0000C0C0C0202020206060606060606060BC6
:1003D0000B0B0B0B0B0B0B0000200023002600293E
:1003E000002C002F0032000001000003010601096B
:1003F0000100002200250028002B002E00310034CF
:100400000002010000050108010B01000021002489
:100410000027002A002D00300033000101000004F5
:100420000107010A0101060D00FE09016602D6203E
:10043000FFFE0BFE0AFE0D0060221969808080809D
:100440008080800080183363A0A0A00357675050BD
:10045000F850F850500259692078A0A0702828F070
:100460002002596948A85010204050A890025868AE
:1004700040A0A040A0989068281363808080113B22
:100480006B2040408080808080404020113B6B800A
:100490004040202020202040408006556520A87044
:1004A000A8200455652020F8202011336360408087
:1004B000065161F811336340E040025969080810A1
:1004C00010204040808002596920508888888888A0
:1004D00050200259692060A02020202020F80259D5
:1004E000697088880810204080F8025969F808105F
:1004F000207008088870025969101030505090F828
:100500001010025969F88080B0C808088870025934
:100510006970888080F088888870025969F80810AE
:10052000102020404040025969708888887088886F
:10053000887002596970888888780808887011382E
:100540006840E040000040E04011386840E0400072
:100550000060408002596908102040804020100847
:10056000045464F80000F802596980402010081013
:1005700020408002596970888808102020002002DD
:10058000596970888898A8A8B08078025969205065
:10059000888888F8888888025969F04848487048EF
:1005A0004848F00259697088808080808088700295
:1005B0005969F048484848484848F0025969F88065
:1005C0008080F0808080F8025969F8808080F08017
:1005D0008080800259697088808080988888700245
:1005E000596988888888F888888888123969E0403D
:1005F000404040404040E00259693810101010104F
:10060000109060025969888890A0C0A090888802E4
:1006100059698080808080808080F802596988884C
:10062000D8A8A88888888802596988C8C8A8A898BE
:1006300098888802596970888888888888887002B4
:100640005969F0888888F080808080015A6A7088B3
:100650008888888888A87008025969F0888888F096
:10066000A090888802596970888080700808887016
:10067000025969F820202020202020200259698872
:10068000888888888888887002596988888888500E
:100690005050202002596988888888A8A8A8A850A6
:1006A00002596988885050205050888802596988BA
:1006B0008850502020202020025969F8081010206E
:1006C000404080F8113B6BE080808080808080809B
:1006D00080E0025969808040402010100808113BDA
:1006E0006BE0202020202020202020E008536320E1
:1006F0005088015161F82A226280400256667008D3
:1007000078889868025969808080F088888888F0A5
:1007100002566670888080887002596908080878D7
:1007200088888888780256667088F88088700259B0
:100730006930484040F04040404000586870888828
:100740008878088870025969808080B0C888888855
:10075000881238684000C040404040E0004A6A10BB
:1007600000301010101090906002596980808090C5
:10077000A0C0A09088123969C0404040404040402D
:10078000E0025666D0A8A8A8A888025666B0C88815
:10079000888888025666708888888870005868F053
:1007A000888888F0808080005868788888887808F1
:1007B0000808025666B0C88080808002566670883D
:1007C000601088700258684040F040404048300255
:1007D0005666888888889868025666888888505047
:1007E000200256668888A8A8A8500256668850201D
:1007F0002050880058688888889868088870025651
:1008000066F810204080F8015B6B1820202020C083
:10081000202020201822196980808080808080809C
:1008200080015B6BC0202020201820202020C008E1
:10083000536348A890FFFFFFFFFFFFFFFFFFFFFF8D
:10084000FFFFFFFFFFFFFFFFFFFFFFFFFFFFFFFFB8
:10085000FFFFFFFFFFFF0D0060221969800080800D
:1008600080808080800358682070A8A0A0A8702095
:1008700002596930484040E0404048B0035666881D
:10088000705050708802596988885050F820F820BC
:1008900020221969808080800080808080124A6ACE
:1008A000609080609090601090601A3262A0A00307
:1008B00059697088A8D8C8D8A88870045767700884
:1008C00078887800F80356662850A0A05028045372
:1008D00063F80808163161E00359697088E8D8D8D0
:1008E000E8D888700A5161F81744646090906003FA
:1008F00057672020F8202000F807356540A02040E9
:10090000E007356540A04020C02A226240800058A0
:10091000688888888898E8808002596978E8E8E8DB
:10092000E868282828262161C020226240800735F7
:100930006540C04040E0045767708888887000F8C0
:10094000035666A050282850A0025A6A40C0404072
:10095000E00818283808025A6A40C04040E01028D1
:10096000081038025A6A40A04020A04818283808C9
:10097000025969200020204080888870025A6A400D
:10098000200020508888F88888025A6A10200020A9
:10099000508888F88888025A6A3048002050888831
:1009A000F88888025A6A28500020508888F8888879
:1009B000025A6A50500020508888F88888025A6A83
:1009C00020502020508888F8888802596958A0A0B3
:1009D000A0B0E0A0A0B8005B6B70888080808080B1
:1009E00088702040025A6A402000F88080F08080A1
:1009F000F8025A6A102000F88080F08080F8025ACD
:100A00006A304800F88080F08080F8025A6A5050BE
:100A100000F88080F08080F8123A6A804000E04060
:100A200040404040E0123A6A204000E040404040F0
:100A300040E0124A6A609000E04040404040E012CE
:100A40003A6AA0A000E04040404040E0025969F00E
:100A5000484848E8484848F0025A6A2850008888C0
:100A6000C8A8988888025A6A4020007088888888B8
:100A70008870025A6A1020007088888888887002FE
:100A80005A6A30480070888888888870025A6A28B4
:100A9000500070888888888870025A6A50500070A8
:100AA0008888888888700355658850205088015B45
:100AB0006B08709898A8A8A8C8C87080025A6A40A5
:100AC000200088888888888870025A6A10200088E8
:100AD000888888888870025A6A30480088888888A0
:100AE000888870025A6A5050008888888888887080
:100AF000025A6A102000888850202020200259695C
:100B000080F0888888F0808080025969609090A089
:100B1000A0908888B00259694020007008788898B1
:100B2000680259691020007008788898680259692D
:100B30003048007008788898680259692850007019
:100B40000878889868025969505000700878889829
:100B500068025A6A304830007008788898680256EF
:100B600066702870A0A850005868708880808870CF
:100B700020400259694020007088F880887002592E
:100B8000691020007088F880887002596930480028
:100B90007088F88088700259695050007088F88019
:100BA0008870123969804000C040404040E01239EE
:100BB00069204000C040404040E012496960900018
:100BC000C040404040E0123969A0A000C040404011
:100BD00040E0025A6A50206010708888888870024D
:100BE0005969285000B0C88888888802596940200F
:100BF0000070888888887002596910200070888881
:100C00008888700259693048007088888888700226
:100C10005969285000708888888870025969505036
:100C200000708888888870035767202000F80020AB
:100C300020015868087098A8A8C8708002596940B7
:100C40002000888888889868025969102000888860
:100C50008888986802596930480088888888986828
:100C6000025969505000888888889868005B6B102A
:100C700020008888889868088870005A6A8080B048
:100C8000C88888C8B08080005B6B50500088888816
:100C9000986808887001050700FE0500FB01F22036
:100CA000FFFE05FE05FE0200400215258080800043
:100CB00080053242A0A002556550F850F850014618
:100CC000562070C030E02002556590102040480248
:100CD0005565608068906805122280800225354045
:100CE000808080400225358040404080043343A00E
:100CF00040A003334340E0400122324080043141B0
:100D0000E0021121800255650810204080024555FF
:100D10006090909060022535C040404040024555AB
:100D2000E0106080F0024555E0106010E00245558B
:100D30002060A0F020024555F080E010E00245550B
:100D40006080E09060024555F0102040400245551B
:100D500060906090600245556090701060031323AE
:100D6000800080021424800080800235452040806D
:100D70004020033343E000E00235458040204080BE
:100D8000024555E0106000400255657088B8A870B3
:100D9000024555609090F090024555E090E090E05B
:100DA0000235456080808060024555E0909090E07B
:100DB000023545E080E080E0023545E080E080805B
:100DC0000245557080B090700245559090F090901B
:100DD000023545E0404040E002455530101090603B
:100DE00002455590A0C0A09002354580808080E0EB
:100DF00002556588D8A8888802455590D0B0909053
:100E00000245556090909060024555E09090E080DA
:100E1000014656609090906010024555E09090E039
:100E20009002455570806010E0023545E04040403A
:100E30004002455590909090600245559090A0A03A
:100E40004002556588A8A8A850024555909060902A
:100E5000900245559090701060023545E02040802A
:100E6000E0022535C0808080C0025565804020109A
:100E700008022535C0404040C005324240A0024132
:100E800051F0052232804002445470909070024527
:100E90005580E09090E002344460808060024555C7
:100EA000107090907002445460B0C06002354520CC
:100EB00040E04040004656709090701060024555EA
:100EC00080E0909090021525800080808000273778
:100ED000400040404040800245558090A0E0900294
:100EE00015258080808080025464F0A8A8A8024460
:100EF00054E090909002445460909060004656E018
:100F00009090E080800046567090907010100234EF
:100F100044A0C0808002445470C030E00235454097
:100F2000E0404020024454909090700244549090CD
:100F3000A040025464A8A85050023444A04040A0ED
:100F4000004656909090701060024454F02040F09B
:100F50000235456040804060021525808080808099
:100F6000023545C0402040C005425250A0FFFFFF5F
:100F7000FFFFFFFFFFFFFFFFFFFFFFFFFFFFFFFF81
:100F8000FFFFFFFFFFFFFFFFFFFFFFFFFFFF02006D
:100F900040FFFFFFFFFFFFFFFFFFFFFFFFFFFFFF20
:100FA000FFFFFFFFFFFFFFFFFFFFFFFFFFFFFFFF51
:100FB000FFFFFFFFFFFFFFFFFFFFFFFFFFFFFFFF41
:100FC000FFFFFFFFFFFFFFFFFFFFFFFFFFFFFFFF31
:100FD000FFFFFFFFFFFFFFFFFFFFFFFFFFFFFFFF21
:100FE000FFFFFFFFFFFFFFFFFFFFFFFFFFFFFFFF11
:100FF00001050800FF060121023520FFFF07FF065B
:10100000FF090050221656808080800080153353DF
:10101000A0A0A00257575050F850F8505002575710
:101020002070A07028702013355580A040A02002A9
:10103000475740A0A040A0A05025135380808012A5
:101040002656408080808040122656804040404096
:10105000800245559060F060900255552020F820A0
:1010600020113353604080044151F011335340E06C
:101070004002465610102040808012365640A0A0F4
:10108000A0A04012365640C0404040E002465660A4
:1010900090106080F0024656F0206010906002468A
:1010A000562060A0F02020024656F080E0109060AC
:1010B0000246566080E0909060024656F010202074
:1010C00040400246566090609090600246566090A4
:1010D00090701060122555C0C000C0C01136566017
:1010E00060006040801236562040808040200343DC
:1010F00053F000F0123656804020204080123656C1
:1011000040A020400040015858304898A8A890407E
:1011100030024656609090F09090024656E090E083
:101120009090E0024656609080809060024656E0C3
:1011300090909090E0024656F080E08080F0024669
:1011400056F080E0808080024656609080B09060CB
:101150000246569090F0909090123656E0404040F3
:1011600040E002465670202020A04002465690A043
:10117000C0A0A0900246568080808080F002465633
:1011800090F0F090909002465690D0F0B0B090025F
:101190004656609090909060024656E09090E080B5
:1011A00080014757609090D0B06010024656E090A2
:1011B00090E0909002465660904020906012365623
:1011C000E04040404040024656909090909060022F
:1011D0004656909090906060024656909090F0F045
:1011E00090024656909060609090025656888850C3
:1011F000202020024656F010204080F0123656E0A3
:1012000080808080E0024656808040201010123698
:1012100056E020202020E016325240A0014151F03B
:1012200016225280400244547090907002465680BC
:1012300080E09090E0123454608080600246561046
:10124000107090907002445460B0C0600246562006
:101250005040E04040014555609070106002465695
:101260008080E09090901236564000C04040E011DF
:1012700037572000202020A040024656808090E072
:101280009090123656C040404040E0025454D0A8DE
:10129000A8A8024454E0909090024454609090605A
:1012A000014555E090E08080014555709070101028
:1012B000024454A0D0808012345460C020C0024642
:1012C000564040E0405020024454909090701234B8
:1012D00054A0A0A04002545488A8A850024454909E
:1012E0006060900145559090709060024454F020E9
:1012F00040F0024757304020C02040302216568030
:101300008080808080024757C02040304020C00647
:10131000425250A0FFFFFFFFFFFFFFFFFFFFFFFF55
:10132000FFFFFFFFFFFFFFFFFFFFFFFFFFFFFFFFCD
:10133000FFFFFFFFFF0900502216568000808080CB
:10134000800146562070A0A070200246562050E032
:101350004050A002555588705070880256568850EB
:10136000F820F82022175780808000808080024774
:10137000577080E0907010E0173151A002565670FF
:10138000A8C8C8A87014355560A06000E003435396
:1013900050A050123353E02020143151E002565631
:1013A00070E8D8E8D870173151E015335340A040A9
:1013B00012355540E04000E014355540A02040E093
:1013C000143555C020C020C016225240800145551A
:1013D000909090E08002565678E8E868282824111A
:1013E0005180112252408014355540C04040E014D5
:1013F000355540A04000E0034353A050A00247579A
:10140000808080A060F0200247578080A0D010200C
:101410007002475780408060A0F02012365640008E
:101420004080A04002475740206090F090900247D3
:101430005720406090F0909002475760906090F085
:10144000909002475750A06090F0909002475790BC
:10145000006090F0909002475760906090F09090FC
:1014600002465670A0A0F0A0B0014757609080805F
:101470009060400247574020F080E080F0024757DC
:101480002040F080E080F00247576090F080E080DC
:10149000F00247579000F080E080F012375780400C
:1014A000E0404040E01237572040E0404040E0122A
:1014B000375740A0E0404040E0123757A000E040DE
:1014C0004040E00256567048E8484870024757507E
:1014D000A090D0B0909002475740206090909060CC
:1014E000024757204060909090600247576090609C
:1014F0009090906002475750A06090909060024793
:101500005790006090909060123353A040A0024624
:101510005670B0B0D0D0E0024757402090909090E5
:10152000600247572040909090906002475760902B
:101530009090909060024757900090909090600239
:1015400057571020885020202002465680E0909067
:10155000E0800246566090A0A090A002475740202D
:101560000070909070024757204000709090700279
:1015700047572050007090907002475750A000705D
:1015800090907002465650007090907002475760DD
:10159000906070909070025454F068B07811355596
:1015A000608080604002475740200060B0C0600209
:1015B000475720400060B0C060024757609000600D
:1015C000B0C060024656500060B0C060123757800D
:1015D0004000C04040E0123757204000C04040E08B
:1015E00012375740A000C04040E0123656A000C05D
:1015F0004040E0024757A040A0107090600247575B
:1016000050A000E0909090024757402000609090DA
:1016100060024757204000609090600247576090FA
:10162000006090906002475750A000609090600268
:1016300046569000609090601235554000E00040A2
:1016400002445470B0D0E002475740200090909080
:10165000700247572040009090907002475760906A
:1016600000909090700246569000909090700148C3
:101670005820400090907090600147578080E09023
:10168000E08080014757900090907090602020206B
:101690002000202020202020200025753A253032EF
:1016A0007500253032753A25303275002575642075
:1016B000253032753A25303275003FFFF038007022
:1016C0003186302387102787902F87D02F03D02093
:1016D00030102078102078102030102F03D02F8762
:1016E000D02787902387103186303800703FFFF075
:1016F0003FFFF038007030FC3020FC1020781020C4
:1017000030102C00D02E31D02F7BD02F7BD02E311B
:10171000D02C00D020301020781020FC1030FC306D
:101720003800703FFFF00410400208200208200437
:101730001040082080104100104100082080041053
:10174000400000001FFFF81FFFF81FFFF81FFFF801
:101750001FE020102010201010201020201020103A
:1017600030300840048003001FE03FF03FF03FF0BE
:101770001FE01FE03FF03FF03FF00FC00780030085
:101780004572723A207574663820666F6E74206EEA
:101790006F7420696E697469616C697A65642E0082
:1017A0004572723A207574663820666F6E74206ECA
:1017B0006F7420696E697469616C697A65642E0062
:1017C0004572723A207574663820666F6E74206EAA
:1017D0006F7420696E697469616C697A65642E0042
:1017E000506C656173652052657365740050524991
:1017F0004E5445522048414C54454400687474701E
:101800003A2F2F6D61726C696E66772E6F7267006A
:10181000322E302E302E313734007F80FFC0FFC093
:10182000FFC07F807F80FFC0FFC0FFC03F001E0061
:101830000C00FFFFFF0E000E000E000E000E000E4B
:10184000000E000E007FC03F801F000E0004000449
:10185000000E001F003F807FC00E000E000E000E25
:10186000000E000E000E000E0000FE0003FF8007B9
:1018700083C00E01C00E00E01C00E07F00E03E00CF
:10188000E01C00E00800E00000E00001C00E01C024
:101890000F078007FF0001FC0001FC0007FF000F9D
:1018A00007800E01C00001C00000E00800E01C003D
:1018B000E03E00E07F00E01C00E00E00E00E01C012
:1018C0000783C003FF8000FE00000C0D00FE07022E
:1018D0002603BC017FFE08FE08FE0508080600007E
:1018E00040F0C88888987810050808060000C0F8FD
:1018F0008888888888F80505050600012030F830BA
:10190000200508080600002070F820202020E005AF
:1019100009090600FF2070A8A8B88888702005066D
:1019200006060001E08CEA8C8A0A0509090600FF18
:10193000F8A88888888888A8F8050A0A0600FE2082
:101940005050505088A8A888700303030600034035
:10195000A040FFFFFFFFFFFFFFFFFFFFFFFFFFFFB5
:10196000FFFFFFFFFFFFFFFF0000000605FF01076D
:101970000706020080808080800080030303060148
:1019800005A0A0A005060606000050F85050F8502B
:101990000509090600FF2070A8A07028A87020057E
:1019A0000707060000C8C8102040989805070706DA
:1019B000000040A0A040A890680103030602058033
:1019C00080800309090601FF20404080808040405C
:1019D000200309090601FF8040402020204040806C
:1019E00005070706000020A8702070A8200505053F
:1019F0000600012020F820200203030601FFC0405A
:101A000080050101060003F8020202060100C0C0C1
:101A10000507070600000810102040408005070752
:101A2000060000708898A8C88870030707060100A0
:101A300040C040404040E0050707060000708808AD
:101A4000102040F8050707060000F8081030088845
:101A50007005070706000010305090F810100507B9
:101A600007060000F880F0080888700507070600E0
:101A700000304080F0888870050707060000F808ED
:101A80001010202020050707060000708888708845
:101A900088700507070600007088887808106002C3
:101AA0000505060100C0C000C0C00206060601FF11
:101AB000C0C000C0408003050506010120408040F1
:101AC00020050303060002F800F8030505060101DE
:101AD0008040204080050707060000708810202005
:101AE00000200507070600007088B8A8B8807005B8
:101AF0000707060000708888F888888805070706A9
:101B00000000F04848704848F005070706000070DC
:101B1000888080808870050707060000F0484848E4
:101B20004848F0050707060000F88080F08080F83C
:101B3000050707060000F88080F080808005070711
:101B400006000070888080988870050707060000EE
:101B5000888888F8888888030707060100E04040E5
:101B6000404040E0050707060000381010101090B4
:101B7000600507070600008890A0C0A090880507B0
:101B800007060000808080808080F8050707060037
:101B90000088D8A8888888880507070600008888F4
:101BA000C8A8988888050707060000708888888874
:101BB0008870050707060000F08888F0808080059F
:101BC000070706000070888888A890680507070640
:101BD0000000F08888F0A0908805070706000070D4
:101BE000888070088870050707060000F82020200C
:101BF00020202005070706000088888888888870CC
:101C000005070706000088888888505020050707C8
:101C100006000088888888A8A850050707060000E5
:101C2000888850205088880507070600008888505B
:101C300020202020050707060000F808102040801B
:101C4000F80309090601FFE080808080808080E041
:101C5000050707060000804040201010080309090E
:101C60000601FFE020202020202020E005030306BD
:101C700000052050880501010600FEF80303030655
:101C80000105804020050505060000700878887869
:101C90000507070600008080F0888888F0050505A4
:101CA000060000708080887005070706000008089D
:101CB00078888888780505050600007088F08070AF
:101CC000050707060000304840E040404005070790
:101CD0000600FE70888888780870050707060000EF
:101CE0008080F0888888880307070601004000C0CC
:101CF000404040E00409090601FE100030101010B9
:101D000010906005070706000080808890E09088AA
:101D1000030707060100C04040404040E0050505BC
:101D2000060000D0A8A8A8A8050505060000B0C8B0
:101D30008888880505050600007088888870050772
:101D4000070600FEF0888888F080800507070600F7
:101D5000FE78888888780808050505060000B0C860
:101D600080808005050506000078807008F0050772
:101D7000070600002020F820202018050505060091
:101D800000888888986805050506000088888850BE
:101D9000200505050600008888A8A8500505050649
:101DA000000088502050880507070600FE888888B4
:101DB00050204080050505060000F8102040F8037B
:101DC00009090601FF2040404080404040200109B1
:101DD000090602FF8080808080808080800309095E
:101DE0000601FF804040402040404080050303063C
:101DF000000248A890FF1FFFFFFFFFFFFF600000E9
:101E0000000001FF400000000000FF800000000013
:101E1000007F83CF00000C303F87FF80000C301F15
:101E2000867980000C000F8C30C7838C30E78C30B3
:101E3000CFC7CC31F38C30DCECEC33B98C30D86CC0
:101E40006C33198C30D06C0C33198C30D86C0C334B
:101E5000198C30DC6C0E3B198C30CF7C079F198CB1
:101E600030C77C038F1940000000000002600000B2
:101E7000000000061FFFFFFFFFFFF800060900FE3D
:101E800006018902FE20FFFE07FE06FE0000000696
:101E900000070106060602008080808000800303A0
:101EA00003060103A0A0A00507070600FF5050F895
:101EB00050F850500509090600FE2070A8A07028AF
:101EC000A870200608080600FF40A84810204854C3
:101ED000080507070600FF6090906098906801036E
:101EE000030602038080800207070602FF4080800D
:101EF000808080400207070602FF8040404040404B
:101F0000800505050600008850F85088050505067F
:101F100000002020F820200204040602FEC04040F9
:101F200080050101060002F8020202060200C0C09C
:101F300004060606010010102040808004060606F4
:101F4000010060909090906003060606010040C07A
:101F5000404040E00406060601006090102040F07A
:101F6000040606060100F020601010E005060606D3
:101F7000000010305090F810040606060100F080B2
:101F8000E01010E00406060601006080E09090601A
:101F9000040606060100F010102040400406060664
:101FA0000100609060909060040606060100609059
:101FB00090701060020505060200C0C000C0C0029B
:101FC00007070602FEC0C000C040408005050506A8
:101FD00000001860806018050303060001F800F88F
:101FE000050505060000C0300830C00407070601DB
:101FF00000609010604000400506060600007090EA
:10200000A8B08070050606060000205088F8888871
:10201000050606060000F088F08888F0040606062B
:102020000100609080809060040606060100E09048
:10203000909090E0040606060100F080E08080F0B9
:10204000040606060100F080E08080800406060693
:102050000100609080B09060040606060100909038
:10206000F0909090030606060100E040404040E0FA
:1020700005060606000038101010906004060606DB
:10208000010090A0C0A09090040606060100808088
:10209000808080F005060606000088D8A8A88888F9
:1020A00004060606010090D0B09090900506060642
:1020B0000000708888888870040606060100E09099
:1020C00090E080800407070601FF609090D0B06028
:1020D00010040606060100E09090E09090040606C9
:1020E000060100609040209060050606060000F89A
:1020F0002020202020040606060100909090909059
:1021000060040606060100909090F06060050606E7
:102110000600008888A8A8D888050606060000885A
:102120005020205088050606060000888850202090
:1021300020040606060100F010204080F003060689
:10214000060100E080808080E00406060601008031
:102150008040201010030606060100E02020202009
:10216000E00503030600032050880501010600FE78
:10217000F802020206020480400404040601007012
:102180009090700406060601008080E09090E004C4
:102190000404060100708080700406060601001029
:1021A000107090907004040406010060B0C07004C8
:1021B0000606060100205040E040400406060601E5
:1021C000FE6090907010600406060601008080E0BA
:1021D0009090900306060601004000C04040E003D6
:1021E00008080601FE200060202020A0400406060A
:1021F0000601008080A0C0A090030606060100C072
:1022000040404040E0050404060000D0A8A888042F
:102210000404060100E090909004040406010060AC
:102220009090600406060601FEE09090E080800435
:1022300006060601FE70909070101004040406015A
:1022400000A0D0808004040406010070C030E004C7
:1022500006060601004040E0405020040404060148
:102260000090909070040404060100909060600556
:10227000040406000088A8A8500404040601009085
:102280006060900406060601FE90909070906004D5
:102290000404060100F02040F003070706010020B7
:1022A0004040804040200107070602FF8080808078
:1022B0008080800307070601008040402040408066
:1022C00004020206010350A0FFFFFFFFFFFFFFFF14
:1022D000FFFFFFFFFFFFFFFFFFFFFFFFFFFFFFFF0E
:1022E000FFFFFFFFFFFFFFFFFF00000006000701E9
:1022F0000606060200800080808080040606060133
:10230000FF2070A0A070200507070600FF3048409E
:10231000F04040F8050505060000A8508850A805C3
:1023200006060600008850F820F82001070706027C
:10233000FF808080008080800407070601FF708096
:1023400060906010E0030101060105A00607070682
:102350000000788494A49484780305050601016044
:10236000A06000E00505050600002850A0502804E4
:102370000303060100F01010040101060102F0063B
:1023800007070600007884B4A4A484780401010639
:102390000105F004030306010260906005070706CB
:1023A00000FF2020F8202000F80305050601014069
:1023B000A02040E0030505060101C0204020C00226
:1023C000020206020440800405050601FF9090B059
:1023D000D08005060606000078E8E8682828010194
:1023E00001060202800202020602FE408003050589
:1023F00006010140C04040E003050506010140A080
:102400004000E0050505060000A0502850A0050882
:10241000080600FF40C040507030781005080806DC
:1024200000FF40C04050680810380508080600FF4B
:10243000C0204030F030781004070706010020006B
:102440002060809060050707060000402020507043
:10245000888805070706000010202050708888052E
:1024600007070600002050205070888805070706DF
:10247000000028502050708888050707060000508B
:102480000020507088880507070600002050205063
:1024900070888805060606000078A0F0A0A0B804A1
:1024A00008080601FE6090808090602040040707C5
:1024B0000601004020F080E080F0040707060100DC
:1024C0002040F080E080F00407070601002050F073
:1024D00080E080F00407070601005000F080E080F3
:1024E000F00307070601008040E0404040E003079A
:1024F000070601002040E0404040E00307070601D6
:102500000040A0E0404040E0030707060100A000B3
:10251000E0404040E00506060600007048E84848F4
:102520007004070706010050A090D0B090900407F7
:1025300007060100402060909090600407070601A4
:102540000020406090909060040707060100205032
:10255000609090906004070706010050A060909082
:10256000906004070706010050006090909060059D
:10257000050506000088502050880408080601FF61
:102580001070B0B0D0D0E0800407070601004020F2
:102590009090909060040707060100204090909072
:1025A000906004070706010020509090909060040E
:1025B00007070601005000909090906005070706FD
:1025C000000010208850202020040606060100800C
:1025D000E09090E0800406060601006090A0A090C4
:1025E000A0040707060100402000709090700407C7
:1025F0000706010020400070909070040707060154
:10260000002050007090907004070706010050A051
:1026100000709090700406060601005000709090C3
:102620007004070706010020502070909070050488
:102630000406000070A8B0780406060601FE70804B
:102640008070204004070706010040200060B0C0F1
:102650007004070706010020400060B0C070040746
:102660000706010020500060B0C070040606060195
:1026700000500060B0C070030707060100804000F2
:10268000C04040E0030707060100204000C0404072
:10269000E003070706010040A000C04040E0030639
:1026A00006060100A000C04040E004070706010044
:1026B0003060107090906004070706010050A00081
:1026C000E090909004070706010040200060909081
:1026D0006004070706010020400060909060040736
:1026E0000706010020500060909060040707060173
:1026F0000050A000609090600406060601005000A3
:10270000609090600505050600002000F800200498
:10271000040406010070B0D0E00407070601004081
:102720002000909090700407070601002040009060
:102730009090700407070601002050009090907060
:1027400004060606010050009090907004090906E6
:1027500001FE2040009090907090600408080601EF
:10276000FE8080E09090E080800408080601FE5022
:1027700000909090709060536E346B3300496E7689
:10278000616465727300427269636B6F7574004DAA
:1027900061696E00536D6F6F7468696E6700536D89
:1027A0006F6F7468696E67005A005A0059005900CB
:1027B00058005800436F7272656374696F6E00430E
:1027C0006F7272656374696F6E004D61696E004669
:1027D000696C616D656E740054656D7065726174CD
:1027E00075726500447269766520537472656E6710
:1027F0007468004261636B6C617368005374657048
:10280000732F6D6D004A65726B00416363656C6583
:10281000726174696F6E0056656C6F6369747900DC
:10282000436F6E66696775726174696F6E00457398
:10283000746570732F6D6D004573746570732F6DC3
:102840006D005A73746570732F6D6D005A737465E3
:1028500070732F6D6D005973746570732F6D6D00FB
:102860005973746570732F6D6D0058737465707350
:102870002F6D6D005873746570732F6D6D0041641A
:1028800076616E6365642053657474696E67730066
:1028900056652D4A65726B0056652D4A65726B0050
:1028A000567A2D4A65726B00567A2D4A65726B0016
:1028B00056792D4A65726B0056792D4A65726B0008
:1028C00056782D4A65726B0056782D4A65726B00FA
:1028D000416476616E6365642053657474696E67E4
:1028E0007300416D6178204500416D61782045009D
:1028F000416D6178205A00416D6178205A00416D28
:102900006178205900416D6178205900416D6178EE
:10291000205800416D6178205800412D5472617635
:10292000656C00412D54726176656C00412D5265D5
:10293000747261637400412D526574726163740036
:10294000416363656C00416363656C00416476615B
:102950006E6365642053657474696E6773005654C2
:10296000726176204D696E005654726176204D6911
:102970006E00566D696E00566D696E00566D617819
:10298000204500566D6178204500566D6178205ACB
:1029900000566D6178205A00566D617820590056B6
:1029A0006D6178205900566D6178205800566D6130
:1029B00078205800416476616E63656420536574C5
:1029C00074696E67730020082046616374002008F4
:1029D0002046616374002008204D617800200820A3
:1029E0004D6178002008204D696E002008204D6957
:1029F0006E004175746F74656D70004F6666004FB0
:102A00006E004175746F74656D7000416476616E1F
:102A10006365642053657474696E6773004C6F61FD
:102A200064206D6D004C6F6164206D6D00556E6C9F
:102A30006F6164206D6D00556E6C6F6164206D6D0B
:102A400000416476616E6365204B00416476616E7F
:102A50006365204B00416476616E63656420536555
:102A60007474696E677300450045005A005A005837
:102A70005900585900416476616E6365642053655E
:102A80007474696E67730044697361626C65205386
:102A900074657070657273004D3834004175746FE1
:102AA0002043616C696272617465004D3131372079
:102AB0005374617274696E67204175746F2D436140
:102AC0006C6962726174696F6E0A54300A473238F9
:102AD0000A4731320A4D3131372043616C696272E5
:102AE0006174696E672E2E2E0A473432350A4D35D1
:102AF00030300A4D3131372043616C696272617444
:102B0000696F6E2064617461207361766564004151
:102B100075746F20486F6D6500473238004D6F76D1
:102B2000652041786973004D61696E004578747263
:102B30007564657220004175746F20486F6D650083
:102B4000473238004D6F7665205A004D6F7665200C
:102B500059004D6F76652058004D6F74696F6E0097
:102B6000457874727564657220004D6F7665202516
:102B7000736D6D00004D6F766520302E316D6D00E8
:102B80004D6F766520316D6D004D6F76652031306B
:102B90006D6D004D6F7665204178697300486F74E4
:102BA000656E6420746F6F20636F6C640045787489
:102BB000727564657220004D6F7665205A004D6F06
:102BC00076652059004D6F76652058004D6F76650B
:102BD000205A004D6F76652059004D6F766520585C
:102BE000005072696E742066726F6D204D65646965
:102BF00061005072696E742066726F6D204D65645D
:102C0000696100022E2E004D61696E005072696E7E
:102C1000740043616E63656C00537461727420507C
:102C200072696E7420003F005761697420666F728C
:102C30000066696C616D656E742070757267650001
:102C400000506C6561736520776169742E00507265
:102C500065737320427574746F6E00746F207265B3
:102C600073756D65207072696E74005761697420A8
:102C7000666F720066696C616D656E74206C6F6161
:102C80006400496E736572742066696C616D656E6F
:102C90007400616E64207072657373206275747461
:102CA0006F6E00746F20636F6E74696E756500508F
:102CB0007265737320627574746F6E00746F206830
:102CC000656174206E6F7A7A6C65004E6F7A7A6CEB
:102CD000652068656174696E6700506C6561736535
:102CE00020776169742E2E2E005761697420666FFB
:102CF000720066696C616D656E7420756E6C6F61D3
:102D000064005761697420666F720066696C616D5A
:102D1000656E74206368616E676500746F207374FC
:102D2000617274005061726B696E672E2E2E0043C3
:102D300068616E67696E672046696C616D656E7467
:102D400000554E4C4F41442046494C414D454E5450
:102D5000004C4F41442046494C414D454E540020C3
:102D6000204E6F7A7A6C653A20002000456E642010
:102D700066696C616D656E74206368616E6765007D
:102D80005075726765206D6F726500004368616EF3
:102D900067652046696C616D656E7400556E6C6F79
:102DA00061642046696C616D656E74004C6F61648E
:102DB0002046696C616D656E74004D36303020427E
:102DC0003020542564004D373032203B2564004DBF
:102DD00037303220542564004D373031205425647B
:102DE000005072656865617420437573746F6D007F
:102DF0005072656865617420437573746F6D00501F
:102E0000726568656174204142530050726568655F
:102E1000617420504C41004261636B004E6F204D45
:102E200065646961005072696E742066726F6D200E
:102E30004D65646961004368616E6765204D656436
:102E40006961004D32310041626F757420507269C2
:102E50006E746572004368616E67652046696C61D7
:102E60006D656E74004368616E67652046696C61CC
:102E70006D656E74004D36303020423000436F6E09
:102E800066696775726174696F6E0054656D70650F
:102E9000726174757265004D6F74696F6E00526572
:102EA00073756D65205072696E740054756E65009F
:102EB00053746F70205072696E7400506175736541
:102EC000205072696E7400496E666F20536372659C
:102ED000656E0053746F70004261636B0053746FD2
:102EE00070205072696E74003F0050726F626520EE
:102EF0005A204F6666736574004261627973746527
:102F000070205900426162797374657020580046E0
:102F10006C6F7700466C6F770046616E205370656A
:102F200065640046616E20537065656400426564A7
:102F300000426564004E6F7A7A6C65004E6F7A7A53
:102F40006C65005370656564005370656564004D81
:102F500061696E0042616279737465702059004244
:102F60006162797374657020580047616D65730004
:102F70004669726D776172652056657273696F6E0E
:102F8000004D61696E00436F6F6C646F776E004631
:102F9000616E2053706565640046616E20537065F4
:102FA00065640042656400426564004E6F7A7A6C25
:102FB00065004E6F7A7A6C65004D61696E006F6FC7
:102FC0006F0000001FC07FF0DDD8FFF87FF04440A5
:102FD000248000003180000024804440107CFEFEEC
:102FE000FE04000E000E007FC0FFE0FFE0FFE0FFE8
:102FF000E006000F001F8036C03FC0090016802980
:103000004006000F001F8036C03FC01680204010D1
:1030100080104008801FC037607FF05FD050500D97
:1030200080104048905FD077707FF01FC010402024
:10303000200F007FE0FFF0E670FFF0198036C0C07F
:10304000300F007FE0FFF0E670FFF0198036C01906
:103050008047414D45204F56455200526573746F6D
:103060007265206661696C73616665004C6F6164AE
:103070002053657474696E67730053746F726520B2
:1030800053657474696E67730050726F6265205A7D
:10309000204F666673657400416476616E63656493
:1030A0002053657474696E6773004D61696E0050DA
:1030B000726F6265205A204F6666736574004D6FAB
:1030C00076696E672E2E2E004D3234004D3235203B
:1030D000500A4D3234005072696E7420506175731D
:1030E0006564005061757365205072696E7400509C
:1030F00072696E742041626F72746564004C756C05
:103100007A426F74204D696E692072656164792E10
:10311000005072696E74696E672E2E2E00507269AF
:103120006E7420506175736564004D65646961203B
:1031300052656D6F766564004D6564696120496E06
:10314000736572746564004D313137004D33310061
:1031500043616E6E6F7420656E7465722073756264
:103160006469723A20002E0A006F70656E206661F5
:10317000696C65642C2046696C653A200061757441
:103180006F25632E67006572726F722077726974A3
:10319000696E6720746F2066696C650A004E6F74F3
:1031A000205344207072696E74696E670A0053443C
:1031B000207072696E74696E672062797465200090
:1031C0002E0A0044656C6574696F6E206661696CD7
:1031D00065642C2046696C653A200046696C652060
:1031E00064656C657465643A0057726974696E67EA
:1031F00020746F2066696C653A20002E0A006F709B
:10320000656E206661696C65642C2046696C653A60
:1032100020002E0A006F70656E206661696C65641F
:103220002C2046696C653A200046696C6520736500
:103230006C65637465640A002053697A653A2000FE
:1032400046696C65206F70656E65643A2000206683
:10325000696C653A2000667265736800646F696E18
:1032600067004E6F772000454E4420535542524F21
:103270005554494E450A002220706F730022207079
:103280006172656E743A2200535542524F5554494B
:103290004E452043414C4C207461726765743A225C
:1032A00000747279696E6720746F2063616C6C20A2
:1032B0007375622D67636F64652066696C65732042
:1032C0007769746820746F6F206D616E79206C650A
:1032D00076656C732E204D4158206C6576656C20A8
:1032E00069733A310A004D3234004D323320257370
:1032F0000053442063617264206F6B0A006F706535
:103300006E526F6F74206661696C65640A00766F37
:103310006C756D652E696E6974206661696C656493
:103320000A00534420696E6974206661696C0A0062
:10333000286E6F2066696C65290043616E6E6F743C
:10334000206F70656E2073756264697220007C3C2A
:103350003E5E2B3D3F2F5B5D3B2C2A225C000A002A
:103360003B20454550524F4D20496E6465783A20C8
:10337000005570646174696E67207A6F6666736564
:103380007420696E20454550524F4D3A20003474E8
:10339000682070726F626520706F696E742C206493
:1033A000697374616E63652066726F6D20706C6105
:1033B0006E653A20000000000000000000000000E0
:1033C00000000000000000000000000000000000FD
:1033D00000000000000000000C00000000000000E1
:1033E0000C000000000000001200000000000000BF
:1033F0002300000000000000210000000000000089
:103400004C800000000000005E8000000000000012
:103410009240000000000000A140000000000001F8
:1034200021200000000000027F9000000000000248
:103430000010000000000007FFF80000000000047A
:103440000008000000000008000400000000000860
:103450000006000000000010000200000000003024
:103460001E010000000000207F81000000000041DC
:10347000FFE0800000000043FCF0800000000087B7
:103480003B7840000000018EDBFC60000000010F73
:10349000EBCC20000000021FEDB610000000021F60
:1034A000DEB6100000000439CD7F080000000436AD
:1034B000E0FF08000000087EC0BB84000000187F09
:1034C000005D86000000107FC0ED82000000203CFF
:1034D000C07301000000203B337F01000000701B1F
:1034E000E77E03800000C81DEEDE04C00000880FE8
:1034F000DEDC04400001240FDF3C09200001260728
:10350000DBF8192000027203E7F01390000251016A
:10351000FFE02290000489007F8024480009048095
:103520001E004824000BFE400000DFF400100040A5
:1035300000008002001FFFFFFFFFFFFE00000000F1
:10354000000000000000000000000000000000007B
:1035500000000000001022103C3C0E1F0010221042
:10356000042211040010221008221104001022105D
:10357000083C110400102210102211040010221027
:1035800020221104001E1C1E3C3C0E040000000002
:10359000000000000000000000000000000000002B
:1035A000000000000000000000000000000000001B
:1035B000000000000000000000000000000000000B
:1035C00000000000000000000000000000000000FB
:1035D00000000000000000000000000000000000EB
:1035E00000000000000000000000000000000000DB
:1035F000000000000C0D00FE07022603BC017FFE48
:1036000008FE08FE05080806000040F0C8888898F3
:103610007810050808060000C0F88888888888F8AF
:103620000505050600012030F830200508080600D1
:10363000002070F820202020E00509090600FF2066
:1036400070A8A8B888887020050606060001E08CDE
:10365000EA8C8A0A0509090600FFF8A88888888884
:1036600088A8F8050A0A0600FE205050505088A885
:10367000A8887003030306000340A040FFFFFFFF7C
:10368000FFFFFFFFFFFFFFFFFFFFFFFFFFFFFFFF4A
:10369000FFFF0000000605FF01070706020080800B
:1036A0008080800080030303060105A0A0A005061A
:1036B0000606000050F85050F8500509090600FFB2
:1036C0002070A8A07028A87020050707060000C871
:1036D000C8102040989805070706000040A0A040A9
:1036E000A89068010303060205808080030909068B
:1036F00001FF2040408080804040200309090601EE
:10370000FF80404020202040408005070706000041
:1037100020A8702070A8200505050600012020F8CB
:1037200020200203030601FFC040800501010600BE
:1037300003F8020202060100C0C0050707060000E8
:103740000810102040408005070706000070889888
:10375000A8C8887003070706010040C040404040E9
:10376000E0050707060000708808102040F80507EC
:1037700007060000F80810300888700507070600E3
:103780000010305090F81010050707060000F88070
:10379000F008088870050707060000304080F088B0
:1037A0008870050707060000F80810102020200583
:1037B000070706000070888870888870050707066C
:1037C000000070888878081060020505060100C0B6
:1037D000C000C0C00206060601FFC0C000C0408095
:1037E0000305050601012040804020050303060073
:1037F00002F800F80305050601018040204080051D
:103800000707060000708810202000200507070623
:1038100000007088B8A8B88070050707060000701F
:103820008888F8888888050707060000F0484870EF
:103830004848F0050707060000708880808088707F
:10384000050707060000F04848484848F005070704
:10385000060000F88080F08080F805070706000069
:10386000F88080F08080800507070600007088805F
:1038700080988870050707060000888888F888887F
:1038800088030707060100E04040404040E005078C
:10389000070600003810101010906005070706009A
:1038A000008890A0C0A090880507070600008080CF
:1038B00080808080F805070706000088D8A88888DF
:1038C00088880507070600008888C8A898888805A2
:1038D0000707060000708888888888700507070633
:1038E0000000F08888F080808005070706000070DF
:1038F000888888A89068050707060000F08888F087
:10390000A0908805070706000070888070088870FE
:10391000050707060000F8202020202020050707C3
:1039200006000088888888888870050707060000D8
:1039300088888888505020050707060000888888F6
:1039400088A8A850050707060000888850205088DE
:1039500088050707060000888850202020200507DA
:1039600007060000F80810204080F8030909060146
:10397000FFE080808080808080E0050707060000EF
:10398000804040201010080309090601FFE02020B4
:103990002020202020E00503030600052050880594
:1039A00001010600FEF8030303060105804020051F
:1039B00005050600007008788878050707060000EE
:1039C0008080F0888888F0050505060000708080FA
:1039D0008870050707060000080878888888780539
:1039E00005050600007088F08070050707060000D6
:1039F000304840E04040400507070600FE708888D8
:103A0000887808700507070600008080F08888889D
:103A1000880307070601004000C0404040E0040959
:103A2000090601FE10003010101010906005070705
:103A300006000080808890E0908803070706010058
:103A4000C04040404040E0050505060000D0A8A861
:103A5000A8A8050505060000B0C8888888050505E2
:103A600006000070888888700507070600FEF08849
:103A70008888F080800507070600FE7888888878A7
:103A80000808050505060000B0C88080800505050A
:103A900006000078807008F0050707060000202067
:103AA000F8202020180505050600008888889868F9
:103AB00005050506000088888850200505050600D4
:103AC000008888A8A85005050506000088502050E9
:103AD000880507070600FE88888850204080050575
:103AE00005060000F8102040F80309090601FF2030
:103AF00040404080404040200109090602FF80808C
:103B0000808080808080800309090601FF8040401A
:103B100040204040408005030306000248A890FF73
:103B20004F4646004F4E006563686F3A004572721B
:103B30006F723A004572726F722077726974696EA3
:103B40006720746F20454550524F4D210A00507236
:103B500065737320627574746F6E20286F72204DC8
:103B60003130382920746F2068656174206E6F7A57
:103B70007A6C650A00507265737320627574746F95
:103B80006E20286F72204D3130382920746F2072DA
:103B90006573756D650A00496E7365727420666998
:103BA0006C616D656E7420616E64207072657373F4
:103BB00020627574746F6E20286F72204D3130381A
:103BC000290A004D3630303A20546F6F20436F6C15
:103BD0006400486F74656E6420746F6F20636F6C4F
:103BE000640A00486F74656E6420746F6F20636FA1
:103BF0006C640A00496E736572742066696C616D4D
:103C0000656E7420616E64207072657373206275D6
:103C100074746F6E20286F72204D313038290A007D
:103C200063616E63656C00726573756D65640072C7
:103C30006573756D650070617573656400706F778D
:103C400065726F6666002F2F616374696F6E3A004C
:103C500020573A0020573A00486F74656E6420433D
:103C60006F6F6C696E672E2E2E00486F74656E64E0
:103C70002048656174696E672E2E2E00202F00206B
:103C800042403A0020403A004D3834205820592014
:103C90005A204500546865726D616C2052756E61E2
:103CA00077617900486F74656E6420544845524DC1
:103CB000414C2052554E41574159004245442054F1
:103CC0004845524D414C2052554E415741590020D4
:103CD0002D20496E76616C69642065787472756414
:103CE0006572206E756D62657220210A00486561FB
:103CF00074696E67206661696C6564004265642062
:103D000048656174696E67204661696C656400543A
:103D10006865726D616C2052756E617761790042E1
:103D2000454420544845524D414C2052554E415730
:103D300041590048656174696E67206661696C6508
:103D40006400486F74656E642048656174696E67CD
:103D5000204661696C656400546865726D616C2011
:103D600052756E6177617900486F74656E64205496
:103D70004845524D414C2052554E41574159004DF6
:103D8000494E54454D502074726967676572656489
:103D900000486F74656E64204572723A204D494E3A
:103DA00054454D50004572723A204D494E54454D90
:103DB0005020424544004D415854454D50207472A6
:103DC0006967676572656400486F74656E64204555
:103DD00072723A204D415854454D50004572723A26
:103DE000204D415854454D50204245440062656481
:103DF000002C2073797374656D2073746F70706517
:103E00006421204865617465725F49443A2000234B
:103E1000646566696E652044454641554C545F00B3
:103E20004B6420004B6920004B70200000626564E9
:103E300000504944204175746F74756E6520666941
:103E40006E697368656421205075742074686520FC
:103E50006C617374204B702C204B6920616E642060
:103E60004B6420636F6E7374616E74732066726F3F
:103E70006D2062656C6F7720696E746F20436F6E82
:103E800066696775726174696F6E2E680A005049C1
:103E900044204175746F74756E65206661696C6548
:103EA00064212074696D656F75740A0054686572C9
:103EB0006D616C2052756E6177617900486F746531
:103EC0006E6420544845524D414C2052554E415746
:103ED00041590042454420544845524D414C2052DE
:103EE000554E415741590048656174696E672066B7
:103EF00061696C656400486F74656E642048656133
:103F000074696E67204661696C656400426564206F
:103F100048656174696E67204661696C656400502C
:103F20004944204175746F74756E65206661696CD3
:103F30006564212054656D706572617475726520C9
:103F4000746F6F20686967680A00204B643A20002C
:103F5000204B693A2000204B703A20000A20436C25
:103F6000617373696320504944200A00204B643A0E
:103F70002000204B693A2000204B703A20000A2094
:103F80004E6F206F76657273686F6F740A002054ED
:103F9000753A2000204B753A2000206D61783A2058
:103FA00000206D696E3A200020643A20002062698A
:103FB00061733A2000504944204175746F74756EE6
:103FC000652073746172740A00504944204175740D
:103FD0006F74756E65206661696C65642120546537
:103FE0006D706572617475726520746F6F20686999
:103FF00067680A001000AD0330016A0150022B010E
:1040000070030A019004F500B005E500D006D80061
:10401000F007CE001009C500300ABE00500BB700F3
:10402000700CB100900DAB00B00EA600D00FA20036
:10403000F0109D001012990030139500501492005A
:1040400070158E0090168B00B0178700D018840072
:10405000F0198100101B7E00301C7B00501D790080
:10406000701E7600901F7300B0207000D0216E008B
:10407000F0226B0010246900302566005026630092
:104080007027610090285E00B0295C00D02A59009A
:10409000F02B5600102D5400302E5100502F4E00A2
:1040A00070304B0090314800B0324500D0334200B0
:1040B000F0343E0010363B003037370050383300C4
:1040C00070392E00903A2900B03B2300D03C1B00F1
:1040D000F03D1100103F0100F03F00001000C90248
:1040E00010012C014001220170011801B0010E01E4
:1040F000F00104015002FA00B002F0003003E600C3
:10410000D003DC009004D2007005C800A006BE00F9
:104110000008B400B009AA00D00BA000600E960001
:1041200060118C000015820020197800C01D6E00FF
:10413000A0226400B0275A00902C500000314600A5
:10414000E0343C0010383200903A2800603C1E00F9
:10415000A03D1400803E0A00203F00006F70656E95
:1041600000545249474745524544003A20007A5F7F
:104170006D6178007A5F6D696E00795F6D617800BE
:10418000795F6D696E00785F6D617800785F6D6949
:104190006E005265706F7274696E6720656E64732D
:1041A000746F70207374617475730A00456E647364
:1041B000746F707320256320256320256320256399
:1041C00000205A3A0020593A0020583A00656E649F
:1041D00073746F7073206869743A2000486F6D695A
:1041E0006E67204661696C656400496E76616C6932
:1041F000642065787472756465720A0045303A20EF
:10420000005A3A2000593A20004D53312C4D533278
:104210002C4D53332050696E730A583A20004D6973
:1042200063726F737465707320756E617661696C0B
:1042300061626C650A00205A3A0020593A00204316
:104240006F756E7420583A00C23100001C260000C1
:10425000F4190000D80F0000EB080000C0040000B3
:10426000750200004001000024F4D43050C38E20B9
:10427000C2A24017828B7011127A910D816CD90AFB
:10428000A861E108C7586607615143061E4B5D05EA
:10429000C145A7041A411104093D9803713931033E
:1042A0004036DB0265339102D4305402802E1D0269
:1042B000632CEE01752AC501B028A00110278101E9
:1042C0008F2564012B244B01E0223401AC211F0116
:1042D0008D200D01801FFC00841EED00971DDF0066
:1042E000B81CD200E61BC600201BBC00641AB2003A
:1042F000B219A8000A19A0006A189900D1179100F4
:1043000040178B00B516840031167E00B315790076
:104310003A157300C7146F0058146A00EE13660054
:104320008813630025135E00C7125B006C125700F0
:1043300015125400C111510070114F0021114B0092
:10434000D61049008D10470046104400021042006C
:10435000C00F4000800F3E00420F3C00060F3B00A4
:10436000CB0E3800930E37005C0E3500270E34005C
:10437000F30D3200C10D3100900D3000600D2E00A4
:10438000320D2D00050D2C00D90C2B00AE0C290090
:10439000850C29005C0C2700350C27000E0C26002C
:1043A000E80B2400C40B2400A00B23007D0B23008A
:1043B0005A0B2100390B2100180B2000F80A1F00AE
:1043C000D90A1E00BB0A1E009D0A1D00800A1D009E
:1043D000630A1C00470A1B002C0A1B00110A1A0062
:1043E000F7091A00DD091900C4091900AB09190001
:1043F000920917007B091800630917004C09160081
:1044000036091600200916000A091500F5081500DE
:10441000E0081400CC081400B8081400A408140024
:10442000900813007D0812006B0813005808120052
:104430004608120034081100230811001208110068
:1044400001081100F0071000E0071000D00710006D
:10445000C0071000B0070F00A107100091070E0061
:1044600083070F0074070F0065070E0057070E0043
:1044700049070E003B070D002E070E0020070D0018
:1044800013070D0006070D00F9060C00ED060D00E0
:10449000E0060C00D4060C00C8060C00BC060C009C
:1044A000B0060C00A4060B0099060C008D060B004C
:1044B00082060B0077060B006C060B0061060A00F3
:1044C00057060B004C060A0042060A0038060A008E
:1044D0002E060A0024060A001A060A001006090021
:1044E00007060A00FD050900F4050900EB050900AF
:1044F000E2050900D9050900D0050900C705090032
:10450000BE050900B5050800AD050800A5050900B0
:104510009C050800940508008C0508008405080027
:104520007C050800740508006C0507006505080097
:104530005D050700560508004E0507004705070002
:104540004005080038050700310507002A05070067
:10455000230507001C050600160507000F050700C8
:104560000805060002050700FB040600F504070025
:10457000EE040600E8040600E2040700DB0406007F
:10458000D5040600CF040600C9040600C3040600D3
:10459000BD040600B7040600B1040500AC04060023
:1045A000A6040600A00405009B040600950405006F
:1045B000900406008A0405008504050080040600B6
:1045C0007A04050075040500700405006B040500FD
:1045D00066040500610405005C040500570405003D
:1045E000520405004D04050048040500430405007D
:1045F0003E0404003A0405003504050030040400BC
:104600002C04050027040400230405001E040400F4
:104610001A04040016040500110404000D0404002B
:10462000090405000404040000040400FC03040061
:10463000F8030400F4030400F0030400EC03040096
:10464000E8030400E4030400E0030400DC030400C6
:10465000D8030400D4030400D0030400CC030400F6
:10466000C8030300C503030024F404D9201BC40CB1
:104670005C0E9804C4095F0265077101F405F90036
:10468000FB04B30048048700C103690058035500C8
:1046900003034500BE023A008402310053022A009F
:1046A0002902250004022000E4011C00C8011900B1
:1046B000AF0117009801140084011300710110006C
:1046C0006101100051010E0043010D0036010B0085
:1046D0002B010B0020010B00150109000C01090042
:1046E00003010800FB000800F3000800EB000700CE
:1046F000E4000600DE000600D8000600D200060036
:10470000CC000500C7000500C2000500BD00040084
:10471000B9000400B5000400B1000400AD000400BD
:10472000A9000400A5000300A20003009F000400EC
:104730009B00030098000300950002009300030013
:10474000900003008D0002008B000300880002002F
:104750008600020084000300810002007F00020046
:104760007D0002007B00020079000200770001005A
:104770007600020074000200720001007100020065
:104780006F0002006D0001006C0002006A00010071
:104790006900020067000100660001006500010079
:1047A000640002006200010061000100600001007D
:1047B0005F0002005D0001005C0001005B00010081
:1047C0005A00010059000100580001005700010083
:1047D0005600010055000100540001005300000084
:1047E000530001005200010051000100500001007F
:1047F0004F0001004E0000004E0001004D0001007E
:104800004C0001004B0000004B0001004A00010079
:104810004900010048000000480001004700010075
:104820004600000046000100450000004500010070
:10483000440001004300000043000100420000006A
:104840004200010041000000410001004000010061
:104850003F0000003F0001003E0000003E0001005C
:104860003D0000003D0001003C0000003C00000055
:104870003C0001003B0000003B0001003A0000004A
:104880003A00010039000000390001003800000042
:104890003800000038000100370000003700010038
:1048A0003600000036000000360001003500000030
:1048B0003500000035000100340000003400000025
:1048C0003400010033000000330000003300010019
:1048D0003200000032000000320001003100000010
:1048E0003100000031000100300000003000000005
:1048F000300001002F0000002F0000002F000000FA
:104900002F0001002E0000002E0000002E000100EC
:104910002D0000002D0000002D0000002D000100E2
:104920002C0000002C0000002C0000002C000100D6
:104930002B0000002B0000002B0000002B000100CA
:104940002A0000002A0000002A0000002A000100BE
:1049500029000000290000002900000029000000B3
:1049600029000100280000002800000028000000A5
:104970002800000028000100270000002700000098
:10498000270000002700000027000100260000008B
:10499000260000002600000026000000260001007E
:1049A0002500000025000000250000002500000073
:1049B0002500000025000100240000002400000064
:1049C0002400000024000000240001002300000057
:1049D000230000002300000023000000230000004B
:1049E000230000002300010022000000220000003C
:1049F000220000002200000022000000220001002E
:104A00002100000021000000210000002100000022
:104A10002100000021000000210001002000000012
:104A20002000000020000000200000002000000006
:104A30002000000020000000200001001F000000F6
:104A40001F0000001F0000001F0000001F000000EA
:104A50001F0000001F0001001E0000001E000000DB
:104A60001E0000001E00000020204D3630332000C4
:104A70003A0A0020286D6D2900205300205A00209A
:104A8000590020580020204D343235204600426124
:104A9000636B6C61736820636F6D70656E736174B6
:104AA000696F6E3A0A002055004C0046696C616DD2
:104AB000656E74206C6F61642F756E6C6F6164201D
:104AC0006C656E677468733A0A00204500205A00CE
:104AD00020204D393037205800537465707065724E
:104AE000206D6F746F722063757272656E74733AA5
:104AF0000A0020204D393030204B004C696E656132
:104B00007220416476616E63653A0A0020204D3858
:104B10003531205A005A2D50726F6265204F6666FB
:104B20007365740020440020490020204D33303448
:104B300020500020440020490020204D33303120F7
:104B400050005049442073657474696E67733A0A63
:104B50000020460020420020480020204D313435FE
:104B60002053004D6174657269616C2068656174E1
:104B7000757020706172616D65746572733A0A00B8
:104B800020204D3432302053004175746F2042652F
:104B900064204C6576656C696E673A0A00204500B2
:104BA000205A002059002058002054002053002093
:104BB000204D32303520420020453C6D61785F65E4
:104BC0005F6A65726B3E0020583C6D61785F785F6C
:104BD0006A65726B3E20593C6D61785F795F6A65EA
:104BE000726B3E205A3C6D61785F7A5F6A65726BCA
:104BF0003E00416476616E6365643A20423C6D69B3
:104C00006E5F7365676D656E745F74696D655F7502
:104C1000733E20533C6D696E5F66656564726174B6
:104C2000653E20543C6D696E5F74726176656C5FA1
:104C300066656564726174653E0020540020520010
:104C400020204D323034205000416363656C657222
:104C50006174696F6E2028756E6974732F733229C1
:104C60003A20503C7072696E745F616363656C3E9C
:104C700020523C726574726163745F616363656C3A
:104C80003E20543C74726176656C5F616363656C51
:104C90003E0A00204500205A0020590020204D32B5
:104CA00030312058004D6178696D756D2041636326
:104CB000656C65726174696F6E2028756E697473B6
:104CC0002F7332293A0A00204500205A002059004B
:104CD00020204D3230332058004D6178696D756D5C
:104CE000206665656472617465732028756E6974E9
:104CF000732F73293A0A00537465707320706572BC
:104D000020756E69743A0A0020204D3134392043F1
:104D1000203B20556E69747320696E2043656C7367
:104D20006975730A002020473231202020203B2063
:104D3000556E69747320696E206D6D0048617264F0
:104D4000636F6465642044656661756C74205365A7
:104D50007474696E6773204C6F616465640A00281F
:104D60002300002823000064000000E80300000086
:104D700000964300009643000000410000204200DE
:104D800000C9420000C9420000C8440000D24345A7
:104D90004550524F4D20496E697469616C697A655E
:104DA000640A00290A002062797465733B206372EB
:104DB0006320002073746F72656420736574746976
:104DC0006E67732072657472696576656420280069
:104DD000202863616C63756C6174656429210A0025
:104DE00020213D2000454550524F4D204352432045
:104DF0006D69736D61746368202D202873746F7200
:104E000065642920002053697A653A2000496E6460
:104E100065783A2000204D61726C696E3D563639D6
:104E2000290A00454550524F4D2076657273696FCF
:104E30006E206D69736D617463682028454550521A
:104E40004F4D3D004E6F20454550524F4D2E0A00AC
:104E5000290A002062797465733B20637263200025
:104E600053657474696E67732053746F7265642040
:104E700028004E6F20454550524F4D2E0A004545A3
:104E800050524F4D206461746173697A6520657278
:104E9000726F722E0A004175746F6C6576656C20B6
:104EA0006661696C65640A004175746F6C6576654E
:104EB0006C206661696C656400205A3A20002059B4
:104EC0003A200042656420583A20005761726E69AA
:104ED0006E673A20486F6D696E672042756D70206D
:104EE00044697669736F72203C20310A0002020423
:104EF000486F6D652025732573257320466972738D
:104F000074002046697273740A00486F6D65200052
:104F100020746F6F206C6F6E672065787472757384
:104F2000696F6E2070726576656E7465640A002024
:104F3000636F6C6420657874727573696F6E20702E
:104F4000726576656E7465640A0020453A00205AE1
:104F50003A0020593A00583A000000F0410000F0B1
:104F60004100000041FF01010000A0400000A040FE
:104F7000000000400000254300004B430000244394
:104F800000000000CDCC3B4300001F430000254340
:104F9000CDCC3B4300001F4300000000333373C1FE
:104FA0000000A0C020746F6F206C6F6E6720657862
:104FB00074727573696F6E2070726576656E746554
:104FC000640A0020636F6C6420657874727573697D
:104FD0006F6E2070726576656E7465640A00627526
:104FE00073793A2070617573656420666F72206909
:104FF0006E7075740A00627573793A20706175730A
:10500000656420666F7220757365720A006275733D
:10501000793A2070726F63657373696E670A004D29
:105020003131372050726F62652073756363657329
:105030007366756C0020496E76616C6964206578D2
:105040007472756465722000205A3A200020593A23
:10505000200042656420583A200050726F6265203B
:105060005A204F66667365743A20003F5A206F7568
:1050700074206F662072616E676520282D3220745F
:105080006F2035290A004D31343520533C696E6458
:1050900065783E206F7574206F662072616E67655B
:1050A0002028302D31290A00436C69636B20746F0E
:1050B00020526573756D652E2E2E00220A00556EE6
:1050C0006B6E6F776E20636F6D6D616E643A202238
:1050D00000454550524F4D204F4B0A004E6F204D1A
:1050E0006F76652E004543484F00494E464F0045B8
:1050F00052524F52530044525952554E00434F4D55
:105100004D554E49434154494F4E006F666600E588
:1051100050EA50EF50F650FD5044454255473A0092
:105120004C756C7A426F74204D696E69204C434413
:10513000204F46462E00205A0020590058002020BB
:105140004D61783A2000205A002059005800202054
:105150004D696E3A2000536F667420656E647374F7
:105160006F70733A20002569730025696D202569E9
:1051700073002569682025696D20256973002569FC
:1051800064202569682025696D20256973002569DB
:105190007920256964202569682025696D202569A5
:1051A00073005072696E742074696D653A20004D09
:1051B0003131332053002F2F20004361703A0043D8
:1051C00048414D4245525F54454D5045524154551A
:1051D0005245004D4F54494F4E5F4D4F444553008B
:1051E000544845524D414C5F50524F5445435449E9
:1051F0004F4E004155544F5245504F52545F534407
:105200005F5354415455530050524F4D50545F53C7
:105210005550504F525400454D455247454E435905
:105220005F50415253455200434153455F4C4947FB
:1052300048545F4252494748544E45535300544FD7
:1052400047474C455F4C494748545300534F4654D9
:10525000574152455F504F574552004255494C44C3
:105260005F50455243454E54004C4556454C494EBF
:10527000475F44415441005A5F50524F42450041FC
:1052800055544F4C4556454C005052494E545F4A78
:105290004F420050524F4752455353004155544FCF
:1052A0005245504F52545F54454D5000564F4C5547
:1052B0004D455452494300454550524F4D004249D7
:1052C0004E4152595F46494C455F5452414E5346F8
:1052D00045520053455249414C5F584F4E5F584F1D
:1052E0004646004649524D574152455F4E414D4555
:1052F0003A4D61726C696E20204649524D574152B9
:10530000455F56455253494F4E3A322E302E302E7D
:105310003137342045585452554445525F54595002
:10532000453A48617264656E6564537465656C5096
:105330006C757320534F555243455F434F44455F4F
:1053400055524C3A68747470733A2F2F636F6465CA
:105350002E616C6570686F626A656374732E636F2B
:105360006D2F646966667573696F6E2F4D41524C7F
:10537000494E2050524F544F434F4C5F5645525365
:10538000494F4E3A312E30204D414348494E455FFA
:10539000545950453A4C756C7A426F74204D696E81
:1053A00069204C43442045585452554445525F436C
:1053B0004F554E543A3120555549443A30383366AA
:1053C000363866312D303238652D343934632D3915
:1053D0003865312D663265306466616565396135E1
:1053E0000A0020284E6F7420796574206D65617302
:1053F00075726564290020204176657261676520B9
:105400006D65617375726564206261636B6C617355
:105410006820286D6D293A002020536D6F6F7468E5
:10542000696E6720286D6D293A20202020202020D9
:1054300020202020202020202020530020204261F6
:10544000636B6C6173682044697374616E6365207B
:10545000286D6D293A20202020202020200020289F
:1054600046312E30203D2066756C6C2C2046302E47
:1054700030203D206E6F6E65290A002020436F7238
:1054800072656374696F6E20416D6F756E742F461F
:105490006164652D6F75743A2020202020460061DC
:1054A00063746976653A0A00696E004261636B6CE9
:1054B00061736820436F7272656374696F6E200058
:1054C000205A0020506F736974696F6E616C2045BB
:1054D00072726F723A0A004E6F7A7A6C6520546964
:1054E00070204F757465722044696D656E73696FC5
:1054F0006E733A0A002020546F703A200020204634
:10550000726F6E743A200020204C6566743A200059
:105510004261636B6C6173683A0A00205A0043650C
:105520006E7465723A0A00202046726F6E743A20DB
:105530000020204C6566743A20002020546F703A99
:10554000200053696465733A0A00426564204C6523
:1055500076656C696E6720004661696C65642074CD
:105560006F20656E61626C6520426564204C6576D3
:10557000656C696E670A00426564204C6576656CEF
:1055800020436F7272656374696F6E204D6174722F
:1055900069783A000A0A426564204C6576656C2099
:1055A000436F7272656374696F6E204D61747269C6
:1055B000783A00202B000A436F7272656374656449
:1055C00020426564204865696768742076732E20E0
:1055D00042656420546F706F6C6F67793A0A0020DF
:1055E0002B000A4265642048656967687420546F1F
:1055F000706F6772617068793A0A2020202B2D2D18
:105600002D204241434B202D2D2B0A2020207C2091
:10561000202020202020202020207C0A204C207CBC
:1056200020202020282B29202020207C20520A20E6
:1056300045207C20202020202020202020207C208D
:10564000490A2046207C20282D29204E20282B295D
:10565000207C20470A2054207C202020202020204D
:10566000202020207C20480A2020207C2020202070
:10567000282D29202020207C20540A2020207C2036
:10568000202020202020202020207C0A2020204FA5
:105690002D2D2046524F4E54202D2D2B0A202830E0
:1056A0002C30290A000A4D65616E206F66207361F7
:1056B0006D706C656420706F696E74733A200020A1
:1056C000643A200020623A200045716E20636F65C5
:1056D0006666696369656E74733A20613A200050AA
:1056E000726F62696E6720506F696E742025692F32
:1056F0002569002E0A002F0050726F62696E6720C4
:105700006D65736820706F696E74200020284452A4
:105710005952554E2900473239204175746F204245
:105720006564204C6576656C696E67003F20284C87
:105730002C522C462C4229206F7574206F662062F3
:105740006F756E64732E0A003F50726F6265207031
:105750006F696E74732028592920696D706C6175AA
:105760007369626C652028322D32292E0A003F5061
:10577000726F626520706F696E74732028582920DB
:10578000696D706C61757369626C652028322D32A9
:10579000292E0A003F2856296572626F7365206CB6
:1057A0006576656C20696D706C61757369626C6596
:1057B0002028302D34292E0A0043757272656E74CC
:1057C0002066696C653A2000456E642066696C65E8
:1057D000206C6973740A00426567696E2066696CA3
:1057E00065206C6973740A00416476616E6365209C
:1057F0004B3D003F4B2076616C7565206F757420C2
:105800006F662072616E67652028302D3130292E39
:105810000A004D31313720486F7420656E6420686E
:10582000656174696E672E2E2E0A4D313034205317
:105830003137300A473238204F310A4D3131372065
:10584000576970696E67206E6F7A7A6C650A54309A
:105850000A473120583131352059313734205A31F7
:10586000302046343030300A4D3130392052313713
:10587000300A4731205A310A4D3131340A4731203C
:105880005831313520593137340A473120583435B1
:1058900020593137340A47312058313135205931B8
:1058A00037340A47312058343520593137340A47C4
:1058B00031205831313520593137340A4731205899
:1058C000343520593137340A4731205831313520A9
:1058D000593137340A47312058343520593137345B
:1058E0000A4731205831313520593137340A473190
:1058F0002058343520593137340A47312058313156
:105900003520593137340A47312058343520593140
:1059100037340A4731205A31350A4D3430300A4D78
:1059200031303620533235350A473020583020592F
:105930003136384D31303920523136300A4D313020
:1059400037004732380020466C6F773A20002064D9
:105950003A0020693A0020703A00204500205A00A1
:10596000205900204D393220580043290A00616235
:105970006C656420286D696E2074656D702000640C
:10598000697300656E00436F6C642065787472758E
:10599000646573206172652000205400205200412C
:1059A0006363656C65726174696F6E3A205000497B
:1059B0006E76616C69642065787472756465720ACC
:1059C0000020643A0020693A0020703A00536C6568
:1059D00065702E2E2E0047322F47332062616420DF
:1059E000706172616D65746572730A0050726F62E6
:1059F00065205A204F66667365743A2000446F6EC6
:105A00006520736176696E672066696C652E0A0091
:105A100053442072656164206572726F720A00449B
:105A20006F6E65207072696E74696E672066696C4E
:105A3000650A004D32390053544F505045442E20D2
:105A4000005072696E7465722073746F7070656453
:105A50002064756520746F206572726F72732E20DA
:105A600046697820746865206572726F7220616E75
:105A70006420757365204D39393920746F20726543
:105A800073746172742E202854656D706572617430
:105A90007572652069732072657365742E20536575
:105AA0007420697420616674657220726573746114
:105AB0007274696E67290A004E6F20436865636BD4
:105AC00073756D2077697468206C696E65206E75DA
:105AD0006D6265722C204C617374204C696E653A5E
:105AE00020004E6F20436865636B73756D20776986
:105AF0007468206C696E65206E756D6265722C200D
:105B00004C617374204C696E653A2000636865636C
:105B10006B73756D206D69736D617463682C204CB7
:105B2000617374204C696E653A20004C696E652083
:105B30004E756D626572206973206E6F74204C61C2
:105B40007374204C696E65204E756D6265722B31E1
:105B50002C204C617374204C696E653A20004D31E5
:105B6000313000526573656E643A20002042002097
:105B700050006F6B00220A00656E7175657565696E
:105B80006E67202200504944204175746F74756E11
:105B900065206661696C65642120426164206578D6
:105BA000747275646572206E756D6265720A00426A
:105BB000656420436F6F6C696E672E2E2E00426500
:105BC000642048656174696E672E2E2E006F6B002D
:105BD0004732385859002020506C616E6E65724211
:105BE000756666657242797465733A200020467264
:105BF0006565204D656D6F72793A2000436F6D7059
:105C0000696C65643A204F6374202039203230314A
:105C1000390A00207C20417574686F723A2028414F
:105C20006C657068204F626A6563747320496E63A7
:105C30002E2C204C756C7A426F7420476974205268
:105C400065706F7369746F7279290A004F637420ED
:105C50002039203230313931343A32353A35360054
:105C6000204C61737420557064617465643A20003F
:105C7000322E302E302E3137340A004D61726C696D
:105C80006E0020536F66747761726520526573658C
:105C9000740A00205761746368646F6720526573EB
:105CA00065740A002042726F776E206F75742052FF
:105CB000657365740A002045787465726E616C20A6
:105CC00052657365740A00506F77657255700A00EB
:105CD00073746172740A004B494C4C45442E200089
:105CE0005072696E7465722068616C7465642E20F0
:105CF0006B696C6C28292063616C6C6564210A00F7
:105D00004B494C4C20636175736564206279204B6C
:105D1000494C4C20627574746F6E2F70696E0A0066
:105D20004B494C4C20636175736564206279207423
:105D30006F6F206D75636820696E61637469766545
:105D40002074696D65202D2063757272656E7420F4
:105D5000636F6D6D616E643A20004D3132310A47D8
:105D600030205A31300A4732382058302059300A12
:105D70004731320A4D31303920523136300A4D34F4
:105D800030300A4D3131372050726F62696E6720B2
:105D90006265640070726F62655F726577697065D5
:105DA000004175746F6C6576656C206661696C6521
:105DB00064004D31313720426564206C6576656C36
:105DC000696E67206661696C65642E0A4730205AE7
:105DD00031300A47302045300A4D333030205032C0
:105DE0003520533838300A4D33303020503530208C
:105DF00053300A4D3330302050323520533838304C
:105E00000A4D333030205035302053300A4D333076
:105E1000302050323520533838300A47342053313F
:105E20000070726F62655F6661696C6564005072D4
:105E30006F7465637465642050696E0A0025301DB7
:105E40000C1E282924311C0B184527232F1B0A1749
:105E50004443222B1A4142043803FF360408060645
:105E60000001894740897593E3AA45C6E400E6002E
:105E7000E200E000959311241FBECFEFD1E2DEBF18
:105E8000CDBF00E00CBF13E0A0E0B2E0E6EEF7EC1F
:105E900002E00BBF02C007900D92A63EB107D9F7F2
:105EA00026E1A6EEB3E001C01D92AB3DB207E1F7DB
:105EB0001FE2CAE3DFE200E006C021970109802F5C
:105EC000FE010F942359C133D10780E00807A9F7D9
:105ED0000E94A83B0D94E1630C9400001F920F9266
:105EE0000FB60F9211242F933F938F939F93AF93ED
:105EF000BF938091E7039091E803A091E903B091EB
:105F0000EA033091E60323E0230F2D3720F40196B6
:105F1000A11DB11D05C026E8230F0296A11DB11DCC
:105F20002093E6038093E7039093E803A093E903AB
:105F3000B093EA038091EB039091EC03A091ED0301
:105F4000B091EE030196A11DB11D8093EB039093D8
:105F5000EC03A093ED03B093EE03BF91AF919F913B
:105F60008F913F912F910F900FBE0F901F9018951A
:105F70002FB7F8946091E7037091E8038091E903EB
:105F80009091EA032FBF08953FB7F8948091EB03F7
:105F90009091EC03A091ED03B091EE0326B5A89B80
:105FA00005C02F3F19F00196A11DB11D3FBFBA2FAB
:105FB000A92F982F8827820F911DA11DB11DBC010B
:105FC000CD0142E0660F771F881F991F4A95D1F7D0
:105FD00008958F929F92AF92BF92CF92DF92EF92ED
:105FE000FF926B017C01D0DF4B015C01C114D10435
:105FF000E104F104F1F09CD3C7DFDC01CB01881987
:106000009909AA09BB09883E9340A105B10570F31F
:1060100021E0C21AD108E108F10888EE880E83E079
:10602000981EA11CB11CC114D104E104F10421F794
:10603000DDCFFF90EF90DF90CF90BF90AF909F901B
:106040008F9008958230910538F0880F991F880F3E
:10605000991F05970197F1F70895789484B58260A8
:1060600084BD84B5816084BD85B5826085BD85B5FC
:10607000816085BDEEE6F0E0808181608083E1E8AB
:10608000F0E01082808182608083808181608083E3
:10609000E0E8F0E0808181608083E1EBF0E08081E6
:1060A00084608083E0EBF0E0808181608083E1E9BF
:1060B000F0E0808182608083808181608083E0E97C
:1060C000F0E0808181608083E1EAF0E0808182609D
:1060D0008083808181608083E0EAF0E0808181605C
:1060E0008083E1E2F1E08081826080838081816051
:1060F0008083E0E2F1E0808181608083EAE7F0E084
:1061000080818460808380818260808380818160DF
:1061100080838081806880831092C10008951F93DE
:10612000CF93DF93182FEB0161E016D1209711F484
:1061300060E004C0CF3FD10531F461E0812FDF91F1
:10614000CF911F9145C1E12FF0E0EB5FFC4FE4914F
:106150004E2F50E0FA013197E231F10508F09DC071
:106160008827EE58FF4F8F4F0D94235984B58068D0
:1061700084BDC7BD97C084B5806284BDC8BD92C0D0
:1061800080918000806880938000D0938900C093C4
:10619000880088C080918000806280938000D093C6
:1061A0008B00C0938A007EC08091800088608093BD
:1061B0008000D0938D00C0938C0074C08091B0009B
:1061C00080688093B000C093B3006CC08091B00031
:1061D00080628093B000C093B40064C0809190004E
:1061E000806880939000D0939900C09398005AC023
:1061F00080919000806280939000D0939B00C09328
:106200009A0050C080919000886080939000D09355
:106210009D00C0939C0046C08091A0008068809340
:10622000A0008091A0008F7B8093A000D093A90054
:10623000C093A80037C08091A00080628093A00026
:10624000D093AB00C093AA002DC08091A0008860BD
:106250008093A000D093AD00C093AC0023C0809188
:106260002001806880932001D0932901C0932801E8
:1062700019C080912001806280932001D0932B016E
:10628000C0932A010FC08091200188608093200173
:10629000D0932D01C0932C0105C0C038D1050CF05E
:1062A0004CCF46CFDF91CF911F91089590E0FC0134
:1062B0003197E231F10508F04EC08827EC57FF4FC7
:1062C0008F4F0D942359809180008F7703C0809168
:1062D00080008F7D80938000089580918000877F6B
:1062E000F9CF84B58F7702C084B58F7D84BD0895C2
:1062F0008091B0008F7703C08091B0008F7D809334
:10630000B0000895809190008F7707C08091900031
:106310008F7D03C080919000877F809390000895C7
:106320008091A0008F7707C08091A0008F7D03C06F
:106330008091A000877F8093A00008958091200124
:106340008F7707C0809120018F7D03C0809120014D
:10635000877F809320010895CF93DF9390E0FC0125
:10636000E55BFC4F2491FC01EF56FC4F84918823A0
:1063700061F190E0880F991FFC01E55FFB4FC5912B
:10638000D491FC01EF50FC4FA591B491611109C06B
:106390009FB7F8948881209582238883EC912E23DF
:1063A0000BC0623061F49FB7F8943881822F8095DA
:1063B00083238883EC912E2B2C939FBF06C08FB72D
:1063C000F894E8812E2B28838FBFDF91CF91089519
:1063D0001F93CF93DF93282F30E0F901EB5FFC4F41
:1063E0008491F901E55BFC4FD491F901EF56FC4F24
:1063F000C491CC23C1F0162F811158DFEC2FF0E0AF
:10640000EE0FFF1FEF50FC4FA591B4918FB7F8949A
:10641000111105C09C91ED2FE095E92302C0EC918C
:10642000ED2BEC938FBFDF91CF911F910895CF9308
:10643000DF93282F30E0F901EB5FFC4F8491F901E5
:10644000E55BFC4FD491F901EF56FC4FC491CC238E
:1064500089F081112BDFEC2FF0E0EE0FFF1FE952E6
:10646000FC4FA591B491EC91ED2381E090E021F4F3
:1064700080E002C080E090E0DF91CF910895089520
:106480001F920F920FB60F9211240BB60F922F93FB
:106490003F934F935F936F937F938F939F93AF93AC
:1064A000BF93EF93FF93E0910802F09109021995D1
:1064B000FF91EF91BF91AF919F918F917F916F91DC
:1064C0005F914F913F912F910F900BBE0F900FBE98
:1064D0000F901F9018951F920F920FB60F921124D4
:1064E0000BB60F922F933F934F935F936F937F93CE
:1064F0008F939F93AF93BF93EF93FF93E0910A0223
:10650000F0910B021995FF91EF91BF91AF919F917F
:106510008F917F916F915F914F913F912F910F904C
:106520000BBE0F900FBE0F901F9018951F920F92E9
:106530000FB60F9211240BB60F922F933F934F93E8
:106540005F936F937F938F939F93AF93BF93EF93DB
:10655000FF93E0910C02F0910D021995FF91EF91DC
:10656000BF91AF919F918F917F916F915F914F916B
:106570003F912F910F900BBE0F900FBE0F901F9069
:1065800018951F920F920FB60F9211240BB60F920F
:106590002F933F934F935F936F937F938F939F932B
:1065A000AF93BF93EF93FF93E0910E02F0910F0230
:1065B0001995FF91EF91BF91AF919F918F917F912D
:1065C0006F915F914F913F912F910F900BBE0F9064
:1065D0000FBE0F901F9018951F920F920FB60F923B
:1065E00011240BB60F922F933F934F935F936F93AA
:1065F0007F938F939F93AF93BF93EF93FF93E0911C
:106600000402F09105021995FF91EF91BF91AF91AE
:106610009F918F917F916F915F914F913F912F91BA
:106620000F900BBE0F900FBE0F901F9018951F92EA
:106630000F920FB60F9211240BB60F922F933F9328
:106640004F935F936F937F938F939F93AF93BF937A
:10665000EF93FF93E0910602F09107021995FF91E5
:10666000EF91BF91AF919F918F917F916F915F91CA
:106670004F913F912F910F900BBE0F900FBE0F9037
:106680001F9018951F920F920FB60F9211240BB600
:106690000F922F933F934F935F936F937F938F93BB
:1066A0009F93AF93BF93EF93FF93E0911002F0910C
:1066B00011021995FF91EF91BF91AF919F918F9129
:1066C0007F916F915F914F913F912F910F900BBEF2
:1066D0000F900FBE0F901F9018951F920F920FB63C
:1066E0000F9211240BB60F922F933F934F935F930A
:1066F0006F937F938F939F93AF93BF93EF93FF938A
:10670000E0911202F09113021995FF91EF91BF9160
:10671000AF919F918F917F916F915F914F913F9139
:106720002F910F900BBE0F900FBE0F901F901895DA
:1067300008951F93CF93DF93EC011D821C821F826B
:106740001E82198681E0888782E28A871F861E86DC
:10675000FE01B396CE01C1962FEF2193E817F907FA
:10676000E1F711E018A3CE0122D61F8B188E198EE7
:1067700080E48A8F1B8E88EA97E39AAB89ABDF911E
:10678000CF911F910895DB01ED91FC911994EF9247
:10679000FF921F93CF93DF931F921F92CDB7DEB767
:1067A0007C01DC01D196ED91FC91D29782E0698366
:1067B0007A83199520E030E04AE069817A81C70147
:1067C000E2DF182FD701D196ED91FC91D29783E0AB
:1067D0001995D701D196ED91FC91D29780E019954A
:1067E000812F0F900F90DF91CF911F91FF90EF902D
:1067F00008950F931F93CF93DF93EC018B01E9A9C9
:10680000FAA982E01995E9A9FAA981E0199520E091
:1068100030E044E1B801CE01B6DF9E012D5C3F4F70
:1068200047E1B801CE01AFDFE9A9FAA980E0DF9125
:10683000CF911F910F911994EF92FF921F93CF93D5
:10684000DF93EC017B01E9A9FAA982E01995E9A996
:10685000FAA981E0199520E030E045E1B701CE01C9
:1068600092DF182F882339F09E012D5C3F4F47E1BE
:10687000B701CE0188DFE9A9FAA980E01995812F37
:10688000DF91CF911F91FF90EF900895FC01448F0D
:10689000258F9C01245E3F4F42E375CFCF93DF935A
:1068A0001F92CDB7DEB79E012F5F3F4F46E46BDFEF
:1068B00089810F90DF91CF910895CF93DF931F923D
:1068C000CDB7DEB79E012F5F3F4F47E45CDF898184
:1068D0000F90DF91CF91089520E030E048E453CF4E
:1068E000CF93DF93EC016A817B81D8DF88836A8153
:1068F0007B81CE01E2DF89836A817B81CE01ECDF7F
:106900008B879E012D5C3F4F6A817B8147E1CE01E1
:10691000DF91CF9138CFCF93DF93EC016A817B81F8
:1069200036DF882319F0CE01DBDF81E0DF91CF91E4
:1069300008958F929F92AF92BF92CF92EF920F9352
:10694000CF93DF931F921F92CDB7DEB74C015B014F
:106950002A834983EEDEF401B382A282498147A3F0
:106960002A8120A705A3E4A2C3A2C4010F900F901F
:10697000DF91CF910F91EF90CF90BF90AF909F900C
:106980008F90C9CFFC016281738133CFCF93DF93A6
:10699000EC01EE85FF85309709F019956A817B81BE
:1069A000CE01DF91CF9148CF362F242FFC01628199
:1069B0007381432F6BCF0F93FC0182819381648F8E
:1069C000458F278F068F9F01245E3F4F4BE3BC010D
:1069D000CF010F91D8CEFC0160A30895BF92CF9252
:1069E000DF92EF92FF920F931F93CF93DF936C018F
:1069F000D62FB42EC22F7801CC2369F0F701049171
:106A000020E04B2D6D2FC601D6DFFFEFEF1AFF0AF6
:106A1000C150D85FF1CFDF91CF911F910F91FF90BF
:106A2000EF90DF90CF90BF9008958F929F92AF929A
:106A3000BF92CF92DF92EF92FF920F931F93CF936B
:106A4000DF935C01C62EC42FD22ED02F220F220F2F
:106A5000220F1ED0882379F0DC0F8D2C912CCD17BE
:106A600051F087012D2D4C2F6C2DC501B7DFE80C9F
:106A7000F91CCF5FF4CFDF91CF911F910F91FF9061
:106A8000EF90DF90CF90BF90AF909F908F90089540
:106A90000F93FC010150040F84A996A9941718F0D4
:106AA000081728F402C0081750F0041740F42150CA
:106AB000260F83A995A9961720F4281720F480E0C3
:106AC00007C0281720F481E0261710F0F8CF81E0E6
:106AD0000F91089581E008952EE93FE0009729F095
:106AE000F9013197F1F70197F9CF0895FC0112826E
:106AF00080818150838314820895FC01808192817A
:106B0000980F92832181921760F494819F5F948300
:106B10009381890F821710F08FEF820F838381E0BA
:106B2000089580E00895FC0191E08381861708F4C0
:106B300090E031E0461708F030E0832F892B21E008
:106B40005281451708F420E02823832F8923822BC4
:106B50000895DC01FB01108212968C9112978183BB
:106B600015968C9115978150828313968C9183830F
:106B70000895FB0141812381213029F0233031F434
:106B800068EF640F04C0642F485F01C0642FCBCF4F
:106B9000DC0115962C9115971696ED91FC9117979F
:106BA000CF01820F911D820F911D1192E817F907F5
:106BB000E1F70895FC01A681B7818281481B858198
:106BC000483018F0A80FB11D4770382F369536950C
:106BD0003695562F577080E890E002C095958795BE
:106BE0005A95E2F7439F402D112466956695669568
:106BF000E62FF0E0E40FF11DEA0FFB1F30812223A6
:106C000011F0832B02C08095832380830895FB01BC
:106C10004181DC0112962C911297421760F0139675
:106C20002C911397241738F0608115962C916217D8
:106C300010F42481BFCF0895CF92DF92FF920F937B
:106C40001F93CF93DF936C01EB01FA809B8191300E
:106C500051F030F0923049F0933051F41FEF09C0F9
:106C600010E001E007C011E004C010E00FEF02C027
:106C700010E000E0F7FE03C0BE01C601C8DF988146
:106C8000900F98839981910F9983FF0C99F7DF9169
:106C9000CF911F910F91FF90DF90CF9008950F93A8
:106CA0001F93CF93DF938901FB01C281D3814233CC
:106CB000D9F058F44531E1F0473109F1443141F55B
:106CC000CE0166DFCE0112DF23C04634E1F0473447
:106CD000E1F04B33E9F4B901CE014BDF8823C1F079
:106CE000B801CE01A9DF14C0B901CE0190DF10C0F8
:106CF000CE0103DF882369F0CE014ADF09C0B90164
:106D0000CE0127DF05C08D8101C08981F801808314
:106D100081E0DF91CF911F910F910895CF92DF9283
:106D2000EF92FF920F931F93CF93DF937C01D62FA7
:106D3000D42EC22F122FC62EC20E6C2D611B1830FE
:106D400038F00FEF20E04D2DC70135DE1850F5CF9C
:106D50006C2F687F6D0F2C2F277071F097E029271B
:106D60002F5F27700FEF10E001C0000F2A95EAF7A0
:106D700020E04D2DC7011FDEDF91CF911F910F91B4
:106D8000FF90EF90DF90CF900895CF92DF92EF9237
:106D9000FF920F931F93CF93DF937C01D62ED42FB6
:106DA000C22F122FC42EC20E4C2D411B183038F0AA
:106DB0000FEF21E06D2DC701FEDD1850F5CF4C2FF0
:106DC000487F4D0F2C2F277071F097E029272F5FF8
:106DD00027700FEF10E001C0000F2A95EAF721E0BD
:106DE0006D2DC701E8DDDF91CF911F910F91FF90CD
:106DF000EF90DF90CF900895EF92FF920F931F9343
:106E0000CF93DF93EC01162FF42EE22E01E040DE4B
:106E1000882359F02E2D4F2D612FCE01DF91CF9178
:106E20001F910F91FF90EF9079CFDF91CF911F913C
:106E30000F91FF90EF900895EF92FF920F931F93A1
:106E4000CF93DF93EC01162FF42EE22E022F21E0D8
:106E50001FDE882359F02E2D4F2D612FCE01DF919B
:106E6000CF911F910F91FF90EF908FCFDF91CF9136
:106E70001F910F91FF90EF900895DF92EF92FF9294
:106E80000F931F93CF93DF937C01162FC42FD22E25
:106E9000D02FFEDD8823F9F02D2D4C2F612FC70157
:106EA0003DDF2D2F4C2F612FC7016FDF6FEF6D0D71
:106EB000610F2D2F4C2FC70168DF4FEF4D0F4C0F87
:106EC0002D2D612FC701DF91CF911F910F91FF9061
:106ED000EF90DF9023CFDF91CF911F910F91FF9023
:106EE000EF90DF900895EF92FF920F931F93CF934F
:106EF000DF937C01D62F122FC42F040F212F4C2F8C
:106F00006D2FC7010BDFCF5F0C13F8CFDF91CF914F
:106F10001F910F91FF90EF900895DF92EF92FF92F3
:106F20000F931F93CF93DF93EC01162FF42EE22ED5
:106F3000AFDD882329F02E2D4F2D612FCE01D3DF19
:106F4000DF91CF911F910F91FF90EF90DF90089507
:106F50000895FC01E60FF11D849190E0982F882799
:106F60003196E4918E0F911D0895FC01849108954E
:106F7000FCDF882321F0823011F083E0089586E061
:106F8000089580E00895FC018081089566E0E1CFD6
:106F900068E0DFCF0A96FC01849108950B96FC010E
:106FA00084910895DC011496ED91FC91159731962A
:106FB00084910895BF92CF92DF92EF92FF920F9348
:106FC0001F93CF93DF938C01E62EDC011496CD91B5
:106FD000DC911597CE01C9DFF82EF80184819581E7
:106FE000C7DFC82EF1E0FF1203C02FE0B22E02C0AF
:106FF000BB24BA94D80114968D919C911597CADF41
:10700000F82EF80184819581C9DFD82ED801149615
:107010008D919C911597BCDFB0E6BE1538F40097B2
:1070200029F0C80FD91F91E6F92E0FC0F80184810D
:107030009581ACDFF0E4FE1538F4009729F0C80F15
:10704000D91F81E4F82E01C06196DE1490F4D801B6
:1070500050961C92509753961C92539754961C929C
:10706000549751961C92519752961C9280E090E052
:1070700066C0DF1460F38C2D90E0FE0124912F3F59
:1070800011F4219657C0FE104CC0D80114968D9172
:107090009C9115976ADF9E012F5F3F4FFE01882369
:1070A00011F08230E1F48491D80153968C93539778
:1070B000F901249154962C935497FE013396E49150
:1070C0005096EC935097FE013496E4915196EC93D0
:1070D0005197FE013596E4915296EC9320C084912D
:1070E000982F9F709250D80152969C9352978295F8
:1070F0008F7051968C935197F9012491822F8F7044
:1071000054968C93549722952F7053962C935397A3
:10711000FE013296E491E295EF705096EC93CE0129
:107120000EC0FE013296E491EB219C012E0F311D21
:10713000C20FD31FFD1409F48ACFF3949ECFDF91C1
:10714000CF911F910F91FF90EF90DF90CF90BF9064
:1071500008954F925F926F927F929F92AF92BF92EB
:10716000CF92DF92EF92FF920F931F93CF93DF9313
:107170001F92CDB7DEB72C01C62E942E622F1ADFD8
:107180007C01892B09F43AC0F20184819581F0DEFB
:10719000B82EF201138904898189C80E8289981A50
:1071A000D92CD01A212F4D2D6C2DC20171DC8823D2
:1071B00011F1EB0CF11C195F169516951695612EC1
:1071C000712CD914C1F03C2D57018A2D8E198117CD
:1071D00070F4F501049120E04D2D632FC201398335
:1071E000EADBFFEFAF1ABF0A3981385FEECFE60C5A
:1071F000F71CD394E6CFF201808901C080E00F90A4
:10720000DF91CF911F910F91FF90EF90DF90CF9082
:10721000BF90AF909F907F906F905F904F90089538
:107220000F931F93CF93DF9300D0CDB7DEB78C01C0
:10723000DC015596ED91FC9156972B834A83698327
:1072400019954A81480F2B816981C8010F900F90D1
:107250000F90DF91CF911F910F917BCFAF92BF9293
:10726000DF92EF92FF920F931F93CF93DF931F92C2
:107270001F92CDB7DEB77C01D62E042FDC015596C8
:10728000ED91FC91569729833A831995080F29812E
:10729000A22E3A81B32E10E0F50121915F01222345
:1072A00039F0402F6D2DC70154DFD80E180FF4CFE1
:1072B000812F0F900F90DF91CF911F910F91FF9031
:1072C000EF90DF90BF90AF900895DF92EF92FF9222
:1072D0000F931F93CF93DF937C01D62FD42E890178
:1072E000DC015596ED91FC9156971995D80EC0E0AA
:1072F000F8012491222349F04D2D6D2FC70129DF7C
:10730000D80FC80F0F5F1F4FF3CF8C2FDF91CF9196
:107310001F910F91FF90EF90DF900895DC0114967C
:107320002D913C9115972115310509F43FC05796D1
:107330008C915797F901811108C03596E4915896C0
:10734000EC935897F9013C9611C0813041F43F9677
:10735000E4915896EC935897F901709607C03D96C2
:10736000E4915896EC935897F9013E96E49159961A
:10737000EC93599758968C915897082E000C990BBE
:1073800059962C915997821B910927FD93955A96EE
:107390002C915A97203441F0829FC001112426E09D
:1073A000969587952A95E1F75B968C93089521EC45
:1073B00037E3FC01368B258B0895CF92DF92EF9255
:1073C000FF920F931F93CF93DF938C017B016A0190
:1073D000CB01FA011995D82F882311F1682FC80124
:1073E000E9DDF801C189C195FFEFEF1AFF0AC70176
:1073F000F6011995F801882351F08089C80FC7015B
:10740000F6011995D82F682FC801D4DDEDCFD03201
:1074100021F091898389890F01C080898C0F01C077
:1074200080E0DF91CF911F910F91FF90EF90DF905F
:10743000CF90089543EC57E3C0CFCF93DF93FC0187
:10744000248135812617370741F0EC017583648369
:1074500065DF81EC97E39E8B8D8BDF91CF91089553
:10746000CF93DF9300D01F92CDB7DEB761157105C2
:107470008105910579F09B01AC0169833A834B83C7
:107480005C830F94B85929813A814B815C810F94B8
:10749000075903C060E070E0CB010F900F900F9090
:1074A0000F90DF91CF910895CF92DF92EF92FF92EC
:1074B0000F931F9362177307840795077CF4890164
:1074C0009A016B017C01C901B8016C197D098E0913
:1074D0009F09C6DF6C0D7D1D8E1D9F1D1F910F9195
:1074E000FF90EF90DF90CF9008954F925F926F9250
:1074F0007F92AF92BF92CF92DF92EF92FF920F9363
:107500001F93CF93DF93CDB7DEB729013A019B01DB
:10751000AC0124193509460957098A899B89AC8928
:10752000BD89BC01CD016A197B098C099D090F94A5
:10753000A358A801970124193509460957090F9442
:107540000759CA01B9016A0D7B1D8C1D9D1DDF9174
:10755000CF911F910F91FF90EF90DF90CF90BF9050
:10756000AF907F906F905F904F90089580E090E093
:1075700008950895CF92DF92EF92FF920F931F9399
:10758000CF93DF936C017A018B01C0E0D0E0CE1580
:10759000DF0589F0D8016D918D01D601ED91FC9147
:1075A0000190F081E02DC6011995892B11F47E011F
:1075B00002C02196ECCFC701DF91CF911F910F91AF
:1075C000FF90EF90DF90CF9008956115710579F0ED
:1075D000FB0101900020E9F73197AF01461B570BE3
:1075E000DC01ED91FC910280F381E02D199480E0A3
:1075F00090E00895EACFDC01ED91FC910190F081DB
:10760000E02D19944F925F926F927F92EF92FF92CA
:107610000F931F93CF93DF93CDB7DEB7A1970FB62C
:10762000F894DEBF0FBECDBF7C01FA01CB0119A2D9
:10763000223008F42AE08E010F5D1F4F422E512C9C
:10764000612C712CBF01A30192010F94E558F9013F
:10765000CA01015011096A3014F4605D01C0695C0F
:10766000D8016C93232B242B252B61F7B801C7017C
:10767000ACDFA1960FB6F894DEBF0FBECDBFDF9191
:10768000CF911F910F91FF90EF907F906F905F903F
:107690004F900895CF92DF92EF92FF920F931F9336
:1076A000CF93DF93EC016A017B012115310579F459
:1076B000E881F9810190F081E02D642FDF91CF9175
:1076C0001F910F91FF90EF90DF90CF9019942A3087
:1076D0003105D9F477FF18C06DE28DDF8C014427A6
:1076E0005527BA014C195D096E097F092AE0CE01C0
:1076F00089DF800F911FDF91CF911F910F91FF9034
:10770000EF90DF90CF9008952AE0B701A601CE0157
:10771000DF91CF911F910F91FF90EF90DF90CF906D
:1077200071CF9A01AB01770F660B770BB3CFCF9276
:10773000EF920F93FC0113AE14AE15AE0496F9D878
:107740000F91EF90CF90089580E090E00895089514
:107750000E942D30FCDF0F940B54C0E0D0E00F945A
:107760009D542097E1F30E940000F9CFE0E1F4E09E
:1077700083AF64AF08954AE050E0BC0180E194E03B
:10778000D0CFEF92FF920F931F93CF93DF937A01A5
:107790006F3F71058105910509F040F480E194E0A7
:1077A0002ADF84E194E0FEDB90E014C0C0914B043A
:1077B000D0914C044D2F50E0EC2FF0E08B019C0158
:1077C000BF0184E194E05CD6C80FC0934B04D09312
:1077D0004C049927DF91CF911F910F91FF90EF906B
:1077E0000895EF92FF920F931F93CF93DF938B0136
:1077F000C0E1D4E0FBACECAC4E2D50E06F2D70E05E
:107800009C0184E194E094D6F80EFBAEECAE99278F
:10781000DF91CF911F910F91FF90EF900895EF921C
:10782000FF920F931F93CF93DF938B01C0E1D4E0BE
:10783000FBACECAC4E2D50E06F2D70E09C0184E170
:1078400094E0C2D6F80EFBAEECAE9927DF91CF9153
:107850001F910F91FF90EF9008956FEF7FEFC1CFD1
:10786000CF93DF93EA0182DFCE01DF91CF91F5CF95
:107870004FEF5FEF86CFCF93DF9300D01F92CDB74E
:10788000DEB729833A834B835C8370DF29813A8199
:107890004B815C81CA01B9010F900F900F900F903E
:1078A000DF91CF91E5CF0F931F93CF93DF931F927B
:1078B000CDB7DEB7082F8EE496E00E94A081182F86
:1078C000863168F48EE496E0C8DF153109F43DC0D6
:1078D00060E270E080E090E0CBDF1F5FF6CFCE018A
:1078E00001960E94558560E870E07BDF89818531D3
:1078F00020F56EE270E080E090E0BADF198114318B
:10790000E1F06EE270E080E090E0B2DF1331A9F0C8
:1079100089812EEF3FEF281B310986E0829FB0015D
:10792000839F700D112460587F4F8EE496E059DFDD
:1079300060E270E080E090E09BDF8091EF038017D1
:1079400021F00093EF030E9437850F90DF91CF91D4
:107950001F910F9108954F925F926F927F928F9235
:107960009F92AF92BF92CF92DF92EF92FF920F93CE
:107970001F93CF93DF93CDB7DEB72D970FB6F89453
:10798000DEBF0FBECDBF80914406882309F48AC0B4
:107990006091BB0C7091BC0C072E000C880B990BEE
:1079A0000F943D5611E02091B70C3091B80C4091E6
:1079B000B90C5091BA0C0F949E5718160CF010E0A9
:1079C0006091950C7091960C072E000C880B990B0A
:1079D0000F943D562091910C3091920C4091930C54
:1079E0005091940C0F949E5718160CF41068109335
:1079F000020480906B0290906C02A0906D02B09097
:107A00006E0220E030E0A901C501B4010F949B553E
:107A100087FD05C020E030E040E05FE304C020E0E7
:107A200030E040E05FEBC501B4010F94C2540F9405
:107A30000A56CB010F943949BC018DEF93E00F94A6
:107A4000335E80906F0290907002A0907102B090AF
:107A5000720220E030E0A901C501B4010F949B55EA
:107A600087FD05C020E030E040E05FE304C020E097
:107A700030E040E05FEBC501B4010F94C2540F94B5
:107A80000A56CB010F943949BC0188EF93E00F945B
:107A9000335E83E792E00F944B4EBC0180EF93E09E
:107AA0000F94335E0E94DF83182F81E055D620911A
:107AB000020427FF03C048E00CE002C042E102E0FC
:107AC0008091480490E044977CF480914A048417A4
:107AD00058F027FD36C18AE497E17C0123E060E598
:107AE00084E194E00E941535809148048431B8F413
:107AF00080914A04823098F0112309F425C18091C5
:107B0000B20C882309F420C18AEB96E17C0102E1E2
:107B100023E042E068E684E194E00E94153580911C
:107B200048048C31D0F5909102048090B70C90906D
:107B3000B80CA090B90CB090BA0CC090BB0CD0900F
:107B4000BC0C843128F480914A04883008F035C296
:107B500080914804883008F410C2809148048C3128
:107B600008F412C28090910C9090920CA090930C0B
:107B7000B090940C6091950C7091960C8091480493
:107B8000883008F407C2809148048C3108F409C297
:107B9000809148048C3108F40AC28091280983FF3F
:107BA00027C080915807882319F1809148048433B5
:107BB000F8F480914A048A32D8F007E028E04AE2DB
:107BC0006AE284E194E0A9D905E022E04CE262E3B4
:107BD00084E194E0A2D904E02AE041E36AE284E18E
:107BE00094E04BD94BE262E384E194E00E94D43408
:107BF00080914804853328F480914A04813308F049
:107C0000A6C00E940E89823048F0909148049433B7
:107C100028F490914A04923308F0A1C0809148045E
:107C20008F3208F05DC080914A04883208F458C051
:107C30000F9412502B013C018CE3882E912CA12C27
:107C4000B12CC301B201A50194010F94E558CA01FA
:107C5000B901A50194010F94E558CA01D62EC72E8B
:107C60004901AE014F5F5F4F5A0150E8451651E59B
:107C7000550651E06506710408F48BC0B90128E18E
:107C800030E040E050E00F94E55829013A01CF92EE
:107C9000DF92C40168E170E00F94BE589F938F9308
:107CA0005F924F928CEA96E19F938F93BF92AF922F
:107CB0000F94625E0FB6F894DEBF0FBECDBF5AE0E0
:107CC000451651046104710408F08DC098E0892FB5
:107CD000880F980F892F8195A5016FE2855AC0DD25
:107CE000809148048632A0F480914A048E3180F05D
:107CF00008E020E84EE160E084E194E00ED9809154
:107D00004804863228F480914A048F3108F06DC00F
:107D100080914804823328F480914A048B3208F021
:107D200011C180914804813408F030C280914A0426
:107D3000873308F42BC26EE380E018DD812FB3DDBA
:107D400025C286E297E1C9CE80EF96E1DFCE04E05E
:107D50002AE441E366E384E194E08FD852CFF8E46B
:107D60008F9FB0011124072E000C880B990B0F94E4
:107D70003D562AE037ED43E25CE30F94D9570F9468
:107D80000F56262F02E042E367E384E194E0C5D872
:107D900045CF84E68816910498F4CF92DF923F9302
:107DA0002F9382EA96E19F938F93BF92AF920F94A5
:107DB000625E0FB6F894DEBF0FBECDBF95E087CFF1
:107DC000CF92DF923F932F938AE996E19F938F930F
:107DD000BF92AF920F94625E0FB6F894DEBF0FBEF3
:107DE000CDBF96E074CF99E072CF60E084E194E07B
:107DF0000E94EB3428E530E040E050E065E283E0AB
:107E00003ADD65E28BE0B2DC112321F08DEF93E0E7
:107E100024DD24C080917C0D80FD17C03DEFC32E72
:107E200033E0D32EF60161916F016623B9F06F3212
:107E300034F4062E000C770B880B990B04C06FE30B
:107E400070E080E090E014DDEDCF80917B0D80FD4F
:107E5000DDCF6FEF7FEF8DE896E1E1DC29E530E0E3
:107E600040E050E065E288E206DD65E280E37EDC2A
:107E7000112321F088EF93E0F0DC26C080917C0D87
:107E8000869580FD17C028EFC22E23E0D22EF60182
:107E900061916F016623C1F06F3234F4062E000C3D
:107EA000770B880B990B04C06FE370E080E090E0E3
:107EB000DFDCEDCF80917B0D869580FDDBCF6FEF12
:107EC0007FEF8DE896E1ABDC2AE530E040E050E062
:107ED00065E28DE4D0DC65E285E548DC112321F024
:107EE00080EF93E0BADC28C080917C0D8695869562
:107EF00080FD17C090EFC92E93E0D92EF601619155
:107F00006F016623C9F06F3234F4062E000C770B34
:107F1000880B990B04C06FE370E080E090E0A8DC70
:107F2000EDCF80917B0D8695869580FDD9CF6FEF43
:107F30007FEF82E996E173DC61E084E194E00E94E6
:107F4000EB34E6CE83E008D426E030E040E050E0B9
:107F500062E383E090DC81E0FFD380916502909141
:107F600066020F940349AC0162E38CE079DC65E2C0
:107F700070E080E090E07CDCD4CE8091A80C111100
:107F80002DC08111EACD2AC080914A04853108F0C4
:107F900056C0E8CD8091840C11117EC08111F3CDC3
:107FA0007BC080914A04853108F0A7C0F1CD809153
:107FB0004A04853108F0CEC0F0CD90FD03C080E5C5
:107FC00097E102C088E697E17C010CE022E048E0FE
:107FD00068E084E194E00E941535BACDB601DD0C6D
:107FE000880B990B0F943D5620E030E040E05FE3B2
:107FF0000F94C2540F940A56CB010F940349FC010D
:1080000080818032D1F48181803211F491E001C00D
:1080100092E043E050E0491B51094E0F5F1F892F4A
:10802000880F980F892F819567E0815F19DC69E0DF
:1080300070E080E090E01CDC90CD93E0EACF20E09F
:1080400030E040E05FE3C501B4010F94C2540F94E7
:108050000A56CB010F940349FC0180818032D1F490
:108060008181803211F491E001C092E043E050E060
:10807000491B51094E0F5F1F892F880F980F892FB9
:1080800081956CE1815FECDB69E070E080E090E07D
:10809000EFDB68CD93E0EACF072E000C880B990B3D
:1080A0000F943D5620E030E040E05FE30F94C2546F
:1080B0000F940A56CB010F940349FC018081803252
:1080C000D1F48181803211F491E001C092E043E06B
:1080D00050E0491B51094E0F5F1F892F880F980FE1
:1080E000892F819567E0865ABBDB69E070E080E00C
:1080F00090E0BEDB48CD93E0EACF20E030E040E006
:108100005FE3C501B4010F94C2540F940A56CB012A
:108110000F940349FC0180818032D1F48181803247
:1081200011F491E001C092E043E050E0491B510995
:108130004E0F5F1F892F880F980F892F81956CE153
:10814000865A8EDB69E070E080E090E091DB20CD24
:1081500093E0EACF8091B20C882309F41ECD24E687
:10816000829FC001112481589F4F6FEF70E00F94E0
:10817000D258CB010F940349AC016CE187E670DB68
:1081800065E270E080E090E073DB07CD2D960FB6DE
:10819000F894DEBF0FBECDBFDF91CF911F910F913D
:1081A000FF90EF90DF90CF90BF90AF909F908F9017
:1081B0007F906F905F904F9008950F931F93CF9390
:1081C000DF93CDB7DEB728970FB6F894DEBF0FBEAA
:1081D000CDBF8A0123E0660F771F2A95E1F7680F6C
:1081E000791F48E050E0CE0101960F94965D2981F9
:1081F0003A81F801808191812817390790F0821720
:10820000930760F09C818281981758F081E090E09C
:108210003B812381231738F080E005C081E090E0A6
:1082200002C08FEF9FEF28960FB6F894DEBF0FBE07
:10823000CDBFDF91CF911F910F910895EF92FF92E3
:108240000F931F93CF93DF93EC018B017A018A8503
:108250009B858617970729F088819981EED81B871F
:108260000A8788859985019681F00E811F81B70163
:1082700088819981DFD8080F111D8885998580171D
:10828000910718F481E090E011C06E818A81680F37
:1082900097014C81888199810E942E392E813F81DE
:1082A000280F311D3F832E8380E090E0DF91CF9136
:1082B0001F910F91FF90EF9008954F925F926F92F0
:1082C0007F928F929F92AF92BF92CF92DF92EF9266
:1082D000FF920F931F93CF93DF93CDB7DEB72D9708
:1082E0000FB6F894DEBF0FBECDBF6C012A013B0173
:1082F000490158011B861C86CE0101967C0188E04D
:10830000F70111928A95E9F7DB01CA0127E0B695DA
:10831000A795979587952A95D1F79A838983F42F06
:10832000FF77FD878F2F80588B838C831A86198661
:108330004F3F51056105710509F018F460E070E0E8
:1083400026C060910504709106048E01075F1F4FDF
:1083500097014DED50E480910304909104040E9434
:10836000F17F97FDEBCF69857A8583E0660F771FF4
:108370008A95E1F78091030490910404680F791FB6
:1083800048E050E0C7010F94965D6F8178856115D4
:10839000710519F44B86B60106C0C616D70619F04A
:1083A0008D8580688B87AE01455F5F4FC401F50105
:1083B00019952D960FB6F894DEBF0FBECDBFDF9195
:1083C000CF911F910F91FF90EF90DF90CF90BF90D2
:1083D000AF909F908F907F906F905F904F90089597
:1083E0006F927F928F929F92AF92BF92CF92DF92C5
:1083F000EF92FF920F931F93CF93DF9300D01F92C2
:10840000CDB7DEB76C017B013A01590148011982F1
:108410001A821B821C82AE014F5F5F4FB301C701FE
:108420000E9451807C0149815A816B817C81411578
:1084300051056105710529F084019501C6013DDFF3
:10844000E6CF0F900F900F900F90DF91CF911F917B
:108450000F91FF90EF90DF90CF90BF90AF909F90E3
:108460008F907F906F90089521E020930704E3E0C0
:10847000F4E0918380837383628380E090E00895C9
:108480007F92AF92BF92CF92DF92EF92FF920F93C3
:108490001F93CF93DF93CDB7DEB72C970FB6F89429
:1084A000DEBF0FBECDBF6C01762EF72F842FE52FD8
:1084B000B901A801D6011496AD90BC901597909182
:1084C000070491110AC020EC37E1482F672DC6013F
:1084D0000E94653980E090E019C0DA82C9827B820F
:1084E000FC838D83EE8318861F82FA86E9861C86BC
:1084F0001B860EE111E49E012F5F3F4FC501DDDEBB
:10850000B501C6010E941D3A8F8198852C960FB641
:10851000F894DEBF0FBECDBFDF91CF911F910F91B9
:10852000FF90EF90DF90CF90BF90AF907F90089535
:10853000CF92DF92EF92FF920F931F93CF93DF932F
:10854000CDB7DEB72C970FB6F894DEBF0FBECDBF08
:108550007C01C901F701C480D58020910704211155
:1085600008C020EA37E1C7010E94653980E090E049
:108570001CC0FA82E9826B837C834D835E831886FC
:108580001F821A8709871C861B860EE111E49E0153
:108590002F5F3F4F4BEE5FE7BC01C60121DFB60105
:1085A000C7010E941D3A8F8198852C960FB6F894CA
:1085B000DEBF0FBECDBFDF91CF911F910F91FF9016
:1085C000EF90DF90CF900895CF92DF92EF92FF92DD
:1085D0000F931F93CF93DF93CDB7DEB72C970FB6D2
:1085E000F894DEBF0FBECDBF7C01C901F701C48086
:1085F000D58020910704211108C020E837E1C70188
:108600000E94653980E090E01CC0FA82E9826B83A9
:108610007C834D835E8318861F821A8709871C8698
:108620001B860EE111E49E012F5F3F4F4EEE5FE788
:10863000BC01C601D5DEB601C7010E941D3A8F817B
:1086400098852C960FB6F894DEBF0FBECDBFDF9194
:10865000CF911F910F91FF90EF90DF90CF900895F1
:10866000CF93DF93EC01262F4CAD6BAD04960E94A7
:1086700010392BAD082E000C990B820F911D8BAF7A
:1086800081E090E0DF91CF9108950F939CE0899F66
:10869000802D112421E0280F20930F04845F809304
:1086A0000E0490E002964091480450E0841795072C
:1086B00014F480E033C0822F90E020914A0430E02F
:1086C00082179307B4F76623A9F061E084E194E090
:1086D0000E94EB3440910F044E5F0BE020E860E015
:1086E00084E194E00E948D3760E084E194E00E9490
:1086F000EB3405C061E084E194E00E94EB346091CA
:108700000E04809148046817A0F290910F048091A4
:108710004A04891770F280E029D881E00F9108950A
:10872000CF93DF93FC0185ADEF012496811105C045
:1087300081E085AFCE010E948B34CE01DF91CF91D5
:108740000C94C234CF93DF93EA0110D86FEF7FEF20
:10875000CE01DF91CF9163C8482F50E020910D04E6
:10876000022E000C330B4217530781F080930D0447
:10877000813031F46BE77EE184E194E00C941D3AA2
:1087800069EC78E184E194E00C941D3A089581E06D
:10879000089580E194E0C4DF80E00E94C4A284E1F7
:1087A00094E00E94C6348111F7CF64EC79E080E058
:1087B00090E00C941CA3EF92FF920F9380914D04D4
:1087C000811107C081E080934D0484E194E00E9410
:1087D0008B3484E194E00E94C23486EFE82E8DE170
:1087E000F82E03E127E047E064E284E194E00E9490
:1087F000153583E0B1DF40E158E16BE285E2A2DFAD
:108800004CEF57E167E387E09DDF84E194E00E944D
:10881000C6348111E2CF0F91FF90EF90089581E06F
:10882000CADF64EC79E080E090E00C941CA3B1DF37
:10883000F6CF60E070E08BE79EE116CE1F93CF93FA
:10884000DF93C0911504C695C69580E194E068DF7A
:10885000DC2FDD0F1D2F1C0F83E07EDF6C2F80E0EF
:108860000E94B63B8EE496E00E942D3C4DEE57E10F
:108870006D2F80E067DF40EE57E1612F80E062DF1F
:1088800084E194E00E94C6348111E6CFDF91CF915C
:108890001F9108950895CF93E62F6CE0869F602D79
:1088A000112481E0860F80930F04645F60930E04AF
:1088B000462F50E04E5F5F4F2091480430E0421752
:1088C00053070CF44CC090E020914A0430E082172A
:1088D00093070CF044C0CE2F8EE30E94B63B65E4B4
:1088E00070E080E090E00E94383C61E36C0F062E5F
:1088F000000C770B880B990B0E94383C60E270E00B
:1089000080E090E00E94383C6091B70C7091B80C08
:108910008091B90C9091BA0C0F940A56CB010F9428
:1089200003490E942D3C6FE270E080E090E00E94DD
:10893000383C0E94DF83811109C085E0C89FF001A7
:108940001124EC55F34F8481811109C08091BB0C37
:108950009091BC0C0F940349CF910C942D3CCF9176
:108960000895CF92DF92EF92FF920F931F93CF93D0
:10897000DF931F921F92CDB7DEB77B01622F498331
:1089800084DE4981882309F444C0442311F1011590
:108990001105F9F4C7010E94C18125E130E0281BCF
:1089A000310937FF02C02F5F3F4F3595279530E8DB
:1089B0002158822F830F87FD0DC060E270E080E0B8
:1089C00090E02A8339830E94383C398131502A81D2
:1089D000F0CF30E8C32ED12CB601C7010E940F3C66
:1089E0007601E81AF90A0115110511F41E2D07C0C8
:1089F000FF24B701C8010E94F13B1E2D181B173040
:108A000040F060E270E080E090E00E94383C181B8B
:108A1000F6CF0F900F90DF91CF911F910F91FF90A4
:108A2000EF90DF90CF9008950F93CF93DF93982F1F
:108A3000862FEA01692F29DE882331F162E770E091
:108A4000CE010E940F3CC2E7C81BC73040F060E275
:108A500070E080E090E00E94383CC81BF6CF609147
:108A60000E048AE70E94B63B602F000F770B880B3D
:108A7000990B0E94383C60E270E080E090E0DF916A
:108A8000CF910F910C94383CDF91CF910F910895C5
:108A9000CF92DF92EF92FF920F931F93CF93DF93CA
:108AA000982F862F6A017901692FEFDD882309F459
:108AB0004BC0C701002321F00E94C181182F03C0C1
:108AC0000E94A081182FC3E1D0E0C11BD1098C2FD7
:108AD000880FC80FCC0FD0E0BE01C6010E940F3C2A
:108AE000C81B6AE370E080E090E00E94383CC73029
:108AF00040F060E270E080E090E00E94383CC81BEB
:108B0000F6CF8AEF189F802D112460910E048058B3
:108B10000E94B63B002369F06FEF7FEFC701DF9142
:108B2000CF911F910F91FF90EF90DF90CF900C9419
:108B30000F3CC701DF91CF911F910F91FF90EF90F4
:108B4000DF90CF900C942D3CDF91CF911F910F912E
:108B5000FF90EF90DF90CF900895BF92CF92DF9279
:108B6000EF92FF920F931F93CF93DF936C017B01E2
:108B70000E94C181C82FC7010E94A08103E110E0BB
:108B8000081B11098C2F90E0BB24B3940817190718
:108B90001CF0B12CC5E201C0CFE12C2F30E0A901BF
:108BA0004E5F5F4F8091480490E04817590744F0AA
:108BB0002950310960914A0470E062177307BCF5CF
:108BC000D0E0E114F104C9F16AE370E080E090E0E4
:108BD0000E94383CBB2081F0C45F80914804C817D4
:108BE00060F12C2F30E02950310980914A0490E047
:108BF000821793071CF421C0DD23F9F0802F880F22
:108C0000800F6C2F880F0E94B63B60E270E080E01E
:108C100090E00E94383CC701DF91CF911F910F91E6
:108C2000FF90EF90DF90CF90BF900C942D3CA60169
:108C30006C2F80E087DDD1E0C4CFDF91CF911F9111
:108C40000F91FF90EF90DF90CF90BF900895CF925B
:108C5000DF92EF92FF920F931F93CF93DF931F92B8
:108C6000CDB7DEB7182F7A01D22ECA0169830E94D0
:108C7000C181082F812F880F810FC82ECC0C1CE0DA
:108C80006981169F100D1124DD20C1F061E084E19F
:108C900094E00E94EB34202F220F200F220F2E5F32
:108CA0000BE047EF410F6FEF6C0D84E194E00E9401
:108CB0008D3760E084E194E00E94EB34A701612FDE
:108CC0008C2D40DDDD2071F061E084E194E00F90B7
:108CD000DF91CF911F910F91FF90EF90DF90CF9098
:108CE0000C94EB340F90DF91CF911F910F91FF9077
:108CF000EF90DF90CF900895AF92BF92DF92EF9206
:108D0000FF920F931F93CF93DF93EC015B01D42E5F
:108D1000C901B801A7010E94708391E02D2D292778
:108D2000A50164E081E093DFCE010E94C1812D2D79
:108D3000AE0164E094E1981B892FDF91CF911F91E0
:108D40000F91FF90EF90DF90BF90AF9080CFEF92A8
:108D5000FF920F93CF93DF93D82FC62F7901682FFF
:108D60008C2F93DC8823F1F0002331F062E070E077
:108D700080E090E00E94383C2D2F4C2F64E1C70129
:108D80000E944C8268E770E00E94F13BC8E7C81B74
:108D9000C73040F060E270E080E090E00E94383C34
:108DA000C81BF6CFDF91CF910F91FF90EF90089500
:108DB0008F929F92AF92BF92CF92DF92EF92FF92EB
:108DC0000F936B017C018090090490900A04A0909D
:108DD0000B04B0900C04A50194010F949B558823BB
:108DE00001F120E030E0A901C701B6010F949B55C5
:108DF000882351F0A5019401C701B6010F949B553A
:108E000087FD04C081E003C080E001C08FEF809344
:108E10000804C0920904D0920A04E0920B04F09274
:108E20000C0480914804813128F480914A048330F5
:108E300008F048C080914804853128F480914A04A4
:108E4000843108F04FC0809148048F3308F057C038
:108E500080914A048F3208F452C08091080440E3A4
:108E6000481B8FE4E82E88E1F82E0DE022E06AE549
:108E700084E194E00E9415358091080441E3481B89
:108E800095E3E92E98E1F92E22E065E084E194E093
:108E90000E94153529E6E22E28E1F22E00E123E0BA
:108EA0004FE262E184E194E00E94153539E9E32E56
:108EB00038E1F32E23E04FE267E684E194E00E947C
:108EC00015351DC08091080444E0481B5AE1E52E89
:108ED00058E1F52E0CE022E062E484E194E00E9487
:108EE0001535A8CF42E3E42E48E1F42E01E023E05B
:108EF00044E16CE384E194E00E941535A4CF0F9126
:108F0000FF90EF90DF90CF90BF90AF909F908F90A9
:108F10000895CF92EF920F93CF93DF93C0E1D4E007
:108F20001B821A8284E693E099838883CC24CA94B6
:108F3000EE24EA9402E522E143E164E172E0CE012D
:108F40000E94973B80E793E099838883DF91CF91DC
:108F50000F91EF90CF9008955A9887FD52C05B987B
:108F600000000000000000005A9A5A98282F220F93
:108F700086FD53C05B9800000000000000005A9A74
:108F80005A98922F990F26FD46C05B98000000006A
:108F9000000000005A9A5A98892F880F96FD39C010
:108FA0005B9800000000000000005A9A5A98982F21
:108FB000990F86FD2CC05B980000000000000000A7
:108FC0005A9A5A98892F880F96FD1FC05B98000007
:108FD0000000000000005A9A5A98982F990F86FDB9
:108FE00012C05B9800000000000000005A9A5A98D6
:108FF00096FD15C05B9800000000000000005A9A22
:1090000008955B9AADCF5B9AEDCF5B9AE0CF5B9A08
:10901000D3CF5B9AC6CF5B9AB9CF5B9AACCF5B9A42
:10902000EACF2F923F925F927F929F92AF92BF9230
:10903000CF92DF92EF92FF920F931F93CF93DF9324
:109040007C011B01942E69018AE0481709F47BC05A
:10905000A5E14A134EC0DB011296ED91FC911397E6
:109060001281C681D7815D9A88E28A950000E9F76E
:1090700000EE010F80E1582E510E98E2792E88EF14
:109080006BDF872D8A950000E9F7103208F046C0A3
:10909000812F8077806860DF812F8295807F5CDF01
:1090A000872D8A950000E9F780E856DF80E054DFDD
:1090B000872D8A950000E9F78AEF4EDF872D8A9584
:1090C0000000E9F75E01B0E1AB0EB11C8881807F42
:1090D00043DF89918295807F3FDFCA15DB05B1F7B9
:1090E000872D8A950000E9F71F5F0F5F1511C7CF25
:1090F0005D989601492DB101C701DF91CF911F9174
:109100000F91FF90EF90DF90CF90BF90AF909F9026
:109110007F905F903F902F900C944F36802F8077F8
:1091200080681ADF802F8295807F16DF872D8A95D1
:109130000000E9F780E810DF80E80EDF872D8A95D0
:109140000000E9F7B9CF559A5D98539A5B98529A07
:109150005A9A5D9AC8E28C2F8A950000E9F788E751
:1091600090E00E946C3588EFF7DE8C2F8A95000026
:10917000E9F780E2F1DE80E0EFDE8C2F8A950000D7
:10918000E9F780E0E9DE80E8E7DE8C2F8A950000D1
:10919000E9F780E0E1DE80E1DFDE8C2F8A950000D8
:1091A000E9F78FE090E00E946C3580E2D5DE80E444
:1091B000D3DE8C2F8A950000E9F780E2CDDE80E6D1
:1091C000CBDECA950000E9F710E0D8E208E2812F73
:1091D00080778068C1DE812F8295807FBDDE8D2FF4
:1091E0008A950000E9F780E8B7DE80E0B5DE8D2FD4
:1091F0008A950000E9F78AEFAFDE8D2F8A9500008F
:10920000E9F7C0E280E0A8DE80E0A6DE9D2F9A9517
:109210000000E9F7C150B1F788EF9EDE802F8A95F4
:109220000000E9F71F5F103209F0D1CF80E094DE33
:1092300080EC92DE88E28A950000E9F75D9859CFCC
:10924000CF93DF931F921F92CDB7DEB789839A83A6
:109250000E94B77C20E040E060E070E089819A8164
:109260000F900F90DF91CF910C946A7D0F93CF9365
:10927000DF9361E081E00E94837ED0911C06C0E014
:10928000D11117C080911B06811104C00E949682E3
:10929000811165C080912202882309F457C081E0C2
:1092A00090911B06911180E004E024E04FE857E222
:1092B0004BC0D130C1F480911B06813021F40E9453
:1092C0009682811155C080912202882309F43EC004
:1092D00081E090911B06913009F080E003E02EE3DD
:1092E00046E857E231C0D230B9F480911B06823093
:1092F00021F40E949682811144C080912202882329
:1093000029F181E090911B06923009F080E003E0A2
:109310002EE34DE757E218C0D330C1F480911B060D
:10932000833021F40E949682811134C08091220200
:10933000882361F081E090911B06933009F080E072
:1093400003E02EE347E757E26C2F6EDBCF5FDF5F72
:10935000C53009F095CF84E080931A0622C081E0E1
:109360000E949D7D8091E805882309F493CF19C060
:109370008AE892E765DF8091E805882309F4A3CFA6
:1093800010C08CEA97E75CDF8091E805882309F438
:10939000B4CF07C084EC9BE753DF8091E8058823B6
:1093A00029F2DF91CF910F910895CF93DF93EC01D4
:1093B000CB01BA010F943D5623E333E343E250E47B
:1093C0000F94D9570F940F566883DF91CF9108956A
:1093D000CF93DF93EC01CB01BA010F943D562FE6FA
:1093E00032E143E85AE30F94D957688379838A833B
:1093F0009B83DF91CF91089565ED79E488E09AE44D
:109400000C94C17D68EE79E48BE29AE40C94C17D02
:109410000F943D5623E333E343E250E40F94D957CE
:109420000F940F56862F0D945848CF93DF9300D09A
:109430001F92CDB7DEB769837A838B839C8360E20A
:10944000CE0101960F947C4B0F900F900F900F90D0
:10945000DF91CF9108950F943D562FE632E143E816
:109460005AE30F94D957E1CF2F923F924F925F92D8
:109470006F927F928F929F92AF92BF92CF92DF9224
:10948000EF92FF920F931F93CF93DF93CDB7DEB789
:1094900029970FB6F894DEBF0FBECDBF1C017987A8
:1094A0006887CA01B901E982FA820B831C83DE82D4
:1094B000CD82AF8220E030E04AE754E40F94D957E0
:1094C0006B017C0120E030E040E057EC0F949E57A8
:1094D00018162CF0C12CD12CE12C27ECF22EC70150
:1094E000B6010F940A562B013C0120E030E04AE718
:1094F00054E469817A818B819C810F94D9574B0107
:109500005C0120E03EEF4FEF56E40F949B5587FD42
:1095100007C0812C9EEF992EAA24AA9496E4B92E16
:1095200020E030E04AE754E4E885F9856081718104
:10953000828193810F94D9576B017C01C301B201E1
:109540000F943D569B01AC01C701B6010F94C15465
:109550000F940F5669837A838B839C83C501B40172
:109560000F940A567B018C01E418F50806091709C7
:10957000FF81FF938D809E8082E0A82E8AE4B82E22
:10958000C980DA80A301920168857985C1010E94B2
:10959000DE7C0F9029960FB6F894DEBF0FBECDBFCC
:1095A000DF91CF911F910F91FF90EF90DF90CF90BF
:1095B000BF90AF909F908F907F906F905F904F90F3
:1095C0003F902F9008958F929F92AF92BF92CF922B
:1095D000DF92EF92FF920F931F93CF93DF9361E09F
:1095E00081E00E94837ED0911C06C0E0D11119C099
:1095F00080911B06811104C00E9496828111C4C013
:1096000080912202882309F4B6C081E090911B0664
:10961000911180E004E024E04AEC57E26C2F04DA78
:10962000AAC0D130E1F480911B06813021F40E9460
:1096300096828111B2C080912202882309F49BC0D6
:1096400011E080911B06813009F010E080912C0C14
:109650000F94584800E09C0144EB57E289C0D23097
:1096600009F580911B06823021F40E9496828111B7
:10967000C3C080912202882309F47DC011E080914B
:109680001B06823009F010E060912D0C70912E0CB9
:1096900080912F0C9091300CC8DE00E09C0140EBD3
:1096A00057E266C0D33009F580911B06833021F460
:1096B0000E9496828111B9C080912202882309F408
:1096C0005AC011E080911B06833009F010E06091D0
:1096D000310C7091320C8091330C9091340CA5DEDA
:1096E00000E09C014CEA57E243C0D43001F5809180
:1096F0001B06843021F40E9496828111AFC08091B4
:1097000022028823C1F111E080911B06843009F008
:1097100010E06091350C7091360C8091370C90916F
:10972000380C83DE00E09C0148EA57E221C0D530C6
:1097300011F580911B06853021F40E9496828111DB
:10974000A6C0809122028823B1F011E080911B060F
:10975000853009F010E06091280270912902809113
:109760002A0290912B0261DE00E09C0144E957E25D
:109770006C2F812F8DD9CF5FDF5FC53009F036CFD9
:1097800086E080931A069BC081E00E949D7D8091B7
:10979000E805882309F434CF92C081E00E948B82CF
:1097A00060912C0C70E080E090E00F943B5629EC27
:1097B00038EC48EC5EE30F94D9570F940F561F9284
:1097C000812C912C4CEFA42E49E4B42E6B0114E6AD
:1097D000E12EF12C00E010E020E030E0A9016CE285
:1097E0007CE08FEB97E20E94DE7C0F908091E80591
:1097F000882309F420CF63C081E00E948B82A12CD2
:10980000C12CD12C16E6E12EFE2C0EE111E420E055
:1098100030E0A9016DE27CE082EB97E225DE8091E9
:10982000E805882309F425CF4AC081E00E948B8295
:10983000A12CC12CD12C16E6E12EFE2C0EE111E458
:1098400020E030E0A90161E37CE08EEA97E20CDEE3
:109850008091E805882309F42FCF31C081E00E9470
:109860008B82A12CC12CD12C16E6E12EFE2C0EE110
:1098700011E420E030E0A90165E37CE08AEA97E2A8
:10988000F3DD8091E805882309F439CF18C081E021
:109890000E948B82A12CC12CD12C16E6E12EFE2C2D
:1098A0000EE111E420E030E0A90168E272E08EE907
:1098B00097E2DADD8091E805882309F442CFDF9151
:1098C000CF911F910F91FF90EF90DF90CF90BF90BD
:1098D000AF909F908F900895CF93DF93EC01CB01D1
:1098E000BA010F943D5620E030E048EC52E40F946A
:1098F000D9570F940F56688379838A839B83DF91AE
:10990000CF910895CF93DF93EC01CB01BA010F946F
:109910003D562AE037ED43E25CE30F94D957688364
:1099200079838A839B83DF91CF910895CF93DF93CF
:10993000EC01CB01BA010F943D56688379838A8389
:109940009B83DF91CF910895CF93DF93EC01CB01FF
:10995000BA010F943D5620E030E048EC51E40F94FA
:10996000D957688379838A839B83DF91CF91089548
:10997000CF93DF93EC01CB01BA010F943D5668837E
:1099800079838A839B83DF91CF910895CF93DF936F
:10999000EC01CB01BA010F943D5620E030E048ECD9
:1099A00051E40F94D9570F940F56688379838A83B3
:1099B0009B83DF91CF910895CF93DF93EC01CB018F
:1099C000BA010F943D562AE037ED43E25CE30F9471
:1099D000D957688379838A839B83DF91CF910895D8
:1099E000CF93DF93EC01CB01BA010F943D562DECE0
:1099F0003CEC4CEC5DE30F94D957688379838A8300
:109A00009B83DF91CF9108956CE67CE482E09EE435
:109A10000C94C17D62E87CE489E89DE40C94C17DEE
:109A200066E97CE486EE9DE40C94C17D68EB7CE401
:109A300088E39DE40C94C17D64EA7CE486EA9DE4BD
:109A40000C94C17D66EC7CE484E29EE40C94C17DC0
:109A50006CED7CE48FE49DE40C94C17D60EF7CE4CC
:109A60008CE69DE40C94C17D0D941E050D94650556
:109A7000CF93DF9300D01F92CDB7DEB70F943D5642
:109A800069837A838B839C83CE0101960F94C54CA6
:109A90000F900F900F900F90DF91CF910895CF937B
:109AA000DF9300D01F92CDB7DEB70F943D562AE06A
:109AB00037ED43E25CE30F94D95769837A838B8354
:109AC0009C83CE0101960F94FA4C0F900F900F904B
:109AD0000F90DF91CF910895CF93DF9300D01F9225
:109AE000CDB7DEB70F943D562DEC3CEC4CEC5DE36E
:109AF0000F94D95769837A838B839C83CE01019617
:109B00000F949A4D0F900F900F900F90DF91CF917F
:109B10000895CF93DF9300D01F92CDB7DEB70F9497
:109B20003D562AE037ED43E25CE30F94D957698351
:109B30007A838B839C83CE0101960F943E4A0F90CB
:109B40000F900F900F90DF91CF910895CF93DF93F7
:109B500000D01F92CDB7DEB70F943D5620E030E025
:109B600048EC51E40F94D95769837A838B839C83A3
:109B7000CE0101960F94C54C0F900F900F900F904F
:109B8000DF91CF910895CF92DF92EF92FF926B0118
:109B90007C0120E030E0A9010F949B5587FD05C0B2
:109BA00020E030E040E05FE304C020E030E040E04F
:109BB0005FEBC701B6010F94C2540F940A56CB0154
:109BC000FF90EF90DF90CF900D9403490F943D5696
:109BD000DACFCF93DF9300D01F92CDB7DEB70F94CB
:109BE0000F560F943B5669837A838B839C83CE01F7
:109BF00001960F94C54C0F900F900F900F90DF912E
:109C0000CF9108950F943D5620E030E048EC52E4A7
:109C10000F94D957DECFCF93DF9300D01F92CDB7EB
:109C2000DEB70F940F560F943B5669837A838B836C
:109C30009C83CE0101960F94C54C0F900F900F900E
:109C40000F90DF91CF9108950F943D5620E030E0C2
:109C500048EC51E40F94D957DECF81E00C949D7D00
:109C60000F931F93CF93DF9361E081E00E94837E87
:109C7000C0911C06D0E0C1111AC080911B06811151
:109C800004C00E949682811104C18091220288231F
:109C900009F461C081E090911B06911180E004E01D
:109CA00024E040E258E26D2F0E94144554C0C130B8
:109CB000D9F480911B06813021F40E949682811193
:109CC000EFC080912202882309F445C081E0909181
:109CD0001B06913009F080E003E02EE347E158E2F3
:109CE0006D2F0E94144537C0C230D1F480911B06FD
:109CF000823021F40E9496828111DBC08091220281
:109D0000882349F181E090911B06923009F080E0B0
:109D100003E02EE34AE058E26D2F0E9414451BC079
:109D2000C330C9F480911B06833021F40E949682CF
:109D30008111C8C080912202882369F081E090914E
:109D40001B06933009F080E003E02EE345E058E283
:109D50006D2F0E9414450E94537D81111DC0C43097
:109D6000E9F480911B06843021F40E9496828111CF
:109D7000B2C080912202882309F4B6C081E090919C
:109D80001B06943009F080E003E02EE34CEF57E22D
:109D90006D2F0E941445A8C014E001C015E0C11346
:109DA0001BC080911B068C1304C00E9496828111F7
:109DB0009DC080912202882371F081E090911B0662
:109DC0009C1380E003E02EE343EF57E26D2F0E94E7
:109DD00014451C2F01C01C2F81E0810FC81318C02F
:109DE00080911B068C1304C00E949682811187C04B
:109DF00080912202882361F081E090911B069C13E0
:109E000080E003E02EE344EE57E26D2F0E941445FC
:109E100082E0810FC81318C080911B068C1304C008
:109E20000E949682811174C080912202882361F081
:109E300081E090911B069C1380E003E02EE348ED47
:109E400057E26D2F0E94144583E0810FC81318C09C
:109E500080911B068C1304C00E949682811161C000
:109E600080912202882361F081E090911B069C136F
:109E700080E003E02EE34FEC57E26D2F0E94144583
:109E8000DF5FCF5FD53009F0F6CE1C5F10931A0666
:109E900050C0E3DE8091E805882309F4F6CE49C07E
:109EA00084E797E5CDD98091E805882309F409CFA7
:109EB00040C08FE591E5C4D98091E805882309F475
:109EC0001DCF37C082E499E5BBD98091E80588238E
:109ED00009F430CF2EC086E79BE5B2D98091E80522
:109EE000882309F446CF25C015E076CF83EE9AE4A7
:109EF000A7D98091E805882309F45BCF1AC083E5D0
:109F000090E59ED98091E805882309F471CF11C0AE
:109F100082E196E595D98091E805882309F484CFFC
:109F200008C080EE94E58CD98091E805882309F477
:109F300097CFDF91CF911F910F9108952F923F926C
:109F40004F925F926F927F928F929F92AF92BF9249
:109F5000CF92DF92EF92FF920F931F93CF93DF93F5
:109F6000CDB7DEB729970FB6F894DEBF0FBECDBFD1
:109F70001C0179876887E982FA820B831C83DE8261
:109F8000CD82AF82CA01B9010F943B562AE037ED6A
:109F900043E25CE30F94D9576B017C0120E030E091
:109FA00040E057EC0F949E5718162CF0C12CD12C82
:109FB000E12C27ECF22EC701B6010F940A562B01B3
:109FC0003C0169817A818B819C810F943B562AE008
:109FD00037ED43E25CE30F94D9574B015C0120E07D
:109FE0003EEF4FEF56E40F949B5587FD07C0812C41
:109FF0009EEF992EAA24AA9496E4B92EE885F985B5
:10A0000060817181828193810F943B562AE037ED04
:10A0100043E25CE30F94D9576B017C01C301B201A9
:10A020000F943D569B01AC01C701B6010F94C1547A
:10A030000F940F5669837A838B839C83C501B40187
:10A040000F940A567B018C01E418F50806091709DC
:10A05000FF81FF938D809E8084E0A82E8DE4B82E32
:10A06000C980DA80A301920168857985C1010E94C7
:10A07000DE7C0F9029960FB6F894DEBF0FBECDBFE1
:10A08000DF91CF911F910F91FF90EF90DF90CF90D4
:10A09000BF90AF909F908F907F906F905F904F9008
:10A0A0003F902F900895AF92CF92DF92EF92FF9260
:10A0B0000F931F93CF93DF9361E081E00E94837E33
:10A0C000D0911C06C0E0D1111AC080911B068111ED
:10A0D00004C00E949682811194C08091220288233C
:10A0E00009F486C081E090911B06911180E004E0A4
:10A0F00024E045E75AE26C2F0E94144579C0D13024
:10A1000039F580911B06813021F40E9496828111DD
:10A110007FC080912202882309F46AC011E08091F7
:10A120001B06813009F010E06091460D7091470DDB
:10A130008091480D9091490D0F943B564ADD00E007
:10A140009C014FE65AE26C2F812F0E94484550C077
:10A15000D23039F580911B06823021F40E9496821C
:10A16000811170C080912202882309F441C011E05E
:10A1700080911B06823009F010E060914A0D7091C9
:10A180004B0D80914C0D90914D0D0F943B5621DD60
:10A1900000E09C014BE65AE26C2F812F0E9448455B
:10A1A00027C0D33029F580911B06833021F40E940B
:10A1B0009682811161C0809122028823C9F011E04A
:10A1C00080911B06833009F010E060914E0D709174
:10A1D0004F0D8091500D9091510D0F943B56F9DC2D
:10A1E00000E09C0147E65AE26C2F812F0E9448450F
:10A1F000CF5FDF5FC53009F066CF84E080931A0639
:10A2000054C02BDD8091E805882309F466CF4DC04A
:10A21000A12C4BE2C42E43EDD42E10EDE12E17E01D
:10A22000F12E00E010E024E630E040E050E066E48B
:10A230007DE082E79AE282DE8091E805882309F4D6
:10A2400068CF33C0A12C2BE2C22E23EDD22E10ED0D
:10A25000E12E17E0F12E00E010E024E630E040E0CF
:10A2600050E06AE47DE08DE69AE268DE8091E805E0
:10A27000882309F477CF19C0A12C8BE2C82E83ED77
:10A28000D82E10EDE12E17E0F12E00E010E024E6CC
:10A2900030E040E050E06EE47DE089E69AE24EDE98
:10A2A0008091E805882309F486CFDF91CF911F9133
:10A2B0000F91FF90EF90DF90CF90AF9008956F9245
:10A2C0007F928F929F92AF92BF92CF92DF92EF9246
:10A2D000FF920F931F93CF93DF9300D01F92CDB7C0
:10A2E000DEB761E081E00E94837E60901C06712CE5
:10A2F00061101AC080911B06811104C00E949682D1
:10A3000081114EC180912202882309F440C181E06D
:10A3100090911B06911180E004E024E04CE459E2A6
:10A32000672D0E94144533C181E068122CC08091D2
:10A330001B06813021F40E949682811138C18091E0
:10A340002202882309F423C111E080911B06813089
:10A3500009F010E08091600E9091610EA091620E64
:10A36000B091630E89839A83AB83BC83CE0101963F
:10A370000F94C54C00E09C0140E459E2672D812F09
:10A380000E94484504C182E068122CC080911B06DF
:10A39000823021F40E949682811141C18091220273
:10A3A000882309F4F4C011E080911B06823009F083
:10A3B00010E08091640E9091650EA091660EB091B0
:10A3C000670E89839A83AB83BC83CE0101960F9479
:10A3D000C54C00E09C014CE259E2672D812F0E94A0
:10A3E0004845D5C083E068122CC080911B0683309D
:10A3F00021F40E949682811144C180912202882317
:10A4000009F4C5C011E080911B06833009F010E00B
:10A410008091680E9091690EA0916A0EB0916B0EBA
:10A4200089839A83AB83BC83CE0101960F94C54C7C
:10A4300000E09C014AE159E2672D812F0E944845C6
:10A44000A6C084E0681227C080911B06843021F4E6
:10A450000E94968281114DC180912202882309F4C5
:10A4600096C011E080911B06843009F010E06091E5
:10A470002C0E70912D0E80912E0E90912F0E0F9418
:10A480003B56C9DB00E09C014CE059E2672D812F6F
:10A490000E9448457CC085E0681227C080911B0659
:10A4A000853021F40E94968281115FC18091220241
:10A4B000882309F46CC011E080911B06853009F0F7
:10A4C00010E06091300E7091310E8091320E9091BB
:10A4D000330E0F943B569FDB00E09C014EEF58E299
:10A4E000672D812F0E94484552C086E0681227C020
:10A4F00080911B06863021F40E949682811171C1E1
:10A5000080912202882309F442C011E080911B0649
:10A51000863009F010E06091340E7091350E809114
:10A52000360E9091370E0F943B5675DB00E09C0180
:10A5300040EF58E2672D812F0E94484528C087E0F0
:10A54000681225C080911B06873021F40E949682F4
:10A5500081117CC1809122028823C9F011E0809191
:10A560001B06873009F010E06091380E7091390EAB
:10A5700080913A0E90913B0E0F943B562ADB00E0FF
:10A580009C0142EE58E2672D812F0E94484573944A
:10A59000639485E07812ACCE88E080931A0672C18D
:10A5A0005CDB8091E805882309F4ACCE6BC181E0C7
:10A5B0000E948B822AE037ED43E25DE36091600EFA
:10A5C0007091610E8091620E9091630E0F94D95735
:10A5D00020E030E040E85FE30F94C1540F940F5641
:10A5E0001F92812C912C5CE1A52E5DE4B52E6B01B0
:10A5F00017E7E12E1FE0F12E00E010E021E030E04F
:10A6000040E050E060E67EE086E499E20E94DE7C75
:10A610000F908091E805882309F491CE33C181E041
:10A620000E948B8220E030E048EC52E46091640E9E
:10A630007091650E8091660E9091670E0F94C154D3
:10A640000F940F561F92812C912C36E1A32E3DE4DE
:10A65000B32E6B011BE9E12E1FE7F12E00E010E0A5
:10A6600024E630E040E050E064E67EE086E399E2F4
:10A670000E94DE7C0F908091E805882309F48ECE3D
:10A6800001C181E00E948B822AE037ED43E25DE365
:10A690006091680E7091690E80916A0E90916B0EB8
:10A6A0000F94D95720E030E040E85FE30F94C154A5
:10A6B0000F940F561F92812C912C9CE1A92E9DE4A2
:10A6C000B92E6B0117E7E12E1FE0F12E00E010E03C
:10A6D00021E030E040E050E068E67EE083E299E28D
:10A6E0000E94DE7C0F908091E805882309F485CED6
:10A6F000C9C081E00E948B8260912C0E70912D0E5A
:10A7000080912E0E90912F0E0F943B562AE037ED3C
:10A7100043E25DE30F94D95720E030E040E850E495
:10A720000F94C1540F940F561F92A4E38A2EADE4E8
:10A730009A2EB2E2AB2EBDE4BB2E6B0114E7E12EE4
:10A740001FE0F12E00E010E024E030E040E050E0B7
:10A750006CE27EE083E199E20E94DE7C0F908091C2
:10A76000E805882309F478CE8DC081E00E948B82B1
:10A770006091300E7091310E8091320E9091330EB7
:10A780000F943B562AE037ED43E25DE30F94D9572F
:10A7900020E030E040E850E40F94C1540F940F568D
:10A7A0001F9254E3852E5DE4952EE2E2AE2EEDE499
:10A7B000BE2E6B0114E7E12E1FE0F12E00E010E049
:10A7C00024E030E040E050E060E37EE085E099E2A4
:10A7D0000E94DE7C0F908091E805882309F466CE04
:10A7E00051C081E00E948B826091340E7091350ED1
:10A7F0008091360E9091370E0F943B562AE037ED3C
:10A8000043E25DE30F94D9570F940F561F9224E350
:10A81000822E2DE4922E32E2A32E3DE4B32E6B0164
:10A8200018E7E12E1FE0F12E00E010E020E030E01C
:10A83000A90164E37EE087EF98E20E94DE7C0F903E
:10A840008091E805882309F45BCE1CC081E00E945A
:10A850008B82A12C84E3C82E8DE4D82E18EBE12E38
:10A8600012E8F12E01E010E024E630E040E050E094
:10A8700068E37EE089EE98E261DB8091E805882359
:10A8800009F468CE0F900F900F900F90DF91CF9149
:10A890001F910F91FF90EF90DF90CF90BF90AF90FE
:10A8A0009F908F907F906F9008952F923F924F923C
:10A8B0005F926F927F928F929F92AF92BF92CF9250
:10A8C000DF92EF92FF920F931F93CF93DF9300D00D
:10A8D00000D0CDB7DEB71C017E836D8329013A011C
:10A8E000460120E030E040E057ECB201C3010F9494
:10A8F0009E5718162CF0412C512C612C27EC01C0CE
:10A90000272DB201862D922F0F940A562B013C0160
:10A9100020E03EEF4FEF56E4B701C8010F949B557E
:10A9200087FD06C0B12C9EEFF92E0FEF16E401C093
:10A93000BE2CC301B2010F943D569B01AC01ED81C9
:10A94000FE8160817181828193810F94C1540F9443
:10A950000F5669837A838B839C836B2D7F2DC8016F
:10A960000F940A567B018C01E418F50806091709B3
:10A97000AF9280E1A82E8DE4B82EC980DA80A301C1
:10A9800092016D817E81C1010E94DE7C0F9026962E
:10A990000FB6F894DEBF0FBECDBFDF91CF911F91F0
:10A9A0000F91FF90EF90DF90CF90BF90AF909F906E
:10A9B0008F907F906F905F904F903F902F90089571
:10A9C0006F927F928F929F92AF92BF92CF92DF92BF
:10A9D000EF92FF920F931F93CF93DF9300D01F92BC
:10A9E000CDB7DEB761E081E00E94837E60901C06F7
:10A9F000712C61101AC080911B06811104C00E9445
:10AA00009682811198C080912202882309F48AC01D
:10AA100081E090911B06911180E004E024E045E57F
:10AA20005AE2672D0E9414457DC081E068122CC057
:10AA300080911B06813021F40E949682811182C090
:10AA400080912202882309F46DC011E080911B06D9
:10AA5000813009F010E080919D0D90919E0DA091A4
:10AA60009F0DB091A00D89839A83AB83BC83CE01E7
:10AA700001960F943E4A00E09C0141E45AE2672DA2
:10AA8000812F0E9448454EC082E0681225C0809107
:10AA90001B06823021F40E949682811181C0809130
:10AAA0002202882309F43EC011E080911B06823007
:10AAB00009F010E06091F60B7091F70B8091F80BA4
:10AAC0009091F90B60D800E09C014DE25AE2672DAD
:10AAD000812F0E94484526C083E0681223C08091E0
:10AAE0001B06833021F40E949682811171C08091EF
:10AAF00022028823B9F011E080911B06833009F00F
:10AB000010E06091FA0B7091FB0B8091FC0B90911F
:10AB1000FD0B39D800E09C014DE15AE2672D812FF1
:10AB20000E9448457394639485E0781262CF84E074
:10AB300080931A0664C091D88091E805882309F4AF
:10AB400062CF5DC020E030E048EC52E460919D0DA2
:10AB500070919E0D80919F0D9091A00D0F94D957EB
:10AB60000F940F561F92812C912C2AE0A22E2DE4D7
:10AB7000B22E6B01EE24EA941FE7F12E00E010E004
:10AB800020E030E0A9016DE97DE08BE49AE20E94CB
:10AB9000DE7C0F908091E805882309F451CF2FC007
:10ABA00081E00E948B82A12CC12CD12CE12CF12CB4
:10ABB00008E413E420E030E0A90166EF7BE087E3DE
:10ABC0009AE273DE8091E805882309F468CF17C004
:10ABD00081E00E948B82A12CC12CD12CE12CF12C84
:10ABE00008E413E420E030E0A9016AEF7BE085E2AD
:10ABF0009AE25BDE8091E805882309F478CF0F9014
:10AC00000F900F900F90DF91CF911F910F91FF90B8
:10AC1000EF90DF90CF90BF90AF909F908F907F90FC
:10AC20006F9008956F927F928F929F92AF92BF9292
:10AC3000CF92DF92EF92FF920F931F93CF93DF9308
:10AC400000D01F92CDB7DEB761E081E00E94837E25
:10AC500060901C06712C61101AC080911B06811136
:10AC600004C00E9496828111BFC080912202882375
:10AC700009F4B2C081E090911B06911180E004E0DC
:10AC800024E04BE05AE2672D0E941445A5C081E004
:10AC9000681223C080911B06813021F40E949682A5
:10ACA0008111AAC080912202882309F495C0809165
:10ACB000CA0D811103C02BEF39E202C02FEF39E238
:10ACC00081E090911B06913009F080E001E042EFB5
:10ACD00059E2672D0E9448457FC082E0681226C075
:10ACE00080911B06823021F40E949682811192C0CD
:10ACF00080912202882309F46FC011E080911B0625
:10AD0000823009F010E060917F02709180028091A2
:10AD10008102909182020E94C34D00E09C0144EEAA
:10AD200059E2672D812F0E94484556C083E0681282
:10AD300026C080911B06833021F40E9496828111E7
:10AD40007EC080912202882309F446C011E08091E0
:10AD50001B06833009F010E0609183027091840239
:10AD600080918502909186020E94C34D00E09C0173
:10AD700046ED59E2672D812F0E9448452DC084E0A1
:10AD800068122AC080911B06843021F40E949682AA
:10AD900081116AC0809122028823F1F011E0809134
:10ADA0001B06843009F010E080917B0290917C02B8
:10ADB000A0917D02B0917E0289839A83AB83BC838C
:10ADC000CE0101960F943E4A00E09C0146EC59E208
:10ADD000672D812F0E9448457394639485E0781213
:10ADE0003ACF70921A066DC00E942D4E8091E805F0
:10ADF000882309F43ACF65C040E050E06AEC7DE07A
:10AE000082E09AE20E94457D8091E805882309F45A
:10AE100049CF57C0A12CC12CD12CE12CF12C01E938
:10AE200013E420E030E0A9016FE772E08BEE99E2D5
:10AE30003CDD8091E805882309F45ACF42C0A12C5B
:10AE4000C12CD12CE12CF12C01E913E420E030E0FD
:10AE5000A90163E872E08DED99E227DD8091E805B4
:10AE6000882309F46ECF2DC020E030E048EC52E496
:10AE700060917B0270917C0280917D0290917E02B4
:10AE80000F94D9570F940F561F92812C912C8AE062
:10AE9000A82E8DE4B82E6B0118EEE12E13E0F12EF2
:10AEA00000E010E020E030E0A9016BE772E08EECFA
:10AEB00099E20E94DE7C0F908091E805882309F4D6
:10AEC00069CF0F900F900F900F90DF91CF911F914E
:10AED0000F91FF90EF90DF90CF90BF90AF909F9039
:10AEE0008F907F906F900895AF92CF92DF92EF9204
:10AEF000FF920F931F93CF93DF9361E081E00E9455
:10AF0000837ED0911C06C0E0D1111AC080911B062F
:10AF1000811104C00E949682811109C18091220290
:10AF2000882309F4FBC081E090911B06911180E019
:10AF300004E024E044EB59E26C2F0E941445EEC07B
:10AF4000D13031F580911B06813021F40E94968228
:10AF50008111F5C080912202882309F4DFC011E03D
:10AF600080911B06813009F010E06091500E7091C5
:10AF7000510E8091520E9091530E0E94C34D00E0ED
:10AF80009C0146EA59E26C2F812F0E944845C6C0B9
:10AF9000D23031F580911B06823021F40E949682D6
:10AFA0008111E7C080912202882309F4B7C011E023
:10AFB00080911B06823009F010E06091540E709170
:10AFC000550E8091560E9091570E0E94C34D00E091
:10AFD0009C0148E959E26C2F812F0E9448459EC090
:10AFE000D33031F580911B06833021F40E94968284
:10AFF0008111D9C080912202882309F48FC011E009
:10B0000080911B06833009F010E06091580E70911A
:10B01000590E80915A0E90915B0E0E94C34D00E034
:10B020009C014AE859E26C2F812F0E94484576C066
:10B03000D43031F580911B06843021F40E94968231
:10B040008111CBC080912202882309F467C011E0EE
:10B0500080911B06843009F010E060915C0E7091C5
:10B060005D0E80915E0E90915F0E0E94C34D00E0D8
:10B070009C014CE759E26C2F812F0E9448454EC03D
:10B08000D53031F580911B06853021F40E949682DF
:10B090008111BDC080912202882309F43FC011E0D4
:10B0A00080911B06853009F010E060916C0E709164
:10B0B0006D0E80916E0E90916F0E0E94C34D00E058
:10B0C0009C0142E759E26C2F812F0E94484526C01F
:10B0D000D63021F580911B06863021F40E9496829D
:10B0E0008111AEC0809122028823C1F011E08091CD
:10B0F0001B06863009F010E06091700E7091710EA1
:10B100008091720E9091730E0E94C34D00E09C01DD
:10B110004EE559E26C2F812F0E944845CF5FDF5FDB
:10B12000C53009F0F1CE87E080931A06A1C00E94D5
:10B130002D4E8091E805882309F4F0CE99C081E076
:10B140000E948B82A12CC12CD12CE12C10ECF12E71
:10B1500009E714E420E030E040E85FE360E57EE0EA
:10B160008DEA99E2A2DB8091E805882309F4F2CE0A
:10B170007FC081E00E948B82A12CC12CD12CE12CBC
:10B1800010ECF12E09E714E420E030E040E85FE342
:10B1900064E57EE08FE999E288DB8091E805882309
:10B1A00009F400CF65C081E00E948B82A12CC12CE4
:10B1B000D12CE12C10ECF12E09E714E420E030E072
:10B1C00040E85FE368E57EE081E999E26EDB80912B
:10B1D000E805882309F40ECF4BC081E00E948B82E2
:10B1E000A12CC12CD12CE12C10ECF12E09E714E498
:10B1F00020E030E040E85FE36CE57EE083E899E240
:10B2000054DB8091E805882309F41CCF31C081E02C
:10B210000E948B82A12CC12CD12CE12C10ECF12EA0
:10B2200009E714E420E030E0A9016CE67EE087E75E
:10B2300099E23BDB8091E805882309F42BCF18C005
:10B2400081E00E948B82A12CC12CD12CE12C10EC2E
:10B25000F12E09E714E420E030E0A90160E77EE088
:10B2600088E699E222DB8091E805882309F43ACF49
:10B27000DF91CF911F910F91FF90EF90DF90CF90D2
:10B28000AF9008956F927F928F929F92AF92BF92EC
:10B29000CF92DF92EF92FF920F931F93CF93DF93A2
:10B2A00000D01F92CDB7DEB761E081E00E94837EBF
:10B2B00060901C06712C61101AC080911B068111D0
:10B2C00004C00E9496828111C2C08091220288230C
:10B2D00009F4B5C081E090911B06911180E004E073
:10B2E00024E040ED58E2672D0E941445A8C081E09B
:10B2F000681226C080911B06813021F40E9496823C
:10B300008111ADC080912202882309F498C011E018
:10B3100080911B06813009F010E06091FC0D709166
:10B32000FD0D8091FE0D9091FF0D0E94C34D00E038
:10B330009C0140EC58E2672D812F0E9448457FC058
:10B3400082E0681226C080911B06823021F40E94A0
:10B35000968281119EC080912202882309F46FC0D9
:10B3600011E080911B06823009F010E06091000E20
:10B370007091010E8091020E9091030E0E94C34DB8
:10B3800000E09C0140EB58E2672D812F0E94484568
:10B3900056C083E068122CC080911B06833021F4D4
:10B3A0000E94968281118FC080912202882309F425
:10B3B00046C011E080911B06833009F010E08091B7
:10B3C000040E9091050EA091060EB091070E898390
:10B3D0009A83AB83BC83CE0101960F94FA4C00E0B4
:10B3E0009C0140EA58E2672D812F0E94484527C002
:10B3F00084E0681224C080911B06843021F40E94EE
:10B400009682811198C0809122028823C1F011E0B8
:10B4100080911B06843009F010E06091080E709155
:10B42000090E80910A0E90910B0E0E94C34D00E010
:10B430009C0140E958E2672D812F0E944845739492
:10B44000639485E0781237CF70921A068DC00E94FF
:10B450002D4E8091E805882309F437CF85C081E01F
:10B460000E948B82A12CC12CD12CE12C10E8F12E52
:10B4700007E714E420E030E040E85FE36CEF7DE0B4
:10B4800088EC98E212DA8091E805882309F43ACF33
:10B490006BC081E00E948B82A12CC12CD12CE12CAD
:10B4A00010E8F12E07E714E420E030E040E85FE325
:10B4B00060E07EE088EB98E2F8D98091E805882387
:10B4C00009F449CF51C081E00E948B8220E030E036
:10B4D00048EC52E46091040E7091050E8091060EC6
:10B4E0009091070E0F94D95720E030E040E251E4EC
:10B4F0000F94C1540F940F561F92812C912C98E2F7
:10B50000A92E9DE4B92E6B0115EFE12E1FE7F12E58
:10B5100000E010E02AE030E040E050E064E07EE04F
:10B5200088EA98E20E94DE7C0F908091E8058823EB
:10B5300009F43ACF19C081E00E948B82A12CC12C62
:10B54000D12CE12C10E8F12E07E714E420E030E0E4
:10B5500040E85FE368E07EE088E998E2A6D9809160
:10B56000E805882309F44FCF0F900F900F900F90AC
:10B57000DF91CF911F910F91FF90EF90DF90CF90CF
:10B58000BF90AF909F908F907F906F9008952F9273
:10B590003F924F925F926F927F928F929F92AF9263
:10B5A000BF92CF92DF92EF92FF920F931F93CF93B0
:10B5B000DF93CDB7DEB729970FB6F894DEBF0FBE85
:10B5C000CDBF1C0179876887CA01B901E982FA8277
:10B5D0000B831C83DE82CD82AF8220E030E040E22C
:10B5E00051E40F94D9576B017C0120E030E040E03A
:10B5F00057EC0F949E5718162CF0C12CD12CE12C2F
:10B6000027ECF22EC701B6010F940A562B013C011C
:10B6100020E030E040E251E469817A818B819C81B5
:10B620000F94D9574B015C0120E03EEF4FEF56E4F9
:10B630000F949B5587FD07C0812C9EEF992EAA245D
:10B64000AA9496E4B92E20E030E040E251E4E88587
:10B65000F98560817181828193810F94D9576B0143
:10B660007C01C301B2010F943D569B01AC01C7019F
:10B67000B6010F94C1540F940F5669837A838B835C
:10B680009C83C501B4010F940A567B018C01E41818
:10B69000F50806091709FF81FF938D809E808EE2D1
:10B6A000A82E8DE4B82EC980DA80A30192016885A6
:10B6B0007985C1010E94DE7C0F9029960FB6F8941F
:10B6C000DEBF0FBECDBFDF91CF911F910F91FF90D5
:10B6D000EF90DF90CF90BF90AF909F908F907F9032
:10B6E0006F905F904F903F902F9008959F92AF92F0
:10B6F000BF92CF92DF92EF92FF920F931F93CF935F
:10B70000DF9300D01F92CDB7DEB761E081E00E94E9
:10B71000837E90901C06B12C91101AC080911B065C
:10B72000811104C00E9496828111D4C080912202AE
:10B73000882309F4C7C081E090911B06911180E035
:10B7400004E024E04EE758E26B2D0E941445BAC095
:10B7500081E098122CC080911B06813021F40E9458
:10B7600096828111BFC080912202882309F4AAC069
:10B7700011E080911B06813009F010E08091400EAD
:10B780009091410EA091420EB091430E89839A830D
:10B79000AB83BC83CE0101960F949A4D00E09C01CF
:10B7A0004AE658E26B2D812F0E9448458BC082E00B
:10B7B00098122CC080911B06823021F40E94968240
:10B7C0008111ACC080912202882309F47BC011E072
:10B7D00080911B06823009F010E08091440E909118
:10B7E000450EA091460EB091470E89839A83AB8394
:10B7F000BC83CE0101960F949A4D00E09C0146E572
:10B8000058E26B2D812F0E9448455CC083E098125E
:10B810002CC080911B06833021F40E9496828111F6
:10B8200099C080912202882309F44CC011E08091D4
:10B830001B06833009F010E08091480E9091490E6C
:10B84000A0914A0EB0914B0E89839A83AB83BC833F
:10B85000CE0101960F949A4D00E09C0142E458E21B
:10B860006B2D812F0E9448452DC084E098122AC07C
:10B8700080911B06843021F40E949682811186C03B
:10B88000809122028823F1F011E080911B06843020
:10B8900009F010E080914C0E90914D0EA0914E0E4B
:10B8A000B0914F0E89839A83AB83BC83CE010196FE
:10B8B0000F949A4D00E09C014EE258E26B2D812FCF
:10B8C0000E944845B394939485E0B81225CFB09276
:10B8D0001A0677C00E942D4E8091E805882309F44E
:10B8E00025CF6FC081E00E948B82A12C66E3C62E1B
:10B8F0006DE4D62EE12C1CE3F12E0CE116E420E0E1
:10B9000030E040EA50E460E47EE084E798E23FDE25
:10B910008091E805882309F426CF53C081E00E9476
:10B920008B82A12C46E3C42E4DE4D42EE12C1CE3E3
:10B93000F12E0CE116E420E030E040EA50E464E44B
:10B940007EE080E698E223DE8091E805882309F412
:10B9500039CF37C081E00E948B82A12C26E3C22E12
:10B960002DE4D22EE12C1CE3F12E0CE116E420E0B4
:10B9700030E040EA50E468E47EE08CE498E207DEE0
:10B980008091E805882309F44CCF1BC081E00E9418
:10B990008B82A12C86E3C82E8DE4D82EE12C1CE3EB
:10B9A000F12E0CE116E420E030E040EA50E46CE4D3
:10B9B0007EE088E398E2EBDD8091E805882309F4D6
:10B9C0005FCF0F900F900F900F90DF91CF911F914D
:10B9D0000F91FF90EF90DF90CF90BF90AF909F902E
:10B9E00008950F93CF93DF9361E081E00E94837EFF
:10B9F000C0911C06D0E0C11118C080911B068111B6
:10BA000004C00E9496828111B5C0809122028823D1
:10BA100061F081E090911B06911180E004E024E048
:10BA200049E55BE26D2F0E94144580917C0D877083
:10BA3000873009F058C0C130D9F480911B0681309D
:10BA400021F40E94968281119EC080912202882357
:10BA500009F4C1C081E090911B06913009F080E0AB
:10BA600003E02EE342E55BE26D2F0E941445B3C074
:10BA7000C230D9F480911B06823021F40E94968254
:10BA800081118BC080912202882309F4A4C081E037
:10BA900090911B06923009F080E003E02EE34BE426
:10BAA0005BE26D2F0E94144596C0C330D1F58091A2
:10BAB0001B06833021F40E949682811178C0809108
:10BAC0002202882309F487C081E090911B069330FD
:10BAD00009F080E003E02EE344E45BE26D2F0E9476
:10BAE000144584E03EC0C130F1F480911B068130E2
:10BAF00021F40E949682811164C0809122028823E1
:10BB000009F46BC081E090911B06913009F080E050
:10BB100000E22EE346E35BE26D2F0E94144582E0D3
:10BB200020C084E001C082E0C8131BC080911B06C6
:10BB30008C1304C00E949682811151C08091220210
:10BB4000882371F081E090911B069C1380E003E054
:10BB50002EE34CE25BE26D2F0E9414458C2F01C056
:10BB60008C2FDF5FCF5FD53009F045CF8F5F80939B
:10BB70001A063EC081E00E949D7D8091E8058823E1
:10BB800009F443CF35C08EE192E60E9420498091AE
:10BB9000E805882309F459CF2BC083E292E60E947E
:10BBA00020498091E805882309F46CCF21C088E200
:10BBB00092E60E9420498091E805882309F47FCF0E
:10BBC00017C080E49BE20E94DC7C8091E80588231A
:10BBD00009F493CF0DC084E0C4CF82E0C2CF8DE2E0
:10BBE00092E60E9420498091E805882309F4A6CFB7
:10BBF000DF91CF910F910895CF92DF92EF92FF9254
:10BC0000CF93C82F0E94B82F6B017C0124EA30E744
:10BC10004DE75FE3609133067091340680913506FD
:10BC2000909136060F949B5587FD05C04AEF50E072
:10BC300060E070E003C040E050E0BA01C40ED51EE1
:10BC4000E61EF71EC0922F06D0923006E092310613
:10BC5000F0923206C0932302CF91FF90EF90DF90D5
:10BC6000CF9008952F923F924F925F926F927F9262
:10BC70008F929F92AF92BF92CF92DF92EF92FF92FC
:10BC80001F93CF93DF93CDB7DEB728970FB6F89405
:10BC9000DEBF0FBECDBF1C01162F0E9496828823E7
:10BCA00031F010924A0680E00E949D7DDDC0209117
:10BCB0004206309143063E832D83232B09F4A0C016
:10BCC000E4E01E9FC001112498878F83FC01E55991
:10BCD000FD4F80809180A280B38020E030E04AE771
:10BCE00054E4C501B4010F94C1542B013C0120E080
:10BCF00030E04AE754E4C501B4010F94C2546B012B
:10BD00007C01809160028823B9F1113029F198F00B
:10BD1000123091F5409058025090590260905A02AA
:10BD200070905B02C0905C02D0905D02E0905E0279
:10BD3000F0905F0221C0409048025090490260900C
:10BD40004A0270904B02C0904C02D0904D02E0909D
:10BD50004E02F0904F0210C040905002509051029D
:10BD60006090520270905302C0905402D0905502DD
:10BD7000E0905602F09057022D813E81B901330FB9
:10BD8000880B990B0F943D56209133063091340661
:10BD900040913506509136060F94D9579B01AC015E
:10BDA000C501B4010F94C2549B01AC018F819885E9
:10BDB00085599D4F5C01FC0120833183428353836D
:10BDC0008D819E8197FF0CC0C301B2010F949E57D5
:10BDD00018168CF4F50140825182628273820BC086
:10BDE000C701B6010F949B5587FF05C0F501C082BE
:10BDF000D182E282F382812FFFDE81E080932202F2
:10BE0000109243061092420680912202882361F12B
:10BE100024E0129FF0011124E559FD4F80819181AA
:10BE2000A281B38189839A83AB83BC832DEC3CECE4
:10BE30004CEC5DE3609133067091340680913506D9
:10BE4000909136060F949E5787FD05C0CE0101964E
:10BE50000F94044B05C060E2CE0101960F947C4B19
:10BE6000BC01C1010E94AD4528960FB6F894DEBF13
:10BE70000FBECDBFDF91CF911F91FF90EF90DF906C
:10BE8000CF90BF90AF909F908F907F906F905F907A
:10BE90004F903F902F90089560E08AED9BE2E2CEB4
:10BEA00061E083ED9BE2DECE62E08CEC9BE2DACED9
:10BEB000CF93DF9300D01F92CDB7DEB70E9496825A
:10BEC000882331F010924A0680E00E949D7D57C081
:10BED00060914206709143066115710569F1072E64
:10BEE000000C880B990B0F943D562091330630912E
:10BEF000340640913506509136060F94D9579B0170
:10BF0000AC016091770270917802809179029091F2
:10BF10007A020F94C25460937702709378028093F0
:10BF2000790290937A0283E067DE81E080932202B7
:10BF30001092430610924206809122028823F9F063
:10BF40002091500530915105409152055091530573
:10BF500060917702709178028091790290917A02D3
:10BF60000F94C15469837A838B839C83CE0101969D
:10BF70000F94044BBC0180E69BE20E94AD450F90FC
:10BF80000F900F900F90DF91CF91089521E02093B3
:10BF90004A06609333067093340680933506909377
:10BFA000360620E040E060E070E080914E05909120
:10BFB0004F050C946A7D60E070E080E291E4E6CF8A
:10BFC00060E070E080E89FE3E1CF6DEC7CEC8CEC0E
:10BFD0009DE3DCCF6DEC7CEC8CEC9CE3D7CF8F92B7
:10BFE0009F92AF92BF92CF92DF92EF92FF920F9308
:10BFF0001F93CF93DF93CDB7DEB76E970FB6F8944C
:10C00000DEBF0FBECDBFD82E70934F0560934E0597
:10C0100061E081E00E94837EF0901C068CE0C82ED7
:10C02000E12C91E02AE6A22E2BE2B22E9E012F5F98
:10C030003F4F490131E0D31659F1D31628F082E081
:10C04000D81609F449C06CC0F110D2C0992389F008
:10C0500080911B0618166CF0209142063091430621
:10C060002F5F3F4F30934306209342068F5F8093AC
:10C070001B0680912202882309F432C100E010E0FF
:10C0800021E041E065EC7BE28E2D0E94B14428C1A5
:10C09000F110AEC0992389F080911B0618166CF040
:10C0A00020914206309143062F5F3F4F3093430665
:10C0B000209342068F5F80931B0680912202882383
:10C0C00009F411C100E010E021E041E06EEB7BE2F9
:10C0D0008E2D0E94B14407C1F1108AC0992389F0C6
:10C0E00080911B0618166CF0209142063091430691
:10C0F0002F5F3F4F30934306209342068F5F80931C
:10C100001B0680912202882309F40BC100E010E095
:10C1100021E041E067EB7BE28E2D0E94B14401C13A
:10C1200040917702509178026091790270917A0281
:10C1300040935005509351056093520570935305F9
:10C14000F11020C0992389F080911B0618166CF01D
:10C1500020914206309143062F5F3F4F30934306B4
:10C16000209342068F5F80931B06809122028823D2
:10C1700049F000E010E021E041E06DEA7BE28E2D25
:10C180000E94B14493E0D91233C06091B70C709112
:10C19000B80C8091B90C9091BA0C20917F0C2111B0
:10C1A00027C00F940A562091380230913902621745
:10C1B0007307F4F421E0F21219C080911B0681305C
:10C1C00021F40E9496828111C0C0809122028823AE
:10C1D00069F081E090911B06913009F080E004E065
:10C1E00024E04DE95BE26E2D0E94144582E0A2C07E
:10C1F00031E0F3121BC080911B06813021F40E94B4
:10C2000096828111ABC080912202882309F468C014
:10C2100081E090911B06913009F080E004E024E079
:10C2200043E95BE26E2D0E9414455AC082E0F81289
:10C230001BC080911B06823021F40E9496828111DE
:10C2400096C080912202882309F49BC081E09091DE
:10C250001B06923009F080E003E02EE349E85BE240
:10C260006E2D0E9414458DC093E0F9121BC0809181
:10C270001B06833021F40E949682811186C0809132
:10C280002202882309F4C3C081E090911B069330F9
:10C2900009F080E003E02EE340E85BE26E2D0E94AF
:10C2A0001445B5C024E0F2121BC080911B068430F7
:10C2B00021F40E949682811172C08091220288230B
:10C2C00009F4A5C081E090911B06943009F080E04C
:10C2D00003E02EE345E75BE26E2D0E94144597C014
:10C2E00032E0D31611F085E025C085E0F81219C0C0
:10C2F00080911B06853021F40E949682811159C0DD
:10C3000080912202882369F081E090911B0695308C
:10C3100009F080E003E02EE344E75BE26E2D0E942B
:10C32000144580912202882321F095E0F91609F442
:10C330004AC086E0E394F3942CE0C20E90E035E02E
:10C34000E31278CE80931A0666C081E00E949D7D3C
:10C350008091E805882309F438CF5DC081E00E9410
:10C360009D7D8091E805882309F44DCF54C08BED65
:10C370009FE50E9420498091E805882309F461CF58
:10C380004AC082E0D812AFCFCCCF80EE9FE50E94AA
:10C3900020498091E805882309F471CF3CC085EEDF
:10C3A0009FE50E9420498091E805882309F485CF04
:10C3B00032C08AEE9FE50E9420498091E8058823DB
:10C3C00009F49ECF28C06C2D86E00E94B63B8E01FA
:10C3D0000B5E1F4F23E041E06DEC7CEC8CEC9CE3AA
:10C3E0000F9450599F938F93BF92AF929F928F92C9
:10C3F0000F94625EB40180E194E00E94FA3A0F90DB
:10C400000F900F900F900F900F9086E093CF92E0D7
:10C41000D91269CF86CF6E960FB6F894DEBF0FBEE5
:10C42000CDBFDF91CF911F910F91FF90EF90DF90E3
:10C43000CF90BF90AF909F908F9008954FEF6CE496
:10C440007FE580E0CCCD4FEF60E57FE581E0C7CDB3
:10C450004FEF64E57FE582E0C2CD4FEF68E57FE511
:10C4600083E0BDCD0F93CF93DF9361E081E00E9425
:10C47000837ED0911C06C0E0D1111AC080911B06AA
:10C48000811104C00E94968281118BC0809122028A
:10C49000882309F47EC081E090911B06911180E011
:10C4A00004E024E047E25BE26C2F0E94144571C077
:10C4B000D130D9F480911B06813021F40E949682FC
:10C4C000811178C080912202882309F462C081E042
:10C4D00090911B06913009F080E003E02EE34DE1DE
:10C4E0005BE26C2F0E94144554C0D230D9F4809185
:10C4F0001B06823021F40E949682811165C08091D2
:10C500002202882309F445C081E090911B069230F5
:10C5100009F080E000E22EE34FE05BE26C2F0E9426
:10C52000144537C0D330D1F480911B06833021F4F9
:10C530000E949682811152C080912202882349F183
:10C5400081E090911B06933009F080E000E22EE339
:10C550004CE95AE26C2F0E9414451BC0D430C9F438
:10C5600080911B06843021F40E949682811140C084
:10C5700080912202882369F081E090911B0694301B
:10C5800009F080E000E22EE347E85AE26C2F0E94B7
:10C590001445CF5FDF5FC53009F06ECFC0931A0638
:10C5A00030C081E00E949D7D8091E805882309F4D8
:10C5B0006DCF27C081EF9CE50E9420498091E8055E
:10C5C000882309F47FCF1DC089E19BE20E94DC7CB7
:10C5D0008091E805882309F492CF13C08BEA9AE290
:10C5E0000E94DC7C8091E805882309F4A5CF09C06E
:10C5F00088E99AE20E94DC7C8091E805882309F4AE
:10C60000B7CFDF91CF910F910895CF92DF92EF9244
:10C61000FF920F931F938091D908811103C08BE182
:10C6200099E002C089ED98E026E2C22E2CE2D22EDB
:10C630007C0109E11CE22CE233E64FE253E662E1C1
:10C640007CE28CE09CE20E94917F1F910F91FF9011
:10C65000EF90DF90CF90089580E00C949D7D8BE16A
:10C6600099E00E947C8D0E94967D0C94B4880E9473
:10C670001E9221E030E0811102C020E030E03093D2
:10C6800043062093420610921C0681E08093E80541
:10C6900083E0809322020895EF92FF920F931F93FD
:10C6A000CF93DF9380914406882331F00E942E932C
:10C6B000909355058093540561E081E00E94837E4C
:10C6C000C0911C06D0E0C11118C080911B068111D9
:10C6D00004C00E949682811197C080912202882313
:10C6E00061F081E090911B06911180E004E024E06C
:10C6F00047E05CE26D2F0E9414458091280985FD7A
:10C700001FC083FF1DC0C130C9F480911B0681305A
:10C7100021F40E949682811180C080912202882398
:10C7200069F081E090911B06913009F080E000E211
:10C730002EE343E05CE26D2F0E94144592E001C0BD
:10C7400091E080912202882309F456C0E12CF12C5B
:10C7500011E01C0F2091540530915505E216F306A7
:10C7600008F04AC0C91343C0C901019760E070E0F6
:10C770008E199F090E94F18E9091280980911B06C5
:10C7800094FF1CC08C1350C00E949682882309F429
:10C790004BC08BE199E00E94C39110921C0682E08D
:10C7A00090E0909343068093420681E08093E805F1
:10C7B0001092450683E08093220254C08C1304C07B
:10C7C0000E94968281113FC080912202882369F0E5
:10C7D00081E090911B069C1380E000E024ED36E19F
:10C7E00041EE5BE26D2F0E94A746912F01C09F5F33
:10C7F0008FEFE81AF80AAECFDF5FCF5FD53009F0D0
:10C8000062CF90931A062EC081E00E949D7D809198
:10C81000E805882309F461CF25C029DF8091E80568
:10C82000882309F47ACF1EC0809122028823E9F27E
:10C8300081E090911B069C1380E001E024ED36E13D
:10C8400042EF5BE2CFCF0E94B77C20E040E060E0A7
:10C8500070E085E093E60E946A7D8091E805882378
:10C8600009F4B2CFDF91CF911F910F91FF90EF901C
:10C870000895CF93DF93EC01CB01BA010F943D569D
:10C880000F940A5679836883DF91CF91089569E305
:10C8900074E680ED94E60C94C17D0F931F93CF93C3
:10C8A000DF9361E081E00E94837EC0911C06D0E0AE
:10C8B00081E0C11122C0882389F080911B061816DF
:10C8C0006CF020914206309143062F5F3F4F30932A
:10C8D0004306209342068F5F80931B0680912202BD
:10C8E000882309F441C000E010E020E041E06BE85B
:10C8F0007DE28D2F0E94B14437C0C130D1F48091C8
:10C900001B06813021F40E949682811137C08091EC
:10C910002202882349F181E090911B06913009F0B1
:10C9200080E000E22EE340E85DE26D2F0E941445B6
:10C930001BC0C230C9F480911B06823021F40E94D2
:10C940009682811122C080912202882369F081E0C1
:10C9500090911B06923009F080E000E22EE34CE655
:10C960005DE26D2F0E941445DF5FCF5F80E0D53020
:10C9700009F09FCF83E080931A060DC0C093FE0B91
:10C980008091E805882319F206C0C093FE0B8091C0
:10C99000E8058823C1F2DF91CF911F910F9108958F
:10C9A0000F943D560F940A56CB010D940349EF9214
:10C9B000FF920F931F93CF93DF93CDB7DEB72B97E3
:10C9C0000FB6F894DEBF0FBECDBF7C014091570576
:10C9D000842F042E000C990B20915805223051F021
:10C9E000233019F02AEB3DE20AC047FF06C026ECCF
:10C9F0003DE205C028ED3DE202C02FEC3DE29F93F1
:10CA00004F933F932F938E010F5F1F4F1F930F93F1
:10CA10000F94625E40913602509137024F50510997
:10CA200097010F900F900F900F900F900F904E1551
:10CA30005F050CF49A013093BC0C2093BB0C80E092
:10CA40000E94E1B7C8010E946E7F2B960FB6F89442
:10CA5000DEBF0FBECDBFDF91CF911F910F91FF9031
:10CA6000EF900895E091570587E1E802F001112465
:10CA7000ED54F34F808591859ACF7F928F929F924C
:10CA8000AF92BF92CF92DF92EF92FF920F931F93DC
:10CA9000CF93DF93782E809358056093570561E01C
:10CAA00081E00E94837ED0911C06C0E081E0D1111C
:10CAB0002EC0882389F080911B0618166CF02091F7
:10CAC0004206309143062F5F3F4F30934306209339
:10CAD00042068F5F80931B0680912202882309F40F
:10CAE00094C022E0721649F033E0731203C06CE97F
:10CAF0007DE205C06CE87DE202C06CEA7DE200E008
:10CB000010E021E041E08C2F0E94B1447EC0D13082
:10CB1000D9F480911B06813021F40E949682811104
:10CB20007DC080912202882309F46FC081E090913A
:10CB30001B06913009F080E004E024E047E15EE26A
:10CB40006C2F0E94144561C0D230D9F480911B062D
:10CB5000823021F40E949682811169C08091220264
:10CB6000882309F452C081E090911B06923009F0AD
:10CB700080E000E22EE34BE05EE26C2F0E94144561
:10CB800044C0D330D1F480911B06833021F40E943D
:10CB90009682811157C0809122028823B1F181E0F1
:10CBA00090911B06933009F080E000E22EE34FEFF6
:10CBB0005DE26C2F0E94144528C0D43031F580917D
:10CBC0001B06843021F40E949682811146C0809118
:10CBD00022028823D1F011E080911B06843009F0F5
:10CBE00010E02091570537E12303F0011124ED54A3
:10CBF000F34F808591850F94034900E09C0141EE3D
:10CC00005DE26C2F812F0E944845CF5FDF5F80E09F
:10CC1000C53009F04CCFC0931A065CC081E00E9479
:10CC20009D7D8091E805882309F47BCF53C08091D6
:10CC30005F0590916005BBDE8091E805882309F4CB
:10CC40008DCF48C08091610590916205B0DE8091E2
:10CC5000E805882309F49FCF3DC081E00E948B82C4
:10CC60000091570527E1020380011124F801ED54DA
:10CC7000F34F60857185072E000C880B990B0F947C
:10CC80003D5620E030E040EF52E40F94C1540F9441
:10CC90000F56F801E554F34F1F9282E3882E85E684
:10CCA000982E97E4A92E94E6B92E6B011AEAE12E8C
:10CCB000F12C00E010E028E730E040E050E0BF0158
:10CCC00080EF9DE20E94DE7C0F908091E805882332
:10CCD00009F47DCFDF91CF911F910F91FF90EF90DD
:10CCE000DF90CF90BF90AF909F908F907F900895EE
:10CCF00060E081E0C2CE8F929F92AF92BF92CF92BE
:10CD0000DF92EF92FF920F931F93CF93DF934C012B
:10CD10005B016A0160E085E00E94837ED0911C0681
:10CD2000F12C82E0E82ED1111AC0809122028823D2
:10CD300021F180912702823041F0833019F461E4BF
:10CD40007DE205C06FE27DE202C061E57DE200E0C8
:10CD500010E021E041E08F2D0E94B1440EC0D1309F
:10CD600061F480912202882341F000E010E020E08D
:10CD700041E0B4018F2D0E94B144A114B10481F0AF
:10CD8000D23081F480912202882309F46EC000E041
:10CD900010E020E041E0B5018F2D0E94B14465C054
:10CDA000C2E001C0C3E0C114D10491F0DC130FC094
:10CDB00080912202882351F000E010E020E041E061
:10CDC000B6018F2D0E94B144CD2F01C0CD2FCF5F72
:10CDD00021E030E0A114B10411F420E030E081E062
:10CDE00090E0C114D10411F480E090E0820F931F11
:10CDF000029781F0DC130DC080912202882349F054
:10CE000000E010E020E041E06AE67DE28F2D0E9424
:10CE1000B144CF5FDC1314C080912202882371F0EB
:10CE200000E010E021E040E06FE57DE28F2D0E9400
:10CE3000B144609156058F2D0E944B44E09222022E
:10CE4000F394DF5F85E0F8126ECFCF5FC0931A06D0
:10CE5000DF91CF911F910F91FF90EF90DF90CF90D6
:10CE6000BF90AF909F908F900895C3E0C114D104FC
:10CE700009F0ADCFADCF40E050E060E070E084E27B
:10CE80009DE239CF4BE15DE26BE07DE282E09DE225
:10CE900032CF40E050E062EF7CE289EE9CE22BCFA3
:10CEA00040E050E06AED7CE28BEC9CE224CF40E075
:10CEB00050E06CEB7CE28FEA9CE21DCF43EA5CE23F
:10CEC00062E97CE282E89CE216CF40E050E064E751
:10CED0007CE28BE69CE20FCF40E050E06BE57CE229
:10CEE0008EE49CE208CF40E050E061E47CE280E424
:10CEF0009CE201CF40E050E061E37CE288E29CE20A
:10CF0000FACE61116093270240935605082E000C5B
:10CF1000990BAA0BBB0B8C309105A0F5FC0188275F
:10CF2000EA56FF4F8F4F0D94235982E497E61FC0B6
:10CF300089E497E61CC08CE697E619C08EE597E673
:10CF400016C085E697E613C08AE797E610C083E728
:10CF500097E60DC087E597E60AC080E597E607C02B
:10CF60001092FE0B8DE494E602C08BE397E60097E7
:10CF700049F021E020934A0620E040E060E070E0C4
:10CF80000C946A7D0C94967DCF92DF92EF92FF9283
:10CF90000F931F9388EEC82E8EE2D82EE12CF12C31
:10CFA0000DED1EE22CE233E644ED58E868ED7EE23A
:10CFB00083ED9EE20E94917F1F910F91FF90EF9071
:10CFC000DF90CF9008959091280993FB882780F9EE
:10CFD00093FF06C081E090915807911101C080E055
:10CFE0000895EF92FF920F931F93CF93DF9361E029
:10CFF00081E00E94837EC0911C0610E0C11118C020
:10D0000080911B06811104C00E9496828111C8C1C3
:10D0100080912202882361F081E090911B0691119A
:10D0200080E004E024E047EC5EE2612F0E941445BA
:10D030008091280982FB002700F982FD07C0D1E01A
:10D040009091C616913019F0D0E001C0D02F83FB2B
:10D05000EE24E0F883FF03C0B6DFF82E01C0F12C08
:10D06000DD2309F458C0C130D9F480911B0681300A
:10D0700021F40E94968281119CC180912202882312
:10D0800009F4A9C181E090911B06913009F080E07C
:10D0900000E22EE34BEB5EE2612F0E9414459BC140
:10D0A000C230D9F480911B06823021F40E9496820E
:10D0B000811187C180912202882309F48CC181E00B
:10D0C00090911B06923009F080E003E02EE340EBE4
:10D0D0005EE2612F0E9414457EC1C33009F063C037
:10D0E00080911B06833021F40E949682811175C1C4
:10D0F00080912202882309F46EC181E090911B0681
:10D10000933009F080E003E02EE34BEA5EE2612F0A
:10D110000E94144560C18091C616823029F053DF09
:10D120008823F9F001111DC0C130E9F480911B067C
:10D13000813021F40E949682811159C1809122028E
:10D14000882309F45CC181E090911B06913009F0BD
:10D1500080E000E22EE34EE95EE2612F0E9414457A
:10D160004EC1D1E001C0D2E0CD131BC080911B069F
:10D170008C1304C00E949682811143C180912202C7
:10D18000882371F081E090911B069C1380E003E0FE
:10D190002EE347E95EE2612F0E941445DC2F01C0B7
:10D1A000DC2FDF5F01C0D4E0CD131BC080911B06D4
:10D1B0008C1304C00E94968281112DC1809122029D
:10D1C000882371F081E090911B069C1380E003E0BE
:10D1D0002EE34BE85EE2612F0E941445DC2F01C074
:10D1E000DC2F81E08D0FC81318C080911B068C13B3
:10D1F00004C00E949682811118C180912202882366
:10D2000061F081E090911B069C1380E003E02EE327
:10D210004DE75EE2612F0E94144582E08D0F409140
:10D22000BB0C5091BC0C90917F0C911107C02091C8
:10D2300038023091390242175307DCF0C81333C06B
:10D2400080911B068C1304C00E9496828111F7C046
:10D2500080912202882339F181E090911B069C1372
:10D2600080E000E22EE345E65EE2612F0E94144575
:10D270001AC0C81318C080911B068C1304C00E94EA
:10D2800096828111E6C080912202882361F081E0BC
:10D2900090911B069C1380E003E02EE345E55EE2DF
:10D2A000612F0E941445DD5FCD1318C080911B06CD
:10D2B0008C1304C00E9496828111D5C080912202F5
:10D2C000882361F081E090911B069C1380E003E0CD
:10D2D0002EE347E45EE2612F0E94144591E09D0F2A
:10D2E000EE2009F43BC0F11053C0C91318C080915F
:10D2F0001B068C1304C00E9496828111BEC08091CF
:10D300002202882361F081E090911B069C1380E04B
:10D3100000E22EE346E35EE2612F0E94144582E0C4
:10D320008D0FC81318C080911B068C1304C00E9477
:10D3300096828111ACC080912202882361F081E045
:10D3400090911B069C1380E003E02EE345E25EE231
:10D35000612F0E94144593E09D0F1AC0C91316C097
:10D3600080911B068C1302C00E949682809122023B
:10D37000882361F081E090911B069C1380E000E21D
:10D380002EE34CE15EE2612F0E94144592E09D0F76
:10D390001F5FCF5F153009F031CE90931A0680C021
:10D3A00081E00E949D7D8091E805882309F430CEBC
:10D3B00077C00E94E7888091E805882309F45DCE54
:10D3C0006FC084EC97E60E9420498091E80588238D
:10D3D00009F470CE65C0D4E004CF8FEA9BE60E94CA
:10D3E00020498091E805882309F482CE59C00E9423
:10D3F000F8888091E805882309F4A0CE51C0D2E0D6
:10D40000D0CE82E392E60E9420498091E8058823ED
:10D4100009F4B4CE45C084E39EE60E942049809181
:10D42000E805882309F4CACE3BC08AEC9BE70E943A
:10D4300020498091E805882309F4DFCE31C085E7D3
:10D440009EE20E94DC7C8091E805882309F400CFED
:10D4500027C088E796E60E9420498091E805882346
:10D4600009F411CF1DC08CEA9DE60E9420498091ED
:10D47000E805882309F422CF13C083E49EE20E94CA
:10D48000DC7C8091E805882309F439CF09C08CE45D
:10D4900093E60E9420498091E805882309F44BCF48
:10D4A000DF91CF911F910F91FF90EF9008956091C0
:10D4B000AF0C70E080E00C94B8B260918B02709178
:10D4C0008C02072E000C880B990B0F943D562AE016
:10D4D00037ED43E25CE30F94D95760938702709372
:10D4E00088028093890290938A020895CF93DF93F4
:10D4F000EC01CB01BA010F943D560F940F5668838F
:10D50000DF91CF91089580E00C94E1B766E77AE669
:10D510008CE89AE60C94C17D0F943D560F940F56FB
:10D52000862F0D948748EF92FF920F931F93CF930E
:10D53000DF9300D01F92CDB7DEB7082F7B010E948A
:10D540009682882331F010924A0680E00E949D7DE9
:10D550003BC060914206709143066115710551F020
:10D56000109243061092420681E080932202802F9F
:10D570000E9413AB80912202882331F184E0089F3E
:10D5800080011124045F114F6091E80B7091E90B49
:10D59000072E000C880B990B0F943D569B01AC0194
:10D5A000F80160817181828193810F94D9576983D9
:10D5B0007A838B839C8360E2CE0101960F94144C96
:10D5C000BC01C7010E94AD450F900F900F900F90C6
:10D5D000DF91CF911F910F91FF90EF9008956FE52C
:10D5E0007FE280E0A0CF64E57FE281E09CCF20E095
:10D5F00040E060E070E00E946A7D81E080934A062E
:10D600001092E90B1092E80B08958FEE9AE6EFCF97
:10D6100083EF9AE6ECCF2F923F924F925F926F92F8
:10D620007F928F929F92AF92BF92CF92DF92EF92B2
:10D63000FF920F931F93CF93DF93CDB7DEB7299758
:10D640000FB6F894DEBF0FBECDBF1C017987688787
:10D6500069011A830983EB82BA01550F880B990B74
:10D660000F943D564B015C0120E030E040E057EC68
:10D670000F949E5718162CF0812C912CA12C27EC7E
:10D68000B22EC501B4010F940A562B013C01B6011C
:10D69000DD0C880B990B0F943D564B015C0120E08B
:10D6A0003EEF4FEF56E40F949B5587FD07C0812C4A
:10D6B0009EEF992EAA24AA9496E4B92EE885F985BE
:10D6C00060817181072E000C880B990B0F943D56D9
:10D6D0006B017C01C301B2010F943D569B01AC016B
:10D6E000C701B6010F94C1540F940F566C837D830C
:10D6F0008E839F83C501B4010F940A567B018C0170
:10D70000E418F50806091709FB81FF9389809A80C0
:10D7100087E4A82E84E6B82ECC80DD80A301920198
:10D7200068857985C1010E94DE7C0F9029960FB62D
:10D73000F894DEBF0FBECDBFDF91CF911F910F9147
:10D74000FF90EF90DF90CF90BF90AF909F908F9021
:10D750007F906F905F904F903F902F9008958F92A1
:10D760009F92AF92BF92CF92DF92EF92FF920F9370
:10D770001F93CF93DF9361E081E00E94837ED0917D
:10D780001C06C0E0D1111AC080911B06811104C093
:10D790000E949682811121C180912202882309F47E
:10D7A00013C181E090911B06911180E004E024E018
:10D7B0004FE45FE26C2F0E94144506C1D13011F591
:10D7C00080911B06813021F40E94968281110EC146
:10D7D00080912202882309F4F7C011E080911B0692
:10D7E000813009F010E080916502909166020F94FB
:10D7F000034900E09C0143E45FE26C2F812F0E940B
:10D800004845E2C0D23011F580911B06823021F4E8
:10D810000E9496828111FCC080912202882309F423
:10D82000D3C011E080911B06823009F010E0809196
:10D83000BB0C9091BC0C0F94034900E09C0145E3A4
:10D840005FE26C2F812F0E944845BEC0D33011F596
:10D8500080911B06833021F40E9496828111EDC0D5
:10D8600080912202882309F4AFC011E080911B0649
:10D87000833009F010E08091950C9091960C0F94F4
:10D88000034900E09C014DE25FE26C2F812F0E9472
:10D8900048459AC0D43001F580911B06843021F4AC
:10D8A0000E9496828111DEC080912202882309F4B1
:10D8B0008BC011E080911B06843009F010E080914C
:10D8C000AF0C0F94874800E09C0149E15FE26C2FA8
:10D8D000812F0E94484578C0D53011F580911B06F4
:10D8E000853021F40E9496828111DFC0809122024E
:10D8F000882309F469C011E080911B06853009F086
:10D9000010E080918B0290918C020F94034900E00B
:10D910009C014FE05FE26C2F812F0E94484554C06C
:10D92000D630D9F480911B06863021F40E9496826D
:10D930008111CDC080912202882309F445C081E085
:10D9400090911B06963009F080E003E02EE344E05E
:10D950005FE26C2F0E94144537C0D730D1F480911C
:10D960001B06873021F40E9496828111BAC08091F3
:10D970002202882349F181E090911B06973009F03B
:10D9800080E003E02EE349EF5EE26C2F0E94144535
:10D990001BC0D830C9F480911B06883021F40E9446
:10D9A00096828111A8C080912202882369F081E0CB
:10D9B00090911B06983009F080E003E02EE34AEED8
:10D9C0005EE26C2F0E941445CF5FDF5FC53009F027
:10D9D000D9CE89E080931A0697C081E00E949D7D90
:10D9E0008091E805882309F4D7CE8EC0E12C00E0B1
:10D9F00010E027EE33E04AE050E065E672E089E4AB
:10DA00009FE209DE8091E805882309F4E1CE7CC01D
:10DA100081E00E948B82E12C03E81AE622E231E0E9
:10DA200040E050E06BEB7CE08CE39FE2F4DD809122
:10DA3000E805882309F4F0CE67C081E00E948B825C
:10DA4000E12C0EE218EB2CE830E040E050E065E914
:10DA50007CE081E39FE2DFDD8091E805882309F423
:10DA6000FFCE52C081E00E948B82C090AF0CD12CBF
:10DA70001F9287E5882E8AE6982E96E8A92E9AE6C8
:10DA8000B92EE12CF12C8701EA9420E030E0A901C5
:10DA90006FEA7CE083E29FE20E94DE7C0F9080913F
:10DAA000E805882309F400CF2FC0E12C0DE51AE624
:10DAB00027EE33E04AE050E06BE872E084E19FE259
:10DAC000AADD8091E805882309F410CF1DC085E008
:10DAD0009BE60E9420498091E805882309F42ACF1B
:10DAE00013C088E09BE60E9420498091E8058823C6
:10DAF00009F43DCF09C089EE9EE70E94204980913C
:10DB0000E805882309F44FCFDF91CF911F910F9142
:10DB1000FF90EF90DF90CF90BF90AF909F908F904D
:10DB200008950E949682882329F010924A0680E088
:10DB30000E949D7D80E00C94DB430E9496828823A6
:10DB400041F020E040E060E070E081E99DE60E9465
:10DB50006A7D80E00C94C4A20F93CF93DF9361E0C1
:10DB600081E00E94837ED0911C06C0E0D11117C0D5
:10DB700080911B06811104C00E94968281114CC0C5
:10DB800080912202882309F43EC081E090911B0617
:10DB9000911180E004E024E041E85FE231C0D1303F
:10DBA000B9F480911B06813021F40E949682811184
:10DBB0003CC080912202882331F181E090911B06C4
:10DBC000913009F080E003E02EE340E75FE218C007
:10DBD000D530C9F480911B06853021F40E949682CD
:10DBE00081112DC080912202882369F081E09091FB
:10DBF0001B06953009F080E003E02EE34AE65FE281
:10DC00006C2F0E941445CF5FDF5FC53009F0AECFA7
:10DC100086E080931A061BC081E00E949D7D809162
:10DC2000E805882309F4ACCF12C08DE99DE60E9477
:10DC300020498091E805882309F4BBCF08C086E31A
:10DC400099E40E9420498091E805882359F2DF91E8
:10DC5000CF910F91089560E070E080E00E94B8B22B
:10DC60000E947BB80C94967D8F929F92AF92BF9248
:10DC7000CF92DF92EF92FF920F931F93CF93DF9398
:10DC800061E081E00E94837ED0911C06C0E0D1114A
:10DC90001AC080911B06811104C00E9496828111D6
:10DCA000ABC080912202882309F474C081E0909176
:10DCB0001B06911180E004E024E049EB5FE26C2F49
:10DCC0000E94144567C0D13011F580911B06813048
:10DCD00021F40E949682811198C0809122028823AB
:10DCE00009F458C011E080911B06813009F010E062
:10DCF0008091BB0C9091BC0C0F94034900E09C01F7
:10DD00004BEA5FE26C2F812F0E94484543C0D2301E
:10DD100009F580911B06823021F40E9496828111C0
:10DD20009AC0809122028823A9F111E080911B06FC
:10DD3000823009F010E08091950C9091960C0F9430
:10DD4000034900E09C0143EA5FE26C2F812F0E94AF
:10DD5000484520C0D330F1F480911B06833021F474
:10DD60000E94968281119CC080912202882391F0AA
:10DD700011E080911B06833009F010E08091AF0C18
:10DD80000F94584800E09C014FE85FE26C2F812F10
:10DD90000E9448458091BB0C9091BC0C2091950C41
:10DDA0003091960C232B11F4892BE9F0D430C9F46F
:10DDB00080911B06843021F40E9496828111A1C0BB
:10DDC00080912202882369F081E090911B069430B3
:10DDD00009F080E000E22EE346E85FE26C2F0E944B
:10DDE000144585E001C084E0CF5FDF5FC53009F0F6
:10DDF0004ECF80931A068BC081E00E949D7D80915A
:10DE0000E805882309F44DCF82C081E00E948B820F
:10DE1000C090BB0CD090BC0C1F9263E8862E6AE6C3
:10DE2000962E77E4A72E74E6B72E12E2E12EFF2499
:10DE3000F39400E010E020E030E0A9016BEB7CE01F
:10DE400082EB9FE20E94DE7C0F908091E8058823A0
:10DE500009F443CF5CC081E00E948B82C090950C96
:10DE6000D090960C1F923EE2832E38EB932E47E41F
:10DE7000A42E44E6B42E1CE8E12EF12C00E010E0C4
:10DE800020E030E0A90165E97CE087EA9FE20E949A
:10DE9000DE7C0F908091E805882309F442CF37C0DB
:10DEA00081E00E948B826091AF0C70E080E090E096
:10DEB0000F943B5629EC38EC48EC5EE30F94D957AD
:10DEC0000F940F561F9287E5882E8AE6982E9CEFB6
:10DED000A92E99E4B92E6B0114E6E12EF12C00E095
:10DEE00010E020E030E0A9016FEA7CE089E99FE2E0
:10DEF0000E94DE7C0F908091E805882309F434CFDE
:10DF000006C0A9DE8091E805882309F459CFDF9186
:10DF1000CF911F910F91FF90EF90DF90CF90BF9026
:10DF2000AF909F908F90089580E095E29093730555
:10DF3000809372058CE491E0909377058093760549
:10DF400080EC9EEF909375058093740590916E051B
:10DF500080E2890F863740F080EF890F20E431E0BE
:10DF600030937505209374051092700580937105A8
:10DF70008FEF80936F0508958F929F92BF92CF92FB
:10DF8000DF92EF92FF920F931F93CF93DF931F9235
:10DF9000CDB7DEB7F7D7882309F4D6C18091420602
:10DFA000863214F085E202C087FD80E0282F082E1B
:10DFB000000C330B3093430620934206982F990FA1
:10DFC000890F80936E058091D205882309F4BCC126
:10DFD00020917405309175050091700510917105BF
:10DFE000020F131FE0907205F09073058091760583
:10DFF00090917705E80EF91E01304FE7140768F09D
:10E0000031952195310930937505209374056CED98
:10E0100070E085E090E00F94864FF7FE15C0809188
:10E020007605909177059195819591099093770563
:10E030008093760568E171E085E090E00F94864F6B
:10E0400081E080936F0517C081E0E81680E4F80650
:10E0500094F06BE470E084EF91E00F94864F809130
:10E060006405815080936405882311F05DDF6CC1E5
:10E070001092D20569C12091760530917705C701CC
:10E080009A508130934108F098C08F2D992787FDD1
:10E090009A950A9765E070E00F94D258812F17FF88
:10E0A00002C087E0810F482F45954595459581E051
:10E0B00090E0A0E0B0E004C0880F991FAA1FBB1F2A
:10E0C0004A95D2F7FB01EE0FFF1FEA59FA4F408144
:10E0D00051818A0108231923012B09F419C1809564
:10E0E0009095842395239183808384E090E0861B20
:10E0F000970B4091D3055091D405840F951F9093B1
:10E10000D4058093D3058091650581508093650582
:10E11000811103C082E08093D205932F9095991FBF
:10E120009927991F80916F05881F8827881F981746
:10E13000F1F03195219531093093770520937605DB
:10E1400020E130E040E050E060EF7FEF8FEF9FEFA5
:10E150000E94543A2091740530917505620F731F27
:10E16000709375056093740560E773E021C080913A
:10E170007405909175059195819591099093750518
:10E180008093740520E130E040E050E060EF7FEFE5
:10E190008FEF9FEF0E94543A2091760530917705DA
:10E1A000620F731F709377056093760560E872E0E5
:10E1B00085E090E00F94864FABC0121613060CF06A
:10E1C000A7C0FDE3FF1A41E0E41642E0F40608F0C0
:10E1D0009FC080916E05181B103108F099C03195D1
:10E1E00021953109309377052093760560E773E038
:10E1F00083E090E00F94864F8FEF80936F0521E0CE
:10E2000012300CF020E08EEF810F8C30A0F0809166
:10E2100074059091750541E050E01816190614F048
:10E2200040E050E030E04217530709F055C09195A7
:10E230008195910927C0143050F520E030E0A90104
:10E2400060EC7FEF8FEF9FEF0E94543A20917405AE
:10E2500030917505620F731F709375056093740597
:10E2600061157E4F34F480E09EEF909375058093A6
:10E27000740580917405909175058130924064F128
:10E2800080E092E0909375058093740525C01C3062
:10E290001CF120E430E040E050E060E070E0CB01B1
:10E2A0000E94543A2091740530917505620F731FD6
:10E2B000709375056093740561157E4F34F480E0AA
:10E2C0009EEF9093750580937405809174059091ED
:10E2D000750581309240A4F68091D2058230C1F458
:10E2E00080E4809365058FEF9FEF9093670580939F
:10E2F0006605909369058093680590936B058093FC
:10E300006A0590936D0580936C0581E08093D2053A
:10E31000209170053091710580917405909175057B
:10E32000820F931F90937105809370052091720561
:10E33000309173058091760590917705820F931F38
:10E34000909373058093720561E084E194E00E94EC
:10E35000EB34809148048E3130F0809148048E3344
:10E3600008F456C05AC080914A048A30B0F384E65B
:10E37000E82E85E0F82E9AE0892E912CB82C809119
:10E38000480490E094012C5F3F4F281739075CF454
:10E3900042E0E40EF11C85E0880E911CEEE18E1641
:10E3A000910461F7DACF80914A04881588F330E050
:10E3B000C12CD12CF70182819381A0E0B0E00C2C1C
:10E3C00004C0B695A795979587950A94D2F780FDD6
:10E3D00007C0FFEFCF1ADF0A385F303859F7D8CFC0
:10E3E00000E010E0A801480D591D8091480490E01C
:10E3F000481759073CF080914A0490E0841795072C
:10E400000CF056C00F5F1F4F0430110559F7E1CFD4
:10E4100080914A048C3308F056C08091D20588233D
:10E42000B1F080917305482F582F550F550B9A0165
:10E4300033272F5F3F4F8091480490E0281739071A
:10E440003CF080914A04841708F04EC001C0B3D557
:10E45000809148048B30D8F40091D3051091D405F5
:10E4600069E080E00E94B63BC8010E94BB3B69E0C6
:10E470008EE60E94B63B2091640583E090E0821B0B
:10E4800091096FEF7FEF8254904D0E940F3C0E94E4
:10E490009682882391F10F90DF91CF911F910F9178
:10E4A000FF90EF90DF90CF90BF909F908F90C0C56E
:10E4B00027E04B2D400F632F84E194E039830E94C5
:10E4C000FC3639819FCF20E14DE360916E0584E1F8
:10E4D00094E00E94FC3620E14CE360916E0584E1FB
:10E4E00094E00E94FC3699CF6091710502E022E031
:10E4F00084E194E00E943D37ABCF0F90DF91CF9144
:10E500001F910F91FF90EF90DF90CF90BF909F9061
:10E510008F9008956CEB7FE682E079D5E4E6F5E034
:10E5200088E3828783E0808380E481831382128280
:10E53000158214821782168211861086F5DC82E11C
:10E5400090E0909343068093420608958F929F92A5
:10E55000AF92BF92CF92DF92EF92FF9260918F05C0
:10E5600020E030E090E080E0F901EC59FA4FC7A4D8
:10E57000CC2011F061E0620F8C29722F7295707FB0
:10E5800040E050E0D12CE12CF12C46015701042E43
:10E5900004C0B694A794979487940A94D2F780FE07
:10E5A00008C0E92FF0E0EC59FA4FA72FA42BA2AB3B
:10E5B0009F5F4F5F5F4F4530510539F72F5F3F4FEA
:10E5C0002330310589F660938F0540E050E020E06C
:10E5D00090E0A0E0B0E06C017D01042E04C0F69450
:10E5E000E794D794C7940A94D2F7C0FE05C020934D
:10E5F0008D052AE335E007C02E504F5F5F4F453051
:10E60000510549F7F4CF422F3150A0F0225F6C0141
:10E610007D01032E04C0F694E794D794C7940A941E
:10E62000D2F7C0FEF0CF40938E05809190058230E6
:10E6300069F403C020938E05F8CF80918C051816DD
:10E6400014F08CEF01C084E080938C05FF90EF9074
:10E65000DF90CF90BF90AF909F908F90089580E013
:10E6600090E0FC01EC59FA4F168203968E31910529
:10E67000C1F70895E4E6F5E010828AE0818383E043
:10E6800080A78FE084A78FE187A780AB81AB5EDF97
:10E69000E6CF1F93CF93DF93EC01162FE0DF80913D
:10E6A00067058093890587E380938A0586E08093D8
:10E6B0008B056AE070E088EE93E00F94864F9091AE
:10E6C0006605915090936605992351F01092880544
:10E6D000188310926705109243061092420601C0FB
:10E6E0001882DF91CF911F9108952F923F925F92F0
:10E6F0006F927F928F929F92AF92BF92CF92DF9252
:10E70000EF92FF920F931F93CF93DF931F92CDB79A
:10E71000DEB784E08093220280914406882309F4C6
:10E7200070C280914206909143068E31910514F09B
:10E730008DE190E097FF02C080E090E09093430667
:10E7400080934206880F991F880F991F20916705B3
:10E75000422F022E000C550B4817590774F42D5FF9
:10E76000AC01421B510927FD5395423051051CF065
:10E770002093670502C08093670520916705422FAB
:10E78000022E000C550B841795077CF42350422F62
:10E79000022E000C550B481B590B423051051CF042
:10E7A0002093670502C0809367058091D205882376
:10E7B00009F427C22091A605222349F09091A505CE
:10E7C000920F9093A505933F14F41092A605823002
:10E7D00070F081508093D205823011F44BDF11C26A
:10E7E000843609F00EC281E08093D2050AC280917E
:10E7F00092058F5F809392054091900590E0242FC1
:10E8000030E035952795281739070CF0B3C0909163
:10E81000A70581E089278093A705109292054423DC
:10E8200009F4A8C090918C0580916405890F20910E
:10E830008D05821724F020918E052817D4F4919528
:10E8400090938C05209165052B5F2093650580933F
:10E85000640580918F053AE08302C0011124820F84
:10E86000911D27FD9A95C99724F064E182ED95E00A
:10E8700010DF90918C0580916405890F8093640569
:10E8800080919005882309F475C024E130E040E0D0
:10E8900050E060E070E0CB010E94543A672B682B97
:10E8A000692B09F067C0EAE6F5E080E090E020819E
:10E8B00021115AC09C01220F331F8901080F191F13
:10E8C000C80188599A4F892B09F454C020919005AA
:10E8D00030E02F5F3F4F032E000C440B550B60E0E0
:10E8E00070E0CB010E94543AFB01EC59FA4F42A967
:10E8F000242F30E0B4E035952795BA95E1F7F9017A
:10E90000E258FC4F808190E00C591A4F4F705091A3
:10E9100064056EE0469F500D1124452FFC01E5581B
:10E92000FC4F5081450FFC01E858FC4F90819695B3
:10E93000842F890FF80184838091650582502F5FB1
:10E940003F4FFAE02F9F800D1124F801858322E0CC
:10E9500030E040E050E060E070E0CB010E94543ACB
:10E960006E5FF801668306C0019633968A30910582
:10E9700009F09DCF90918805992341F080918705FA
:10E98000890F8093870587FD1092880580918805FF
:10E99000882309F4A2C020918705E09165052E1710
:10E9A0000CF49BC0022E000C330B0E2E000CFF0B40
:10E9B000CF014D96821793070CF48FC01091640518
:10E9C000E0908605CE2C0E2C000CDD08C601811BC4
:10E9D000910917FD93956EE070E00F94D258F62ED2
:10E9E000653008F07AC02E1B3F0BC90102966AE021
:10E9F00070E00F94D258062F633008F06EC0812C5F
:10EA0000912C540183940F2C04C0880C991CAA1CCF
:10EA1000BB1C0A94D2F7A62F660FBB0BBD016C5925
:10EA20007A4FFB0197A5892F882109F456C0FD0173
:10EA3000E258FC4FE0814E2F50E0812FFEE0FF9E18
:10EA4000800D11249A0125583C4FF901F080F80EF1
:10EA5000EF140CF442C0FA01E858FC4F1081412F2A
:10EA600050E04F0D511DF7FC5A95C416D506ACF574
:10EA700010928805282D20952923FB0127A723E044
:10EA800030E02A1B3B0B8091D3059091D405280FD1
:10EA9000391F3093D4052093D3056AE070E088E2F3
:10EAA00090E00F94864F20916505FAE00F9F200DAE
:10EAB0001124912F96958F2D890F8550809389056C
:10EAC00020938A0584E080938B0580919005815086
:10EAD00080939005882321F039DD0AE615E012C005
:10EAE00084E18093D205BBDDF8CF8291890F8083CA
:10EAF00080346CF0F80110820D5F1F4FF5E008388C
:10EB00001F07E9F0F80190819923B1F3EECF873325
:10EB10009CF3F8013297208180916705281764F3F0
:10EB2000022E000C330B082E000C990B0A9682174C
:10EB3000930714F368E782ED95E0ABDDDDCF8091BC
:10EB4000A605811124C024EF31E040E050E060E0F0
:10EB500070E0CB010E94543A672B682B692BB9F403
:10EB600022E030E040E050E060E070E0CB010E9445
:10EB7000543A672B682B692B09F099C18FEF80936A
:10EB8000A605813009F495C18FE78093A505809192
:10EB900088058823B1F18091A605882391F18091A1
:10EBA0008705873074F5209186058091A505281783
:10EBB00044F1022E000C330B082E000C990B0C961E
:10EBC00082179307F4F01092A605109288058091A1
:10EBD000D3059091D4050A969093D4058093D305DC
:10EBE0006AE070E088E290E00F94864F8091A5057E
:10EBF0008F5F8093890581E080938A0584E080930C
:10EC00008B0580914C0682FF04C080919105815054
:10EC100001C08AE0809391050E9496828823C1F00A
:10EC20008091D205811103C01092910511C08130ED
:10EC300079F48091880581110BC0809167058B5F05
:10EC40008093860584E3809387058CEF8093880505
:10EC500080919105811101C0EBD161E084E194E0E4
:10EC60000E94EB3430916505632F032E000C770B67
:10EC700080918F05AB012AE08202400D511D1124C5
:10EC8000425051098091480490E0841795072CF078
:10EC90008091A60581116BC06FC080914A0490E0FD
:10ECA00086179707ACF3FEE76F2EF3E07F2EC12C9B
:10ECB000D12CF30121913F01432F032E000C550B62
:10ECC000BA01695F7F4F8091480490E06817790727
:10ECD0004CF4365FFFEFCF1ADF0A23E0C216D104EF
:10ECE00041F7D6CF80914A0490E0841795078CF3C2
:10ECF0001091640546E4542E510EA12CB12CC6018E
:10ED00008C599A4F4C01822F90E01C01220C331C2D
:10ED1000F40187A590E0A0E0B0E00A2C04C0B6950D
:10ED2000A795979587950A94D2F780FF19C080918F
:10ED3000A7057101E80EF11CC701E4E0880F991FD7
:10ED4000EA95E1F7AC014F50504D7A0108E022E01E
:10ED5000432F612F84E194E039830E941535398176
:10ED6000125F5FEFA51AB50A1511D2CFB2CF80910D
:10ED70004804883008F49FC08091D205882369F048
:10ED8000909148049F3348F490914A04973328F0B7
:10ED9000823008F49EC081FD9CC080918805882344
:10EDA000B1F040918705242F042E000C330BB901DC
:10EDB0006D5F7F4F8091480490E0681779073CF0C1
:10EDC00080914A0490E0821793070CF090C000E015
:10EDD00010E0F801EC59FA4F8681882399F04581BB
:10EDE000842F042E000C990B2091480430E08217E8
:10EDF000930744F0029720914A0430E0281739071E
:10EE00000CF07DC00D5F1F4F0E31110511F7809181
:10EE10008B058823B1F040918A05242F042E000C25
:10EE2000330BB9016A5F7F4F8091480490E0681707
:10EE300079073CF080914A0490E0821793070CF028
:10EE400066C08091D205811101C0B5D0809148047F
:10EE50008A3008F06EC00091D3051091D40569E0A6
:10EE600080E00E94B63BC8010E94BB3B80916605D2
:10EE7000882309F45EC011E060E1C62ED12C809198
:10EE80006605811708F455C0B601611B7109660F4C
:10EE9000660F660F7CEDE72E7FE2F72E05E021E09E
:10EEA00041E084E194E00E9415351F5FE8CF81E0E6
:10EEB00066CE83EF6ACE24ECE22E2FE2F22E05E03E
:10EEC00022E042E06091A50584E194E00E941535BE
:10EED00053CF91EEE92E9FE2F92E08E022E047E3BE
:10EEE0006091670584E194E00E94153556CF24E0D7
:10EEF0006091860584E194E00E941C3768CF4250FF
:10EF000023E0648184E194E00E941C377BCF8EEC87
:10EF1000E82E8FE2F82E07E022E06091890584E177
:10EF200094E00E94153580918B05815080938B056C
:10EF300088CF0F90DF91CF911F910F91FF90EF90AD
:10EF4000DF90CF90BF90AF909F908F907F906F9009
:10EF50005F903F902F900895CF93DF9365E773E71D
:10EF600084E155D0C4E6D5E083E08A838AE08DA7AA
:10EF70001CA280DB1B821092430610924206DF9196
:10EF8000CF91089580914406882319F082E0809300
:10EF9000630584E0809322028091D205882349F0A2
:10EFA000909163058FEF890F8093630581E01916B7
:10EFB0000CF080E008950F9380914804853228F585
:10EFC00080914A048B3108F160E084E194E00E9472
:10EFD000EB3409E028E34BE164E284E194E00E9431
:10EFE0008D3761E084E194E00E94EB340E94DF837E
:10EFF000882359F063E285E20E94B63B6FEF7FEF12
:10F0000081E590E30F910C940F3C0F910895FB0163
:10F010001092D4051092D3058093D20520E040E0F1
:10F0200060E070E0CF0156D581E080934A060895F4
:10F0300010924A0680E081C58091690590916B0528
:10F0400089130DC080916A0590916C05891714F0A1
:10F050002FEF01C021E0820F80936A0508C0891755
:10F0600014F02FEF01C021E0820F8093690589130E
:10F070001BC02091D10521502093D10530E0832F72
:10F0800090E0DC01AA0FBB1FAC59BA4F880F991F43
:10F09000FC01EA59FA4F8581968116969C938E93CE
:10F0A00015973F5F231758F70895EF92FF921F932C
:10F0B000CF93DF931091D10520916605E22E022EA9
:10F0C000000CFF0830916505C32F032E000CDD0BEB
:10F0D000ECE6F5E040E0411709F446C0CF010397A4
:10F0E000DC019C91BF0161507109DB018C91981387
:10F0F0001DC0692F092E000C770B61507109C617CE
:10F10000D70711F039132DC09081BF0162507109EA
:10F11000DB018C91582F98170CF4592F25170CF1FF
:10F1200089170CF4892F8217E4F020C0BF016250C8
:10F130007109DB015C91652F052E000C770B615086
:10F140007109E616F70611F025130BC0582F981712
:10F150000CF4592F35172CF089170CF4892F8317CD
:10F160002CF44F5F3296B7CF80E001C081E0DF9191
:10F17000CF911F91FF90EF90089528E130E040E09B
:10F1800050E060E070E0CB010E94543A6093650566
:10F190002AE030E040E050E060E070E0CB010E9407
:10F1A000543A6093660581DF8111E7CF089590910D
:10F1B0006405811102C08FEF01C081E0980F937048
:10F1C000909364058091D1058F5F8093D10590E085
:10F1D000FC01EE0FFF1FEC59FA4F2091CE0525835D
:10F1E000880F991FFC01E659FA4F8091D005808362
:10F1F00008951F93CF93DF93C4E6D5E080E091E0BC
:10F200009093CE058093CD0580E095E09093D00556
:10F210008093CF0518821092D1051D8215E01E83C0
:10F2200081E0C5DF1B8310924306109242061C82C8
:10F23000DF91CF911F910895EF92FF920F931F934B
:10F24000CF93DF938091D105843008F4DEC090E045
:10F25000FC01EE0FFF1FEE59FA4F3581FC01EE0F56
:10F26000FF1FEC59FA4F6581AC0142505109361726
:10F2700039F0C0E0880F991FFC01E859FA4F82C0AD
:10F28000F12CDC01AA0FBB1FA659BA4F880F991F9A
:10F29000FC01E859FA4F8F2D90E0841795070CF088
:10F2A000B4C0BC01660F771F6C597A4FEB016D81BA
:10F2B0008C01000F111F0A591A4FE8012D816217A6
:10F2C000F1F0722F62170CF4762F3717ECF1261736
:10F2D0000CF4262F2317C4F1880F991F86599A4FD3
:10F2E000EC01288191E0808128170CF090E081E00A
:10F2F0006C9162170CF480E0981731F188C03613D6
:10F3000023C07C9120818C01000F111F04591A4FDA
:10F31000E8016881880F991F86599A4FEC0188810E
:10F32000122F72170CF4172F982F86170CF4962FA4
:10F33000911754F0922F27170CF4972F68170CF49D
:10F34000862F98170CF063C0F394A5CF7C01DFEFF4
:10F35000ED1AFD0A8C01000F111F06591A4FD80132
:10F360007C918C01000F111F04591A4FD8012C9168
:10F37000721729F1A081B22F72170CF4B72FAB17B7
:10F380003CF4CF5F8C2F90E084179507FCF23DC0D2
:10F3900027170CF4272F2A17A4F3880F991FDC01D5
:10F3A000AC59BA4F15962C9191E023170CF090E0D0
:10F3B00081E062170CF480E0981719F328C02081CF
:10F3C0002713DFCFD701AA0FBB1FAC59BA4F159631
:10F3D0002C91880F991FDC01AC59BA4F15968C916E
:10F3E000762F36170CF4732F982F82170CF4922F68
:10F3F00097173CF2962F63170CF4932F28170CF4F1
:10F40000822F98170CF4BDCF02C080E001C081E0CC
:10F41000DF91CF911F910F91FF90EF900895BF92D0
:10F42000CF92DF92EF92FF920F931F93CF93DF93D0
:10F430001F92CDB7DEB7A6DD882309F486C0809180
:10F44000CD059091CE05392F4091CF055091D00533
:10F4500020916405213061F02CF4211116C0CA01FD
:10F46000C3970AC0223031F0233079F4C39709C022
:10F47000C39607C0CA01C3969093D0058093CF0569
:10F4800004C09093CE058093CD051091CE050091D8
:10F49000D005311303C0051709F457C0183110F413
:10F4A0000A3048F01092D20568E270E080E991E0FD
:10F4B0000F94864F4AC08091D10590E0FC01EE0F79
:10F4C000FF1FEC59FA4F1583880F991FFC01E6596D
:10F4D000FA4F00838091420690916805282F291BDE
:10F4E00039F08093680581E012160CF080E05FDE51
:10F4F00080916705882321F081508093670501C0C2
:10F500009BDD9ADE8111CECF8091650518131DC059
:10F5100080916605081319C06CED70E085E090E0FD
:10F520000F94864F68E171E085E090E00F94864F7C
:10F530008091D3059091D40501969093D405809342
:10F54000D30582E08093670518DE61E084E194E0F2
:10F550000E94EB3480914804893058F4E090D30540
:10F56000F090D40567E080E00E94B63BC7010E949E
:10F57000BB3B06E32CE749E062E084E194E00E94B3
:10F580003D3710E08091D10530914804181708F0FC
:10F5900084C0412F50E0BA01660F771FFB01EC5980
:10F5A000FA4FA581FB01EA59FA4F2581CA0103965A
:10F5B000A21351C0FB01E459FA4F2081880F991F13
:10F5C000FC01EC59FA4FC080DC2CC2160CF4D22E90
:10F5D0008D2D95E08902A0011124425F5F4F832F9A
:10F5E00090E0481759070CF456C02C150CF4C22EA5
:10F5F000EC2DF5E0EF0290011124265F3F4F809142
:10F600004A0490E0281739070CF045C08C2D880F6C
:10F61000880F8C0DEBE0BE2EB80ECB0187599A4FA8
:10F620007C01DC14C4F12B2D0B2C000C330BA90135
:10F630004D5F5F4F8091480490E0481759073CF0B8
:10F6400080914A0490E0821793070CF053C0C39452
:10F6500095E0B90EE6CF880F991FFC01EC59FA4FDF
:10F660008081982F990F990F890F5BE0E52EE80EA6
:10F670004E2D0E2C000C550BBA016D5F7F4F832F62
:10F6800090E0681779073CF060914A0470E06417D5
:10F6900075070CF03EC01F5F75CF40916605842F43
:10F6A000880F880F480F455F642F042E000C770BDE
:10F6B000FB013396832F90E0E817F9073CF0809127
:10F6C0004A0490E0861797070CF045C08091D20558
:10F6D000811101C070DC2AD7882309F44AC00F9039
:10F6E000DF91CF911F910F91FF90EF90DF90CF901E
:10F6F000BF909ECCF7016081862F880F880F680F1E
:10F700006C5F04E024E04B2D84E194E00E948D378F
:10F710009ECFD22EA2170CF4DA2EC22E2A170CF48A
:10F72000CA2EFD2CFF0CFF0C8F2D8D0D30E094E0C8
:10F73000F92EF80ECD140CF4AECF6F2D630F04E04C
:10F7400024E04E2D84E194E039830E948D37D394D8
:10F7500039813B5FEFCF60916505862F880F880F59
:10F76000680F6C5F04E024E084E194E00E943D3780
:10F77000ADCF0F90DF91CF911F910F91FF90EF9040
:10F78000DF90CF90BF9008956FE07AE781E03FDC93
:10F7900030DDF3CC0F931F93CF93DF9361E081E0D3
:10F7A000B2D2D0911C06C0E0D11116C080911B06C8
:10F7B000811103C0BBD681119AC080912202882397
:10F7C00009F43CC081E090911B06911180E004E0B7
:10F7D00024E04AEA50E32FC0D130B1F480911B06F7
:10F7E000813019F4A3D681118AC080912202882326
:10F7F00029F181E090911B06913009F080E003E04F
:10F800002EE348E950E317C0D230C1F480911B06C3
:10F81000823019F48BD681117CC08091220288231A
:10F8200069F081E090911B06923009F080E003E0DE
:10F830002EE349E850E36C2F0E94144534D1182F71
:10F84000D330D1F480911B06833019F46FD6811127
:10F850006AC080912202882309F477C081E09091E8
:10F860001B06933009F080E000E22EE34AE750E304
:10F870006C2F0E94144569C0811169C0D430B1F465
:10F8800080911B06843019F451D6811153C08091A8
:10F890002202882319F181E090911B06943009F02F
:10F8A00080E000E22EE34CE650E315C0D530B1F421
:10F8B00080911B06853009F444C080912202882380
:10F8C00069F081E090911B06953009F080E000E23C
:10F8D0002EE34BE550E36C2F0E94144586E0CF5F8A
:10F8E000DF5FC53009F060CF80931A063BC081E02E
:10F8F00024D18091E805882309F45FCF33C080E3E9
:10F900009EE40E9420498091E805882309F46DCF88
:10F9100029C089EE9EE70E9420498091E80588234E
:10F9200009F47BCF1FC0E2D28091E805882309F457
:10F9300090CF18C0DED28091E805882309F4A7CFC4
:10F9400011C0F4D5811105C0B8CF112339F284E07C
:10F95000C6CF0E94F2D881E028D28091E8058823A2
:10F9600009F4ABCFDF91CF911F910F910895E091F2
:10F97000E905E63000F581E08E0F8093E90580917E
:10F98000420690914306A0E0B0E030911C06209121
:10F990001A0648E0E49FF0011124E651FA4F409125
:10F9A0003D0650913E065183408382839383A48316
:10F9B000B5833683278308950D94203D2F923F927F
:10F9C0004F925F926F927F928F929F92AF92BF926F
:10F9D000CF92DF92EF92FF920F931F93CF93DF931B
:10F9E00000D000D0CDB7DEB71C012B833C834D8304
:10F9F0005E8369837A83BBDF83E080932202309247
:10FA0000E7052092E60569817A817093E5056093A8
:10FA1000E4052B813C814D815E812093E00530938C
:10FA2000E1054093E2055093E305E092DC05F09296
:10FA3000DD050093DE051093DF05D0924306C092EA
:10FA40004206B0923E06A0923D069092DB0580925F
:10FA5000DA058C8D8093D90526960FB6F894DEBF13
:10FA60000FBECDBFDF91CF911F910F91FF90EF900F
:10FA7000DF90CF90BF90AF909F908F907F906F90CE
:10FA80005F904F903F902F900895FB01908181E00F
:10FA90008927808383E0809322024115510511F06C
:10FAA000FA011994089580917A0E9091770E891B2E
:10FAB0008F7071F49091280992FB882780F992FD4C
:10FAC00008C081E09091C616913019F080E0089549
:10FAD00081E00895E0913D06F0913E06E817F907B0
:10FAE00021F130914D0637FD10924D0690933E0660
:10FAF00080933D06709343066093420640931C0634
:10FB000020931A06865F914821F410924A061092BB
:10FB1000E9050E944A4482E08093220281E08093BA
:10FB2000E805109245061092D505089520E040E0C2
:10FB300060E070E086EF91E8CDCFE091E905EE233B
:10FB4000F9F0E150E093E90598E0E99FF001112414
:10FB5000DF01A651BA4F17962C911797811108C053
:10FB600016964C91169712966D917C91139703C03F
:10FB700040E060E070E0E651FA4F80819181AACFC9
:10FB8000D5CFCF93DF93FC01EB018091420690919A
:10FB9000430697FF04C0109243061092420640911C
:10FBA000DC055091DD056091DE057091DF058091E7
:10FBB000420690914306092E000CAA0BBB0B481776
:10FBC00059076A077B0724F4509343064093420683
:10FBD000809122028823D1F0209142063091430681
:10FBE0008091E0059091E105A091E205B091E305D7
:10FBF000BC01CD01620F731F811D911D1995BC01C0
:10FC00008091E6059091E7050E94AD458091370609
:10FC1000811108C08091D905882389F18091220241
:10FC2000882369F18091E4059091E505009791F0B2
:10FC300020914206309143064091E0055091E10544
:10FC40006091E2057091E305420F531F611D711D24
:10FC5000FE011995E091DA05F091DB05309741F04E
:10FC60008091D905811103C08091370681111995C2
:10FC70005DD4882321F080E0DF91CF915ECFDF91CA
:10FC8000CF9108950F931F93CF93DF93809122021A
:10FC9000882359F06091D6057091D70500E010E0F7
:10FCA00020E041E081E00E94B1448091D8058111BB
:10FCB0001CC081E08093D805C0913D06D0913E06DE
:10FCC00020E040E060E070E082E49EE703DF0E9415
:10FCD000CBF51092D80520E040E060E070E0CE0166
:10FCE000DF91CF911F910F91F5CEDF91CF911F91B1
:10FCF0000F910895009711F48EEB90E39093D70540
:10FD00008093D605BFCF282F10923C0680914206E3
:10FD1000909143068130904820F010924306109253
:10FD2000420680914406882331F0809142068093F8
:10FD30001B061092E80580911A061816BCF4082ECE
:10FD4000000C990B821B910920911B06022E000CBE
:10FD5000330B2817390754F097FF02C080E090E07A
:10FD600080931B06909343068093420680911B0666
:10FD70006623C1F090911C06891714F480931C0629
:10FD800020911C06022E000C330B2C5F3F4F482F96
:10FD9000082E000C550B2417350734F4845080933B
:10FDA0001C06089580931C060895882361F063E97A
:10FDB00072E084E690E00F94864F6AEB72E084E68E
:10FDC00090E00D94864F68EB71E084E190E00D9433
:10FDD000864FCF92DF92EF92FF92CF93DF93A6D31D
:10FDE000882361F00E9492A210924A0680E0DF917F
:10FDF000CF91FF90EF90DF90CF909FCE81E08093E6
:10FE00004A06C0914206D0914306209709F442C0A9
:10FE10001092430610924206BE010D2E000C880B74
:10FE2000990B0F943D562091140E3091150E409170
:10FE3000160E5091170E0F94D9572091550D3091F1
:10FE4000560D4091570D5091580D0F94C2546B01AF
:10FE50007C0120E030E040E050EC0F949E5787FD9D
:10FE600019C020E030E040EA50E4C701B6010F9429
:10FE70009B5518167CF0BE0182E00E9413ABC09225
:10FE8000550DD092560DE092570DF092580D82E02C
:10FE900080932202809122028823C9F085E59DE0AB
:10FEA0000F94A049BC018FEA90E30E94AD45609198
:10FEB000550D7091560D8091570D9091580DDF9111
:10FEC000CF91FF90EF90DF90CF900C94D846DF91C8
:10FED000CF91FF90EF90DF90CF90089521E0209395
:10FEE000D8050F94253D1092D80508950E9430D56D
:10FEF0005CCF0E94F8E359CF20914206309143062F
:10FF00002115310559F081E0121613060CF080E03E
:10FF10008093D50510924306109242068091D50534
:10FF200008954F925F926F927F928F929F92AF92BD
:10FF3000BF92CF92DF92EF92FF920F931F93CF93D6
:10FF4000DF931F921F92CDB7DEB75C014A013901E2
:10FF500028018701760169837A83CEDFD82EE6D225
:10FF6000C82E69817A81811104C080912202882380
:10FF7000F9F092014D2DC5010E947C46CC20C1F0C4
:10FF8000DD2011F0F40101C0F3010F900F90DF911B
:10FF9000CF911F910F91FF90EF90DF90CF90BF9086
:10FFA000AF909F908F907F906F905F904F9019943B
:10FFB0000F900F90DF91CF911F910F91FF90EF90D5
:10FFC000DF90CF90BF90AF909F908F907F906F9079
:10FFD0005F904F900895FC0180810895FC01849109
:10FFE00008954F925F926F927F928F929F92AF92FD
:10FFF000BF92CF92DF92EF92FF920F931F93CF9316
:020000021000EC
:10000000DF936C017B015A012901672B31F08824B1
:100010008394912CC0E0D0E019C0F80111821082C5
:1000200027C03701680C791C76946794E301219707
:10003000A201BE01C601F50119951816190654F062
:10004000892BC9F04301FFEF8F1A9F0AE814F904C6
:1000500040F702C07E01FACFCE15DF0530F4CE01A5
:1000600002968816990620F02196F801D183C08364
:100070008FEF9FEF05C0F801D183C08380E090E04F
:10008000DF91CF911F910F91FF90EF90DF90CF9074
:10009000BF90AF909F908F907F906F905F904F90A8
:1000A00008958F929F92AF92BF92CF92DF92EF927C
:1000B000FF920F931F93CF93DF93EC016B017A01B3
:1000C000FB01199587FD06C0082F10E020E030E005
:1000D000219620C1982F907E903CC1F4082F0F717B
:1000E00010E020E030E04801590186E0880C991CBE
:1000F000AA1CBB1C8A95D1F7CE010196F601199571
:100100008F7395018401082B229604C1982F907F4C
:10011000903E19F58F70882E912CA12CB12C16E0F1
:10012000880C991CAA1CBB1C1A95D1F7CE0101960C
:10013000F60119958F73882A06E0880C991CAA1C71
:10014000BB1C0A95D1F7CE010296F60119958F7363
:1001500095018401082B2396DDC0982F987F903F4E
:1001600081F58770882E912CA12CB12CF6E0880C9B
:10017000991CAA1CBB1CFA95D1F7CE010196F60179
:1001800019958F73882AA6E0880C991CAA1CBB1CA1
:10019000AA95D1F7CE010296F60119958F73882A98
:1001A000B6E0880C991CAA1CBB1CBA95D1F7CE01ED
:1001B0000396F60119958F7395018401082B2496F7
:1001C000A9C0982F9C7F983FE9F58370882E912CC9
:1001D000A12CB12C56E0880C991CAA1CBB1C5A956A
:1001E000D1F7CE010196F60119958F73882A66E042
:1001F000880C991CAA1CBB1C6A95D1F7CE010296EB
:10020000F60119958F73882A76E0880C991CAA1C30
:10021000BB1C7A95D1F7CE010396F60119958F7321
:10022000882AE6E0880C991CAA1CBB1CEA95D1F729
:10023000CE010496F60119958F7395018401082B60
:10024000259668C0982F9E7F9C3F09F04AC0817018
:10025000882E912CA12CB12C86E0880C991CAA1C0C
:10026000BB1C8A95D1F7CE010196F60119958F73C3
:10027000882A96E0880C991CAA1CBB1C9A95D1F779
:10028000CE010296F60119958F73882A26E0880C14
:10029000991CAA1CBB1C2A95D1F7CE010396F60126
:1002A00019958F73882A36E0880C991CAA1CBB1CF0
:1002B0003A95D1F7CE010496F60119958F73882AE5
:1002C00046E0880C991CAA1CBB1C4A95D1F7CE01AC
:1002D0000596F60119958F7395018401082B2696D2
:1002E00019C0982F907C903849F4082F007C003872
:1002F00071F42196CE01F6011995F7CF082F0E7FE4
:100300000D3F28F02196CE01F6011995F7CF00E0B8
:1003100010E09801E114F10429F0F7010083118342
:1003200022833383CE01DF91CF911F910F91FF90F4
:10033000EF90DF90CF90BF90AF909F908F900895F7
:100340001F93CF93DF9300D01F92CDB7DEB710E09D
:10035000AE014F5F5F4F6BEE7FE7A3DE49815A81AD
:100360006B817C81452B462B472B11F01F5FF0CF13
:10037000812F0F900F900F900F90DF91CF911F91D1
:1003800008951F93CF93DF9300D01F92CDB7DEB7B0
:1003900010E0AE014F5F5F4F6EEE7FE782DE498176
:1003A0005A816B817C81452B462B472B11F01F5FB7
:1003B000F0CF812F0F900F900F900F90DF91CF9182
:1003C0001F910895FC01A081B1811C92A281B3818B
:1003D0008C918F5F8C930280F381E02D80816CE0A3
:1003E000689F600D112480E00C94B63B10923C068F
:1003F0008091370610923706882349F020E040E0CC
:1004000060E070E081EF97E665DB0C941944209181
:100410006502309166024091420650914306C9013F
:10042000840F951F2436310551F44730510514F0DF
:10043000069720C04A3F5F4F64F506961BC02436DE
:10044000310524F48536910524F504C084369105E0
:1004500024F41FC08A3091053CF0883E43E09407A5
:100460002CF087EE93E002C08AE090E0281739076D
:1004700031F40DC08A30910584F78AE090E09093C2
:1004800066028093650210924306109242060C9415
:10049000AB3C84E690E0E1CFCF93DF931F92CDB7E2
:1004A000DEB78091D908811103C08BE199E02FC09C
:1004B000211103C089ED98E02AC08DE0815048F0F9
:1004C000440F411DE82FF0E0E55EF64F908149278B
:1004D000F5CF80912E068417A9F040932E0689ED62
:1004E00098E069832DDF90E06981861B910997FF71
:1004F00002C080E090E080933F061092400688E0C2
:10050000809324028091400690E08752974F0F908D
:10051000DF91CF91089580933C0610923806109297
:10052000390610923A0610923B06089580913706DC
:100530001092370608957F928F929F92AF92BF924A
:10054000CF92DF92EF92FF920F931F93CF93DF939F
:10055000CDB7DEB728970FB6F894DEBF0FBECDBF7C
:100560007C014B016A015901FB0180816CE0689FAD
:10057000600D1124F7018081982F990F890F880F42
:100580000E94B63BC114D10409F496C0FE82ED82EC
:1005900098868F82011103C01C2D0D2D74C09D2CD7
:1005A0000C2D1D2DD12C88248394AE014F5F5F4FFD
:1005B000B5018C2D992D75DDC82E992E89819A81D2
:1005C000AB81BC81772473940097A105B105C9F074
:1005D000712C80329105A105B10581F0AC01BD01FE
:1005E0004D5251096109710942305105610571058A
:1005F00040F08B97A105B10589F503C0DD2009F412
:1006000055C0F70120818D2D90E0820F911D4697F6
:100610002CF0253018F0CE010596D4DE372D382584
:10062000D30EF70180818D0D8083DD2089F0DA946F
:10063000AE014F5F5F4FB501C80133DD8C016981A9
:100640007A818B819C814FEF5FEF0E94C13BEDCFA0
:10065000711032C00C2D192DD12CA7CFD3940115B8
:10066000110509F0A2CF0C2D192D9FCF4FEF5FEF91
:100670000E94C13BF70120812F5F2083253118F0B4
:10068000CE0105969FDEAE014F5F5F4FB501812F12
:10069000902F07DD182F092F69817A818B819C812A
:1006A000611571058105910509F706C00115110550
:1006B00089F20F5F1F4FD3CF28960FB6F894DEBF95
:1006C0000FBECDBFDF91CF911F910F91FF90EF90A3
:1006D000DF90CF90BF90AF909F908F907F900895C4
:1006E000AF92BF92CF92DF92EF92FF920F931F9340
:1006F000CF93DF931F921F92CDB7DEB75C016B01E2
:100700007A013FDE182FE114F10419F0C70139DE38
:1007100001C080E01A821982C114D104C1F4412FB2
:1007200050E090E09A01280F391F263131057CF402
:1007300025E130E0241B350B281B390B37FF02C0A5
:100740002F5F3F4F359527952A8381E0898301E00C
:100750002EEE3FE7A501BE016F5F7F4FCE010296EF
:10076000EADEC114D10489F08A81882321F01A823B
:1007700089818F5F898300E02BEE3FE7A601BE01F0
:100780006F5F7F4FCE010296D6DEE114F10451F087
:1007900000E02EEE3FE7A701BE016F5F7F4FCE0165
:1007A0000296C9DE0F900F90DF91CF911F910F91AC
:1007B000FF90EF90DF90CF90BF90AF900895CF92D1
:1007C000DF92EF92FF920F931F930E94B82F009138
:1007D0002A0610912B0620912C0630912D066B01D4
:1007E0007C01C01AD10AE20AF30AF7FC13C0209177
:1007F0002906209520932906DC01CB018A549C4FC1
:10080000AF4FBF4F80932A0690932B06A0932C06E0
:10081000B0932D0681E090912906911101C080E0EE
:100820001F910F91FF90EF90DF90CF900895CF939D
:1008300093E090932202811110924C060E94B82FEF
:10084000DC01CB018C509E4FAF4FBF4F80934606CB
:1008500090934706A0934806B093490668E873E171
:1008600082E090E00F94864FC6E0C15049F00F94AB
:100870001B4F62E070E080E090E00E94E92FF5CF2E
:10088000CF910895AF92BF92CF92DF92EF920F93E4
:100890001F93CF93DF9300D01F92CDB7DEB7809127
:1008A00023028F3F09F444C00E94B82F00912F0605
:1008B000109130062091310630913206DC01CB01D7
:1008C000801B910BA20BB30BB7FD32C09091770E3A
:1008D00080917A0E8F5F8F70981751F1E09123020B
:1008E00084E0E802F0011124EF57FC4F20E030E0F3
:1008F00040E752E460817181828193810F94A25517
:1009000069837A838B839C83A12CB12C6501E12CB4
:100910008E010F5F1F4F27E732E043E752E06FE69B
:1009200072E08BE692E00F9439038FEF80932302FD
:100930000F900F900F900F90DF91CF911F910F911B
:10094000EF90DF90CF90BF90AF9008950F931F93DB
:100950000E94B82F00914606109147062091480644
:1009600030914906DC01CB01801B910BA20BB30B2C
:10097000B7FD11C08091030181FB992790F981E0B7
:1009800089279091030192FF82609091000196FF68
:10099000846080934C0680914C06817090914C0647
:1009A00091FD826090911D06891741F18130A9F077
:1009B00028F0823041F0833059F01EC0913089F028
:1009C0009230A9F019C0992361F0933081F014C0DE
:1009D000913069F0923081F404C0992341F0933052
:1009E00059F49091410691509093410605C0909121
:1009F00041069F5F9093410680931D061F910F91C2
:100A00000895CF93DF930E941944E4E0F1E08081E0
:100A10008D7F8083C5E0D1E088818095827043E03E
:100A200051E0DA018C9380818B7F8083888180956F
:100A300084708C9321E031E0D9018C918F7B8C9371
:100A400080910201809580748093000180818E7F67
:100A50008083888180958170FA01808382E0809311
:100A60004B0674DF10924106DF91CF910895CF932A
:100A7000C09192068EE496E063DCC81790F48091F2
:100A800092068F5F21E0280FE82FF0E0E25BF94F3C
:100A90009081907C903811F4822FF4CF809392064D
:100AA00002C010929206CF9108950F931F93CF9397
:100AB000DF938C01C0919206D0E0C25BD94FCE018A
:100AC0003FDCF8018083CE01DF91CF911F910F9120
:100AD000089581E090914E06911101C080E0089543
:100AE000CF93DF9320919106211120C0FC0101904A
:100AF0000020E9F73197EF01C81BD90BC334D105AA
:100B000034F031972081207C2038D9F3F4CFBC0118
:100B1000DD27AE018EE496E00F94485EC25BD94FAC
:100B200018821092920683E080932202DF91CF9187
:100B30000895CF93DF93CDB7DEB78E819091910664
:100B4000891790F0809391069E01275F3F4F4F8158
:100B5000588562E470E08EE496E00F94915E109206
:100B6000920683E080932202DF91CF9108950F9344
:100B70001F93CF93DF938C0167FF03C01092910600
:100B800060E08091910690E0262F062E000C330B3A
:100B9000281739071CF160939106C8010F94AA5DCC
:100BA000F801E80FF91FEF01C01BD10BC334D105C9
:100BB00034F031978491807C8038D9F3F4CFDD27ED
:100BC000AE01B8018EE496E00F94CB5DC25BD94FC5
:100BD00018821092920683E080932202DF91CF91D7
:100BE0001F910F9108954F925F926F927F928F9213
:100BF0009F92AF92BF92CF92DF92EF92FF920F93AC
:100C00001F93CF930E94B82F6B017C013BDE9EDEC9
:100C100080914C0682FF15C080912806811113C077
:100C200091E0909328062091D316211103C0809162
:100C3000D8058927809337061092D31681E0F7DD17
:100C400002C010922806C0910301C095C170809126
:100C50004B06C81779F10E94C743882359F11091B8
:100C60004B06C0934B06CC2309F4CAC164EF71E074
:100C700080E090E00E941CA30E945492123009F080
:100C8000BAC10E942B930E94194483E080932202F0
:100C90000E94B82F6B017C01DC01CB018C599F4F66
:100CA000AF4FBF4F8093240690932506A09326064E
:100CB000B09327068091240690912506A0912606E0
:100CC000B0912706A7019601281B390B4A0B5B0B35
:100CD00057FF05C080914506882309F41FC2D7013C
:100CE000C6018C599F4FAF4FBF4F809324069093FE
:100CF0002506A0932606B093270660914106062E8E
:100D0000000C770B77FF03C0719561957109062E72
:100D1000000C770B880B990B0F943D562B013C016F
:100D200020E030E040E050E40F949E5787FF05C07C
:100D30008091370681117DC08DC080913C0688234B
:100D400009F456C08090380690903906A0903A0673
:100D5000B0903B0681149104A104B104E1F120E0BC
:100D600030E040E05FE3C301B2010F94D9572B019B
:100D70003C01C701B601681979098A099B090F94DA
:100D80003B569B01AC01C301B2010F94A25520E078
:100D900030E04AE754E40F94D9574B015C0120E05E
:100DA00030E040EA52E40F949E5787FF0FC020E0E6
:100DB00030E040EF51E4C501B4010F949E5787FD28
:100DC0000AC02AE030E040E050E009C024E630E00C
:100DD00040E050E004C021E030E040E050E0C0924C
:100DE0003806D0923906E0923A06F0923B0604C0EB
:100DF00021E030E040E050E0A09141060091420641
:100E0000109143060A2E000CBB0B0F944A5922E0A6
:100E100030E040E050E00F940759DA01C901800F3B
:100E2000911FA11DB11D909343068093420610921D
:100E30004106D701C6018856954CAF4FBF4F8093EE
:100E4000200690932106A0932206B093230681E00A
:100E50008093220220913D0630913E0641E8263FD4
:100E6000340741F480912402882309F4D4C08150CE
:100E7000809324022C54334651F580912402882318
:100E800021F081508093240222C084E080932402C8
:100E9000809140068F5F8093400690913F0698179F
:100EA00028F4109240068CE08093240281E0809325
:100EB0002202D701C6018856954CAF4FBF4F809391
:100EC000200690932106A0932206B09323068091DA
:100ED0006F0081FB222720F981FF05C080916F0000
:100EE0008D7F80936F008091890D90918A0DA091E4
:100EF0008B0DB0918C0D222329F020916F00226080
:100F000020936F003AE0B695A795979587953A9507
:100F1000D1F7009721E0A207B10520F08FEF9FEFF6
:100F2000A0E0B0E09695879520912202211105C09E
:100F3000309145063111EEC051C0009741F040910B
:100F40001E0650911F064817590708F047C08091A8
:100F50004506811117C0223008F06DC080914D0404
:100F6000811107C081E080934D0484E194E00E94E8
:100F70008B3484E194E00E94C23481E08093440683
:100F80008093450683E00E94AC4361E084E194E0F5
:100F90000E94EB34E0913D06F0913E0619951092C7
:100FA000440680914506811152C0109237060E9476
:100FB000B82FDC01CB018C199D09AE09BF09009146
:100FC0001E0610911F0620E030E0081719072A07B7
:100FD0003B0720F490931F0680931E0680913D06E8
:100FE00090913E06865F914809F457C080914A0669
:100FF000811153C07EC060E088E391E3B8DD43CE49
:10100000ECD5123009F43FCE60E08AE291E3AFDD27
:101010000E94967D38CE8CE08093240280911E063B
:1010200090911F06019790931F0680931E0681E002
:10103000809322021FCF243030F0243009F08ECF6D
:10104000109222028BCF81E08093220287CF84E12D
:1010500094E00E94C63491E0811101C090E0909329
:101060004506992309F4A1CF0E94B82FDC01CB01DA
:101070008C199D09AE09BF09C0901E06D0901F06AD
:10108000E12CF12CC816D906EA06FB0608F046C08A
:1010900090931F0680931E0641C048E9C40E4AE3A0
:1010A000D41EE11CF11CC0922006D0922106E092D1
:1010B0002206F09223068091450681112FC080916F
:1010C0002202813099F0833049F5CF911F910F9121
:1010D000FF90EF90DF90CF90BF90AF909F908F9058
:1010E0007F906F905F904F900C944A441092220230
:1010F00015C08091200690912106A0912206B09102
:101100002306C81AD90AEA0AFB0AF7FCD4CF0E94C0
:10111000967DD1CF009709F435CF11CFCF911F9194
:101120000F91FF90EF90DF90CF90BF90AF909F9086
:101130008F907F906F905F904F90089561E017DDE2
:101140000C94967DCF93DF931F921F92CDB7DEB79D
:1011500089839A8356DC89819A81F0DF0F900F9002
:10116000DF91CF910C941E448091280982FD05C027
:101170008091C616823061F410C08091D908811127
:1011800003C08BE199E002C089ED98E061E0A8CC52
:10119000813031F08DEF90E305C08DE191E302C025
:1011A00081E191E36FEFE3CC1092D316109292029B
:1011B000809128098064809328090E9476B20F9458
:1011C000CD4F60E08FEE90E3D2DC0C94967D83EE01
:1011D00090E30E947A7E60E086ED90E3C8DC40E018
:1011E00061E080E00E9481678CEC90E30D94203DEB
:1011F000BBDF1092D316109292020E94E3678823FD
:1012000021F08091280982FF04C00E946EB20D94E3
:10121000465088EC90E30F94203DF7CF8091280949
:1012200082FF2AC00E94E367882319F18091E306B8
:101230009091E406A091E506B091E6060097A1051D
:10124000B105B9F0BC01CD016D597F4F8F4F9F4F54
:1012500024E630E040E050E00F94E5586091DF066E
:101260007091E0068091E1069091E2060F94E558B6
:1012700001C020E020934D0680914D068F770895A0
:1012800086EF91E890933E0680933D06089561E0D5
:10129000FC0180810E94E8318FEF0C940EA4CF9363
:1012A000DF93EC018A810E94D0A360E08881DF9106
:1012B000CF910C94E8318F929F92AF92BF92EF92B0
:1012C000FF920F931F93CF93DF93EC018B017A0171
:1012D0000E94B82F4B015C012CE2820E21E0921E8D
:1012E000A11CB11C0E94E8A38B838F3F61F40E9474
:1012F000B82FDC01CB0188199909AA09BB09B7FDF0
:10130000F1CF81E10DC08E3F51F4B701C8010E94B9
:10131000EFA30E94E8A30E94E8A311E003C08FE0BE
:10132000898310E0CE01B3DF812FDF91CF911F9130
:101330000F91FF90EF90BF90AF909F908F90089586
:10134000CF92DF92EF92FF926A017B010E94B82F49
:10135000C60ED71EE81EF91E0E94E8A38F3F61F05B
:101360000E94B82FDC01CB018C199D09AE09BF0981
:10137000B7FDF2CF80E001C081E0FF90EF90DF90F9
:10138000CF900895EF92FF921F93CF93DF9300D0F9
:101390001F92CDB7DEB77C01162F29833A834B838A
:1013A0005C837DDF48E552E060E070E0C701C8DFA4
:1013B000812F80640E940EA48C810E940EA48B81D8
:1013C0000E940EA48A810E940EA489810E940EA40C
:1013D000112311F087E801C085E90E940EA41C309A
:1013E00011F40E94E8A310E00E94E8A3F7018383B0
:1013F00087FF04C01F3F11F01F5FF6CF0F900F90C3
:101400000F900F90DF91CF911F91FF90EF90089573
:101410008F929F92AF92BF92CF92DF92EF92FF9204
:101420000F931F93CF93DF93EC01162F1C82198229
:1014300048830E94B82F6B017C0120EDC20E27E08B
:10144000D21EE11CF11CA89561E088810E94E83160
:1014500061E088810E94AC310E94E1A385E08A832B
:101460000E94D0A30AE08FEF0E940EA40150D9F78A
:10147000A89520E030E0A90160E0CE0183DF8B83F6
:10148000813061F00E94B82FDC01CB018C199D09DD
:10149000AE09BF09B7FDEDCF81E055C0A8952AEA96
:1014A00031E040E050E068E0CE016CDF853011F4BF
:1014B00081E009C004E00E94E8A38B830150D9F7C2
:1014C0008A3A51F482E08C83A8958C81823081F035
:1014D000812C912C540111C00E94B82FDC01CB014A
:1014E0008C199D09AE09BF09B7FDD9CF82E02BC089
:1014F000812C912CA12C80E4B82E20E030E0A901B1
:1015000067E3CE013FDFA501940169E2CE013ADF36
:101510008B83882361F00E94B82FDC01CB018C19EA
:101520009D09AE09BF09B7FDE8CF8AE00CC08C81E8
:101530008230D1F420E030E0A9016AE3CE0122DF5D
:10154000882329F088E08983CE01A1DE16C00E949D
:10155000E8A3807C803C11F483E08C830E94E8A3A4
:101560000E94E8A30E94E8A3CE0191DE173018F490
:101570001A8381E003C088E1898380E0DF91CF9105
:101580001F910F91FF90EF90DF90CF90BF90AF90A1
:101590009F908F9008950F931F93CF93DF93EC014B
:1015A00089018C81833039F089E0440F551F661F13
:1015B000771F8A95D1F79A01AB0161E1CE01E2DE96
:1015C000811109C040E052E0B801CE01DF91CF9116
:1015D0001F910F9170CE84E08983CE0158DE80E0A8
:1015E000DF91CF911F910F910895CF93DF93EC017D
:1015F000862FBA010E9413A48FEF0E940EA48FEFD2
:101600000E940EA40E94E8A38B83982F9F719530AF
:1016100031F083E18983CE013ADE80E001C081E0D0
:10162000DF91CF9108950F931F93CF93DF93EC0138
:1016300089018C81833039F089E0440F551F661F82
:10164000771F8A95D1F79A01AB0168E1CE019ADE46
:1016500081111EC0A8016EEFCE01C7DF8823E1F023
:1016600048E552E060E070E0CE016ADE882371F068
:1016700020E030E0A9016DE0CE0184DE81110AC0D6
:101680000E94E8A3811106C011E007C087E103C0F2
:1016900086E001C086E1898310E0CE01F8DD812F6C
:1016A000DF91CF911F910F910895CF93DF931F92F8
:1016B000CDB7DEB72091D5163091D616CE01019662
:1016C0002115310519F0821B930B02C08B5D9641E9
:1016D0000F90DF91CF910895FC01238121110C948B
:1016E000959C089583E996E0F7CF8EEA96E0F4CFD3
:1016F0008091C906811107C00E94F8E3882319F080
:1017000081E08093C906089580912809847F8B7FAA
:10171000809328091092DF061092E0061092E106ED
:101720001092E2061092E3061092E4061092E5068B
:101730001092E60610925407109293078EE091E003
:10174000E4E9F7E0DF019C011D9221503040E1F710
:101750008FEF8093D8080895FC0120E03EE2DB0182
:101760004C91403241F0283011F430833196DB0146
:101770004C91408331962F5F6F5F7F4F2B3079F70D
:10178000108208952F923F924F925F926F927F92B4
:101790008F929F92AF92BF92CF92DF92EF92FF9281
:1017A0000F931F93CF93DF93CDB7DEB7C356D10905
:1017B0000FB6F894DEBF0FBECDBF8C015B014A01AE
:1017C0004DB65EB6312C7E0187E5E80EF11C9BE13B
:1017D000292E49ED58E0BE016F5F7F4FC5010E9481
:1017E000059B18160CF005C18C85282F2871203117
:1017F00009F074C09091DE069150923008F46EC0EA
:101800006DB67EB6BE016F5F7F4FC701A5DF0115C4
:10181000110521F0F8018081811173C021E081E080
:1018200090E0F70101900020E9F73197EE19FF09E8
:10183000E80FF91F32968DB79EB78E1B9F0B0FB620
:10184000F8949EBF0FBE8DBFEDB7FEB731966F0106
:10185000211102C0B80102C061E973E0C6010F9412
:10186000335EB701C6010F941D5E61E973E0C601E6
:101870000F941D5E1CAE1FAE21E0A701B501CE0185
:10188000CC960E94919E81110DC08091DE0681113F
:1018900009C00E944EA38AE393E30E9440A3C701BC
:1018A0000E9446A9FE01FC96DE019196822D0190D0
:1018B0000D928A95E1F740E050E0BE016F5D7F4FE9
:1018C000C60160DFCE01819607DFCE01CC9604DF32
:1018D0000FB6F8947EBE0FBE6DBE7BCF9981992363
:1018E00009F487C0953E09F474CF9E3209F471CF94
:1018F0009091D9089E3209F46CCF8A7009F069CFB3
:101900000AC0F80101900020E9F73197CF01801B50
:10191000910B20E086CF81E0203109F080E09091AA
:10192000280980FB94F990932809811108C08985C2
:10193000873409F04ECF8A858E3709F44ACF8091DB
:10194000DE06813021F068F08230B9F142CF80911B
:10195000DC069091DD0601969093DD068093DC060F
:1019600038CFBE016F5F7F4F8BE199E0F5DE011547
:10197000110511F0680105C08BE1C82E89E0D82E51
:1019800008C0F60181916F018823B1F30E94EFA88E
:10199000F8CFF60181916F01882319F00E94EFA81A
:1019A000F8CF80E20E94EFA86D8D7E8D8F8D98A17B
:1019B0004AE050E00E94FCA90CCFBE016F5F7F4F50
:1019C0008BE199E0C9DE8114910441F06BE179E08B
:1019D000C4010F940A5E892B51F40BC0832D90E053
:1019E0002091DA063091DB068217930711F03394C9
:1019F000F0CE0FB6F8945EBE0FBE4DBECD59DF4F90
:101A00000FB6F894DEBF0FBECDBFDF91CF911F910F
:101A10000F91FF90EF90DF90CF90BF90AF909F908D
:101A20008F907F906F905F904F903F902F90089590
:101A3000CF93DF93CDB7DEB76B970FB6F894DEBFC9
:101A40000FBECDBF1092DE0640E050E0BA018DEB34
:101A500098E00E94B49B8BE1EDEBF8E0DE0111967B
:101A600001900D928A95E1F740E050E0BE016F5F72
:101A70007F4F80E090E086DECE0101962DDE6B96F2
:101A80000FB6F894DEBF0FBECDBFDF91CF910895A2
:101A90000F931F93CF93DF93CDB7DEB72D970FB67C
:101AA000F894DEBF0FBECDBF80915807882391F018
:101AB000BE016F5F7F4F85E597E00E9427998E01F9
:101AC0000F5F1F4FF80181918F01882339F00E9429
:101AD000EFA8F8CF80E393E30E9440A38AE00E943E
:101AE000EFA82D960FB6F894DEBF0FBECDBFDF91E5
:101AF000CF911F910F910895CF92DF92EF92FF92B5
:101B00000F931F93CF93DF93CDB7DEB7EDB6FEB63D
:101B1000DC010D900020E9F79D01281B390B2C5F9B
:101B20003F4F4DB75EB7421B530B0FB6F8945EBFE5
:101B30000FBE4DBF0DB71EB70F5F1F4F9F938F9303
:101B40008AEE92E39F938F931F930F930F94625E9D
:101B5000680154E0C50ED11C0F900F900F900F90AC
:101B60000F900F90F6018081882349F0082E000C19
:101B7000990B0F948E5DF60181936F01F3CFC8012D
:101B80000F94253D86EE92E30F94333D0FB6F89403
:101B9000FEBE0FBEEDBEDF91CF911F910F91FF9062
:101BA000EF90DF90CF9008958091280983FF03C0C4
:101BB00084608093280908951092F50B809128097C
:101BC0008F7B8B7F809328090E94E367882321F015
:101BD00085E597E00C94959C0895EEDF80912809A7
:101BE000877F8093280908950F931F93CF93DF93E6
:101BF0008B01EA01DB016D917C910E942799D8014C
:101C0000ED91FC919081888191110EC08936B0F4DC
